:100000000C94AC0B0C94E4720C94B9720C948E7238
:100010000C9463720C9438720C940D720C94E2710F
:100020000C94B7710C94DD0B0C94DD0B0C94BA742A
:100030000C94DD0B0C94DD0B0C94DD0B0C94DD0BA0
:100040000C94DD0B0C94DD0B0C94DD0B0C94DD0B90
:100050000C943C730C94DD0B0C94DD0B0C946D71C3
:100060000C94DD0B0C94DD0B0C94DD0B0C94DD0B70
:100070000C94DD0B0C94DD0B0C94DD0B0C94DD0B60
:100080000C94DD0B0C94DD0B0C94DD0B0C940F73B6
:100090000C94DD0B0C94DD0B0C94DD0B0C9496731F
:1000A0000C94DD0B0C94DD0B0C94DD0B0C94DD0B30
:1000B0000C94DD0B0C9440710C94DD0B0C94DD0B57
:1000C0000C94DD0B0C94DD0B0C9469730C94DD0B1C
:1000D0000C94DD0B0C94DD0B0C94DD0B0C94DD0B00
:1000E0000C94DD0B07634236B79BD8A71A396856C4
:1000F00018AEBAAB558C1D3CB7CC5763BD6DEDFD4A
:10010000753EF6177231BF000000803F0800000006
:10011000BE922449123EABAAAA2ABECDCCCC4C3EFC
:1001200000000080BEABAAAAAA3E00000000BF00EB
:100130000000803F0000000000084178D3BB4387E7
:10014000D1133D190E3CC3BD4282AD2B3E68EC82FB
:1001500076BED98FE1A93E4C80EFFFBE01C4FF7F80
:100160003F00000000000C94566F0C94F9280C948A
:1001700023290C94727A0C94D4240C9408290C949E
:100180002B280C947B5C0C9436580C94B2700C9415
:10019000607A0C9443260C94F4670C94D1790C94F7
:1001A000DF0B0C9443230C94A9680C94DD670C942A
:1001B000787A0C94EF660C949D6D0C94116F0C94EE
:1001C000055E0C940F650C9489660C947B3C0C9432
:1001D000756E0C94F1280C9411290C943A0F0C9420
:1001E000C86E0C9468590C94817A0C94FB450C945D
:1001F000911D0C941A360C941A290C941B650C94BE
:1002000079350C943E0F0C94A4590C9412670C94FD
:10021000306C0C943F270C943D100C94A95B0C940B
:1002200014290C94A56F0C941D290C94F7580C9468
:100230006A650C94847A0C94EF5D0C94B3240C944E
:100240001E6E0C94877A0C94A45A0C944A5A0C94FF
:100250004A620C94866D0C94B86C0C9491610C9469
:10026000EB260C9401270C94B7260C94196C0C9473
:10027000156A0C94E4270C9421400C94F2630C94BE
:10028000C9340C94C9700C941B5E0C94E5620C94F8
:10029000A7390C94FF670C94345A0C948C6E0C9410
:1002A000FD2A0C9474690C94030F0C94180F0C9491
:1002B000786A0C94916B0C94D1380C948E3A0C940F
:1002C000220F0C94D7280C94F26A0C940D0F0C9406
:1002D000252A0C94757A0C94D8600C9442100C94D6
:1002E0009E650C94667A0C940A6A0C94B46D0C9416
:1002F000BE5C0C948B690C94A41F0C945A7A0C94D9
:10030000044B0C94480F0C94EE5B0C947D5D0C94A4
:10031000355C0C94F8640C94645D0C94EE3B0C9486
:10032000C1790C9427640C94BF550C9484590C9497
:100330007E7A0C944E5D0C94517A0C9472660C94F7
:100340004E700C9466660C945A660C94B4240C940B
:1003500005290C94EA6D0C94ED220C94DC690C9444
:10036000637A0C9416230C94B36B0C94F5390C94AB
:10037000E96C0C9414570C94454D0C94F3280C9490
:10038000FC580C94696C0C94CC760C9417290C9442
:1003900029670C946D6F0C9444100C94D65D0C94EA
:1003A0009E2B0C94146B0C941E0F0C94A05F0C9459
:1003B000E8450C94746C0C945D690C941C590C9475
:1003C000697A0C94577A0C94226D0C94FB700C94FF
:1003D000A86B0C9471350C94430F0C940E290C945B
:1003E000D26C0C94C1460C94F6280C945D7A0C9453
:1003F000345B0C94BA590C94DD270C9443100C9484
:1004000069290C946F7A0C94096B0C94C5690C944F
:10041000FC620C94FC280C9446570C948A7A0C9439
:10042000076E0C9464440C94FF280C9421470C94A0
:10043000547A0C9472460C94E44B0C94150F0C9463
:100440004E460C94B45B0C94BE360C94BC680C9471
:1004500085640C94593B0C94AE690C94110F0C9468
:100460000B5F0C9420290C945D360C945D380C9431
:100470002B4B0C94440F0C940B290C94CD5B0C94D7
:10048000280F0C940F230C9471630C943E3F0C9432
:10049000360F0C9406670C94325E0C944B5C0C94F3
:1004A000300F0C948D7A0C943A610C94E8330C94D0
:1004B00037700C942C0F0C94616A0C9494670C9414
:1004C000C0290C94090F0C94EC610C9436650C94C3
:1004D00007270C945F570C947B7A0C94396D0C941D
:1004E00097690C9439100C94325D0C94CD6D0C947A
:1004F000836A0C9490620C9448640C949B350C9421
:1005000002290C94BD5A0C946C7A0C94B0440C944F
:10051000E4580C94F3690C9441100C94D85B0C943F
:10052000FC220C9405660C94286F0C94EE650C94D8
:10053000C4870C9490460C9448560C9474600C94A8
:100540006E64532A00572A005375005361004672A7
:10055000005468005765005475004D6F00435552B4
:10056000564520494E5600466572743A2569004644
:100570003A25730044494D2D3E25692525002A2A38
:100580000048454154494E4700542D53453A257380
:1005900000542D52443A25730054454D502D48497E
:1005A00047480054454D502D4C4F5700252D397369
:1005B000202533692525002532693A253032692006
:1005C000202532692E253032690058583A2D2D2DBC
:1005D0002D2D2D2D2D00253032693A252D38730013
:1005E0005058583A2D2D2D2D2D2D2D2D00A7C500FD
:1005F00000CA1A0100037A0100B4F00100969002CB
:1006000000EF7A0300FAFB04008CF707008FDF107D
:100610000045565420454E545259007E2569257395
:1006200020253032693A2530326920252D36730A6B
:100630002531367300252D3873252D387300437509
:100640007276650020257320746F20253032692D65
:10065000253032697E30004C696D69740050253058
:10066000326920253032692E253032696D6C402583
:100670003033696D6C0046657274696C0025322EEA
:10068000327320253032692E253032696D6C402559
:100690003033696D6C0025362E367300253369259D
:1006A0002520696E20253369204D696E200044693C
:1006B0006D002573002531362E3136730025730009
:1006C0004E6F2076616C6964204576656E74004ECD
:1006D0006F204576656E747320666F756E640025B5
:1006E0003032693A252D387300252D387300434187
:1006F0004C2D554E53414645003230253032692D40
:10070000253032692D253032697E256925303269E0
:100710003A253032690A7E25692534733A252D3908
:100720007300455252005741524E00494E464F0009
:100730005468657265206172650A6E6F206D65731D
:100740007361676573004C6F7765723A202430617E
:100750007B2532692C31352D33357D7E300A55703D
:100760007065723A202431617B2532692C31362D37
:1007700034307D7E3000253032693A252D387300C3
:1007800058583A2D2D2D2D2D2D2D2D005025303240
:10079000693A252D387300252D3132732024306CB1
:1007A0007B7E25692C7D0A50756D7065643A202426
:1007B00031617B3030302C302D3235357D6D6C0021
:1007C00050756D703A0A24306F7B252D3132732CB1
:1007D0007D00446F73696E672050756D700A4361C8
:1007E0006C6962726174696F6E00506F727420245C
:1007F000306D7B252D3131732C25697D0A436E7454
:100800003A202431617B253032692C302D31357D01
:10081000204163743A2432647B252D34732C7D008F
:10082000446F73696E672050756D700A506F7274F3
:10083000730050253032693A202430657B25632CC3
:10084000205F412D5A612D7A302D397D2431657B11
:1008500025632C205F412D5A612D7A302D397D245E
:1008600032657B25632C205F412D5A612D7A302D16
:10087000397D2433657B25632C205F412D5A612D02
:100880007A302D397D2434657B25632C205F412D02
:100890005A612D7A302D397D2435657B25632C20D6
:1008A0005F412D5A612D7A302D397D2436657B25A7
:1008B000632C205F412D5A612D7A302D397D2437EC
:1008C000657B25632C205F412D5A612D7A302D39AF
:1008D0007D0053656C65637420506F72743A0A240E
:1008E000306D7B252D3131732C25697D0045646980
:1008F0007420506F72740A4E616D657300526563A7
:100900006F766572205374617465206F6E0A52654C
:10091000626F6F743A202430647B252D33732C7DF5
:10092000005265636F766572205374617465206F41
:100930006E0A5265626F6F74004163746976653A3E
:10094000202430647B252D34732C7D0A2431647B74
:10095000252D33732C7D2077697468696E204C696E
:100960006D69740048656174657220506F72740A15
:1009700024306D7B252D3131732C25697D00486530
:10098000617465720A53657474696E67730024300C
:10099000677B20202054616E6B2C54616E6B7C53FE
:1009A000756D707C416D6269656E747D20706F72CB
:1009B000743A0A24316D7B252D3131732C25697DE4
:1009C0000054656D70657261747572650A53656E69
:1009D000736F7220506F7274730054656D7065721E
:1009E00061747572650A416C657274730053756D3C
:1009F000700054616E6B004E6F205461736B0A730C
:100A000063686564756C6564005363686564756CE0
:100A10006564205461736B0054656D706F72617210
:100A200079205461736B004578697374696E67202F
:100A30005461736B00457865637574652054617308
:100A40006B002430637B20202020202020202020C9
:100A5000202020202020200A2020202020202020AC
:100A600020202020202020202C7D004E6F2054614B
:100A7000736B0A617661696C61626C650052656DC9
:100A80006F7665205461736B0054656D70204C69FE
:100A90006D697473206F660A2430677B25732C544C
:100AA000616E6B7C53756D707D3A202431617B25BE
:100AB0003032692C31352D33347D202D20243261A4
:100AC0007B253032692C31362D33357D7E30005414
:100AD000656D70657261747572650A4C696D6974D3
:100AE000730024306F7B252D3132732C7D0A243125
:100AF000617B253032692C302D36337D2C243261D8
:100B00007B253032692C302D37357C32357D6D6C4C
:100B1000402433617B253033692C312D3235357DCE
:100B20006D6C2F6D6E0046657274696C697A650034
:100B30002430647B204C4F572C7D2024316D7B2545
:100B40002D3131732C7D0A746F2024326D7B252D5D
:100B50003131732C7D0053776974636820506F7254
:100B600074730044696D20746F202430617B2530DC
:100B700033692C302D3130307D25250A696E2024D3
:100B800031617B253033692C302D3235357D206D38
:100B9000696E757465730054656D70657261747506
:100BA00072650A4C696D69747300437572766520CD
:100BB0004F766572726964650046657274696C6926
:100BC0007A650044696D204C6967687400537769E1
:100BD00074636820506F727473005265636F76653A
:100BE00072205461736B730045646974205461739F
:100BF0006B0044696D204C69676874002430647B25
:100C00007E25632C7D205745454B4441592048485B
:100C10003A4D4D0A20202020202431627B25732C60
:100C20007D2020202432617B253032692C302D320A
:100C3000337C317D3A2433617B253032692C302D71
:100C400035397C317D0024306B7B252D3131732C7F
:100C50007D0A24316A7B252D38732C7D20413A246E
:100C600032647B252D34732C7D00437572766520AC
:100C70004F766572726964650041646420546173E3
:100C80006B004E6F20737061636521204576656E41
:100C9000740A4C696D697420726561636865642EBD
:100CA0000059592D4D4D2D4444202048483A4D4D72
:100CB0000A2432617B253032692C302D39397D2D63
:100CC0002431617B253032692C312D31327D2D2448
:100CD00030617B253032692C312D33317D20202449
:100CE00033617B253032692C302D32337D3A243408
:100CF000617B253032692C302D35397D0053657488
:100D0000204461746500436F6E6669726D20746F74
:100D10000A726573746172740052657374617274DF
:100D20000053696E6365203230253032692D2530DD
:100D300032692D253032690A2D3E2535696420251A
:100D40003032696820253032696D00557074696DE4
:100D5000650052656D6F766520616C6C0A4D657338
:100D600073616765730052656D6F7665204D6573BD
:100D700073616765005468657265206172650A6E0B
:100D80006F206D65737361676573002430667B2522
:100D9000732C7D004D6573736167657300416D62EF
:100DA00069656E743A202532692E253032697E30AD
:100DB0000A25730053756D703A202532692E25304F
:100DC00032697E3025730A446576696174696F6E95
:100DD0003A2025346925250054616E6B3A2025326E
:100DE000692E253032697E3025730A446576696143
:100DF00074696F6E3A2025346925250054656D703D
:100E0000657261747572650A53656E736F727300F3
:100E1000322E3020402031323A35333A30360A4DC6
:100E20006179203134203230323600566572736970
:100E30006F6E005461736B733A2025690A52656DB9
:100E400061696E696E673A202569005461736B2091
:100E500053746F726167650050574D20467265711B
:100E600075656E63793A0A2569487A00496E666F3E
:100E7000726D6174696F6E73004578706F6E656E28
:100E8000743A0A2430617B2531692C302D337D2E54
:100E90002431617B2531692C30302D39357C357D0D
:100EA0000049443A2430657B25632C412D5A302D6E
:100EB000397D2431657B25632C20412D5A302D3915
:100EC0007D2432657B25632C20412D5A302D397DC0
:100ED0002433657B25632C20412D5A302D397D2408
:100EE00034657B25632C20412D5A302D397D2435E6
:100EF000657B25632C20412D5A302D397D243665A4
:100F00007B25632C20412D5A302D397D2437657B7C
:100F100025632C20412D5A302D397D002431306A33
:100F20007B252D38732C7D004E6F204375727665BE
:100F30000A617661696C61626C65004175746F0A63
:100F400028766961204578706F6E656E742900415E
:100F500075746F0A28766961204578706F6E656ECA
:100F60007429004639302525202031303025250AC6
:100F70002430687B253034692C302D383030307D7A
:100F8000202431687B253034692C302D38303030C6
:100F90007D00463630252520203730252520203875
:100FA0003025250A2430687B253034692C302D38D3
:100FB0003030307D202431687B253034692C302D51
:100FC000383030307D202432687B253034692C3035
:100FD0002D383030307D0046333025252020343008
:100FE00025252020353025250A2430687B253034FE
:100FF000692C302D383030307D202431687B25300D
:1010000034692C302D383030307D202432687B25F7
:101010003034692C302D383030307D00462030257A
:10102000252020313025252020323025250A243066
:10103000687B253034692C302D383030307D2024C9
:1010400031687B253034692C302D383030307D20AC
:101050002432687B253034692C302D383030307D97
:1010600000523830252520393025252031303025D3
:10107000250A202430697B253033692C302D31300E
:10108000307D202431697B253033692C302D31307F
:10109000307D202432697B253033692C302D31306E
:1010A000307D00523430252520353025252036303E
:1010B000252520373025250A202430697B2530332B
:1010C000692C302D3130307D202431697B2530333F
:1010D000692C302D3130307D202432697B2530332E
:1010E000692C302D3130307D202433697B2530331D
:1010F000692C302D3130307D0052203025252031B3
:10110000302525203230252520333025250A20247E
:1011100030697B253033692C302D3130307D2024EF
:1011200031697B253033692C302D3130307D2024DE
:1011300032697B253033692C302D3130307D2024CD
:1011400033697B253033692C302D3130307D0049B7
:10115000443A2430657B25632C412D5A302D397D4E
:101160002431657B25632C20412D5A302D397D2477
:1011700032657B25632C20412D5A302D397D243357
:10118000657B25632C20412D5A302D397D24346513
:101190007B25632C20412D5A302D397D2435657BEC
:1011A00025632C20412D5A302D397D2436657B2531
:1011B000632C20412D5A302D397D2437657B2563E2
:1011C0002C20412D5A302D397D002431396A7B2560
:1011D0002D38732C7D004E6F2043757276650A6141
:1011E0007661696C61626C650052656D6F76652031
:1011F0004375727665004D616E75616C0A2876697B
:101200006120506F696E74732900456469742043CE
:1012100075727665004D616E75616C0A287669613C
:1012200020506F696E7473290041646420437572A5
:1012300076650041737369676E204C4544204469AC
:101240006D0A43757276657320746F20506F7274E7
:1012500073004C45442044696D0A4375727665738A
:101260000043757276653A2024306A7B252D3873E9
:101270002C7D0A4163746976653A202431647B25AC
:101280002D34732C7D004E6F2043757276650A6194
:101290007661696C61626C6500506F72743A0A2401
:1012A000306B7B25732C7D0050574D204672657145
:1012B00075656E63793A0A2430687B2534692C3170
:1012C00032352D313030307C3132357D487A004432
:1012D000696D6D696E670A50574D2046726571756C
:1012E000656E63790041646170743A202430647BD8
:1012F000252D33732C7D0A4F66662D5374617465FA
:101300003A202431647B252D34732C7D004C4544D8
:101310002044696D6D65722053746174650A576865
:10132000656E20506F7765726564204F6666005267
:10133000656D6F7665204C45442D44696D0A506F8C
:1013400073742D46696E697368205461736B004C29
:1013500045442044696D6D65720A506F73742D4663
:10136000696E697368205461736B0052656D6F76A6
:1013700065204C45440A5072652D53746172742087
:101380005461736B002430647B252D34732C7D20D5
:1013900024316D7B252D3131732C25697D0A746FC5
:1013A0002024326D7B252D3131732C25697D00245D
:1013B00030647B252D34732C7D2024316D7B252DCD
:1013C0003131732C25697D0A746F2024326D7B25A1
:1013D0002D3131732C25697D004C45442044696DC5
:1013E0006D65720A5072652D537461727420546178
:1013F000736B0024306D7B252D3131732C25697D75
:101400000A4163746976653A202431647B252D3462
:10141000732C25697D004C454420506F7765720A16
:10142000506F7274005254432054656D703A2025F9
:1014300032692E253032697E300A4F6666736574D4
:101440003A202430647B25632C7D2431617B253157
:10145000692C302D337C317D2E2432617B2532691D
:101460002C302D37357C32357D7E300041646A75F5
:10147000737420436C6F636B0A54656D70657261A1
:1014800074757265004C45442053657474696E67C9
:10149000730054656D70657261747572650A536589
:1014A0007474696E67730053657474696E67730052
:1014B0005461736B73008D5D13C01002CEBFCA1BE5
:1014C0009ABF0C926ABF157231BF7EC502BF1B9EC8
:1014D000B6BEDC7F64BE82C7D7BD486561746572E5
:1014E0000054656D70416D62690054656D7053758F
:1014F0006D700054656D7054616E6B004556454EBD
:101500005420414444004556454E54204649580015
:101510004556454E542044454C00435552564520AF
:1015200045445400435552564520414444004355D8
:101530005256452045445400435552564520414497
:10154000440043555256452044454C00435552569D
:1015500045204445560043555256452049440050C5
:10156000554D5020504F5254530050756D702025EA
:1015700069004C45445F506F7772004B6579204499
:101580004F574E004B6579204C454654004B6579CA
:101590002055500044494D20330044494D2032002D
:1015A00044494D2031005254432053434C0052547F
:1015B00043205344410052544320496E74005374F5
:1015C000617475730044494D20370044494D2036FD
:1015D000004C434420424C004C434420454E004CB8
:1015E0004344205253004C4344204437004C43446E
:1015F000204436004C4344204435004C43442044AE
:10160000340044494D20350044494D2034004B6599
:10161000792052494748540052454320534B495082
:101620000057445420524553455400424F442052E1
:10163000455345540000002100240027002A002DB6
:10164000003000330001010000040107010A01001D
:10165000002200250028002B002E0031003400025B
:10166000010000050108010B0100000A0B02090C32
:101670000D0E080703040100000000000000000038
:10168000000000000000000000000000000000005A
:101690000000000000121110000000000000000017
:1016A000000000000000000000000000000000003A
:1016B0000020002300260029002C002F003200000B
:1016C00001000003010601090105050505070508DC
:1016D000080808020202020A0A08080404040401B5
:1016E00001010101010101030303030303030304D7
:1016F0000707070C0C0C0C0C0C0C0C020202020667
:10170000060606060606060B0B0B0B0B0B0B0B0156
:101710000210202008081020401020408002010202
:1017200001080402010102040810204080804020CA
:101730001008040201800402018040201008040205
:101740000108040201010204081020408001020483
:10175000081020408000CC7611241FBECFEFD1E2CC
:10176000DEBFCDBF00E00CBF13E0A0E0B2E0ECEDC7
:10177000F0E101E00BBF02C007900D92A63EB10759
:10178000D9F728E0A6EEB3E001C01D92AC3DB20748
:10179000E1F71BE0CCEADBE000E006C0219701099D
:1017A000802FFE010E949683CB3AD10780E0080784
:1017B000A9F70E9443770C946C880C94000008955C
:1017C000FC0190E0615050F02191922728E08CE8D4
:1017D000969508F498272A95D9F7F4CF892F08957C
:1017E000DC012C911196ED91FC91F8948181822B72
:1017F00081839281322F30959323928387E090E00A
:101800000197F1F781818323818383E290E001973F
:10181000F1F790817894EFECF0E03197F1F79223B3
:1018200081E009F480E00895FC0190810180F2815B
:10183000E02D292F209560FF14C0F8948281822327
:1018400082838181892B8183A3E2B0E01197F1F734
:101850008281982B9283789487ED90E00197F1F73D
:101860000895F8948281822382838181892B8183E8
:10187000AFEFB0E01197F1F78281982B92837894C3
:101880008FE090E0EBCFDF92EF92FF920F931F93E8
:10189000CF93DF93EC01D62EE42E08E010E0FF2476
:1018A000F39461E08D2D8F2109F460E0CE010E9458
:1018B000140CFF0C01501109A1F7E11010C0F894AD
:1018C000E981FA8191818881809589238183E981E9
:1018D000FA81928188818095892382837894DF912F
:1018E000CF911F910F91FF90EF90DF900895FC0131
:1018F00090810180F281E02DF8948181292F20953B
:101900008223818378943DE743E050E0315029F110
:10191000DA011197F1F780818923C1F3F89482816C
:10192000822382838181892B81837894ABE7B7E01E
:101930001197F1F7F894818182238183A3E1B1E0CB
:101940001197F1F78081982381E009F080E0789485
:10195000E3E6F6E03197F1F7089580E00895E0912D
:101960004707F09148070684F785E02D8081816064
:1019700080830895E0914707F09148070684F78532
:10198000E02D80818E7F808308959A01AB018330A2
:1019900011F148F4813099F0A1E2B0E0823049F0D1
:1019A00090E080E008958430C9F0A2E6B0E185308F
:1019B000B9F70E94B48370588F4F9F4F0895305EDF
:1019C0004F4F5F4F82E0220F331F441F551F8A95F0
:1019D000D1F7CA010895A6E0B1E0EBCFA9E1B4E0E8
:1019E000E8CFEFE3F7E0A085B18514960D90BC91A8
:1019F000A02D4D915C9170E060E084810C94C50C49
:101A0000062E000C770BDC011896ED91FC91828973
:101A10008617170641F40190F081E02D808186FB46
:101A2000882780F9089583898617170639F401906D
:101A3000F081E02D808182958170089584898617D8
:101A4000170641F40190F081E02D808182FB882708
:101A500080F9089580E00895062E000C770BDC01D4
:101A60001896ED91FC91828990E04423F1F068177B
:101A7000790739F40190F081E02D808180648083C2
:101A8000089583898617170631F40190F081E02DBF
:101A900080818061F4CF84898617170689F70190C9
:101AA000F081E02D80818460EACF6817790731F4F6
:101AB0000190F081E02D80818F7BE1CF83898617B3
:101AC000170631F40190F081E02D80818F7ED7CF11
:101AD000848986171706A1F60190F081E02D808198
:101AE0008B7FCDCFCF93DF93FC01C62F2281338133
:101AF000DA010E94AD832581DC01CB0104C0B695DB
:101B0000A795979587952A95D2F70C2E000CDD0B9B
:101B10000084F185E02D42894C171D0641F40084B4
:101B2000F185E02D91838083DF91CF9108954389E2
:101B30004C171D0621F40284F385E02DF3CF448970
:101B40004C171D0689F70484F585E02DEBCF0F9324
:101B50001F93CF93DF93FC01141615061606170684
:101B600024F041E050E060E070E0868197810097CA
:101B7000B9F513E0440F551F661F771F1A95D1F76B
:101B80004115510521E06207710590F521E024839C
:101B90008A019B01019721F40150110921093109A2
:101BA00013830283A085B1851696CD91DC9117979A
:101BB0001983088312960D90BC91A02D8C91887F7B
:101BC0008C93A085B18512960D90BC91A02D8C911F
:101BD0009481892B8C93DF91CF911F910F91089560
:101BE000D4E0440F551F661F771FDA95D1F7C8CF91
:101BF0008A019B01C3E03695279517950795CA95ED
:101C0000D1F701151105A1E02A07310518F442E0CA
:101C10004483C0CF8A019B01B6E03695279517957E
:101C20000795BA95D1F701151105A1E02A073105ED
:101C300010F443E0EDCF052F162F272F3327011582
:101C40001105A1E02A07310510F444E0E1CF8A0133
:101C50009B014AE036952795179507954A95D1F748
:101C60000115110541E02407310510F445E0D0CFFE
:101C700025E024830FEF1FEF20E030E08BCFCF93E0
:101C8000DF93FC01A085B1851696CD91DC91179765
:101C90006881798190E080E012960D90BC91A02D32
:101CA0002C91277046815781452B89F52330F9F017
:101CB00040F4213091F02230B9F060E070E0CB01C7
:101CC00013C02430E1F02530C1F7F7E0660F771F2D
:101CD000881F991FFA95D1F707C0C3E0969587959D
:101CE00077956795CA95D1F7DF91CF910895B3E0C5
:101CF000660F771F881F991FBA95D1F7F5CFA5E01A
:101D0000660F771F881F991FAA95D1F7EDCF6F5FD8
:101D10007F4F8F4F9F4F2330F1F048F4213099F0DF
:101D2000223059F69695879577956795DDCF2430C3
:101D3000D1F0253011F626E0660F771F881F991F16
:101D40002A95D1F7D1CFE4E0969587957795679559
:101D5000EA95D1F7C9CF42E0660F771F881F991F18
:101D60004A95D1F7C1CF34E0660F771F881F991FBE
:101D70003A95D1F7B9CF0F931F93FC0117830683D0
:101D8000A085B1850D90BC91A02D1C928681978174
:101D9000A085B185892B61F412960D90BC91A02D80
:101DA00080E18C932583CF011F910F910C94A70D97
:101DB0000D90BC91A02D82E08C93A085B1851296E8
:101DC0000D90BC91A02D88E1ECCF8150823108F0BC
:101DD0005AC0E82FF0E08827EF50F14F8F4F0C9456
:101DE0009683110F150F030F090F0D0F430F180FD7
:101DF0001E0F220F280F2C0F300F360F3A0F430FF4
:101E00003E0F440F480F809180008F7780938000B1
:101E10000895809180008F7DF9CF80918000877F29
:101E2000F5CF84B58F7784BD089584B58F7DFBCFC2
:101E30008091B0008F778093B00008958091B000BA
:101E40008F7DF9CF809190008F77809390000895D7
:101E5000809190008F7DF9CF80919000877FF5CFA2
:101E60008091A0008F778093A00008958091A000BA
:101E70008F7DF9CF8091A000877FF5CF80912001E1
:101E80008F77809320010895809120018F7DF9CF75
:101E900080912001877FF5CF1F93CF93DF93282F69
:101EA00030E0F901E759F94E8491F901E15FF84E0C
:101EB000D491F901E753F94EC491CC23A9F0162F20
:101EC00081110E94E50EEC2FF0E0EE0FFF1FE15BA9
:101ED000F94EA591B4918FB7F894EC91111108C007
:101EE000D095DE23DC938FBFDF91CF911F910895B2
:101EF000DE2BF8CFCF93DF9390E0FC01E15FF84E4B
:101F000024918753994EFC0184918823C9F090E075
:101F1000880F991FFC01EB5CF94EA591B491FC016F
:101F2000E15BF94EC591D49161110DC09FB7F89452
:101F30008C91209582238C938881282328839FBFAE
:101F4000DF91CF910895623051F49FB7F8943C919E
:101F5000822F809583238C93E8812E2BEFCF8FB730
:101F6000F894EC912E2B2C938FBFEACF1F93CF9335
:101F7000DF93EC01162F60E0812F0E947A0F612F12
:101F800070E0FB01E15FF84EE491E883FB01E75369
:101F9000F94EE491F0E0EE0FFF1FE155F94E859107
:101FA00094919A8389831B861D861C861A861986BE
:101FB00018861F821E821D821C821B82DF91CF9198
:101FC0001F9108953FB7F8948091C1069091C20681
:101FD000A091C306B091C40626B5A89B05C02F3FAB
:101FE00019F00196A11DB11D3FBFBA2FA92F982F3F
:101FF0008827BC01CD01620F711D811D911D42E03A
:10200000660F771F881F991F4A95D1F708958F9201
:102010009F92AF92BF92CF92DF92EF92FF924B01CD
:102020005C010E94E20F6B017C010E94E20F6C19BF
:102030007D098E099F09683E734081059105A8F3CB
:1020400021E0821A9108A108B10888EEC80E83E049
:10205000D81EE11CF11C81149104A104B10429F7DC
:10206000FF90EF90DF90CF90BF90AF909F908F90B8
:1020700008958AB588608ABD089581E08093CC0672
:102080000895089508950895AF92BF92CF92DF9278
:10209000EF92FF920F931F93CF93DF936C017B011D
:1020A0008B01040F151FEB015E01AE18BF08C017AE
:1020B000D10759F06991D601ED91FC910190F08121
:1020C000E02DC6011995892B79F7C501DF91CF91D4
:1020D0001F910F91FF90EF90DF90CF90BF90AF9046
:1020E0000895DF92EF92FF920F931F93CF93DF93A8
:1020F0007C01FB01C381D481DD8010E000E00D157F
:1021000018F5EE81FF81C801880F991FE80FF91FAC
:10211000808191810097A9F08E159F05B9F08B8180
:102120009C81892B71F0BE01C7010E947110882328
:1021300041F0DF91CF911F910F91FF90EF90DF90D1
:1021400008950F5F1F4FDBCF80E0F3CF81E0F1CF29
:10215000CF93DF93EC01892B09F445C029813A81A3
:102160002115310509F43FC0D90180E0FD01E21BD2
:10217000F30B9D919923B9F19432C1F79C9194325C
:10218000A9F386132EC0E20FF31F8191882359F122
:10219000BF01621B730B8B37C1F79B01A22FA61BDC
:1021A000E981FA81E20FF31F80818823E1F08C320C
:1021B000D1F0A40FB52FB11D8C9181110EC090E20A
:1021C000E981FA81E20FF31F8081882361F08C326C
:1021D00051F090832F5F3F4FF3CF80832F5F3F4FAE
:1021E000DDCF8F5FC3CFDF91CF910895EF92FF9244
:1021F0001F93CF93DF93E0914F06F09150063097F5
:1022000009F444C0EC0189819A81009709F019957D
:102210008E819F81892B49F110E08E819F812D81D4
:102220001217F0F4212F30E0220F331F820F931F7B
:10223000FC01E080F180E114F10481F08B819C814C
:10224000892B31F0BE01C7010E947110811106C0B7
:10225000E0914F06F0915006C70119951F5FDDCF41
:10226000E0914F06F091500619958885882371F00A
:1022700089859A85009751F0E0914F06F0915006BC
:10228000DF91CF911F91FF90EF901994DF91CF9143
:102290001F91FF90EF900895AF92BF92CF92DF927F
:1022A000EF92FF920F931F93CF93DF937C0100E097
:1022B000B12C40E010E0212F30E06701C20ED31EA8
:1022C000D601DC91C701840F911DE0914B06F0917E
:1022D0004C06DD2341F1AA24A394A10ED43289F443
:1022E000E9012196CE0DDF1DD880B4E2DB1207C0D4
:1022F00018821995080FD88242E0410F1A2D1F5FEE
:10230000DACFDA30E1F71C921995080FF601D08385
:10231000B394E0914706F09148066B2D80E0199543
:102320004A2D1A2DECCF1995800FDF91CF911F9177
:102330000F91FF90EF90DF90CF90BF90AF900895F6
:10234000882351F0662341F0861731F0883031F44C
:102350009FEF960F953040F481E00895893021F485
:102360009AEF960F9230C0F3683039F49FEF980FD0
:1023700081E0953048F080E007C06930E1F79AEFDE
:10238000980F81E09230B8F70895FB019C01295F16
:102390003F4FDC015D91CD014191541305C0A2175F
:1023A000B307B9F781E0089580E00895FC018FEF4D
:1023B0008083818382838383848385838683089556
:1023C0000F931F93CF93DF9300D000D01F92CDB710
:1023D000DEB729833A834B835C836D837E838F834F
:1023E00010E003E0809133061817B8F4E09131064D
:1023F000F0913206109FE00DF11D11242C812F77F2
:10240000808190E02817190631F40180F281E02DD7
:10241000CE01059619951F5FE5CF27960FB6F89464
:10242000DEBF0FBECDBFDF91CF911F910F910895F9
:1024300020913F06309140068217930710F40896CA
:10244000089580914106909142060895FC019C01F7
:10245000295F3F4F90E08191982788E04CE896955E
:1024600008F494278A95D9F72E173F07A1F7892FEB
:102470000895AF92BF92DF92EF92FF920F931F9356
:10248000CF93DF931F92CDB7DEB78C017B01809194
:102490003F06909140068617970738F080914106D5
:1024A000909142066817790778F4C8010E94D61106
:1024B00084E00F90DF91CF911F910F91FF90EF90EB
:1024C000DF90BF90AF90089588E0D82E5B0187E041
:1024D000A80EB11C1982E0913906F0913A0641E04C
:1024E000BE016F5F7F4FC5011995E0913906F091EC
:1024F0003A0647E0B801C7011995C8010E942612A3
:102500009981DA94DD2021F08913E4CF80E0D1CFE6
:102510008917E1F3C8010E94D61188E0CACFEF9273
:10252000FF920F931F93CF93DF93CDB7DEB72E9714
:102530000FB6F894DEBF0FBECDBF182F7B0100E0B1
:10254000B701CE0108960E943912882339F0CE01D6
:1025500008960E94D611002321F149C0C7010E94AC
:1025600018127C013885832F8F7032953F709985C2
:10257000292F21702295207F232B96959F738A30D7
:1025800028F4283118F401E09C3308F000E0612FB2
:102590000E94A011882319F08B8587FFDCCF0111E1
:1025A0001EC080917D04873010F58F5F80937D047D
:1025B000609141067091420681E0173008F4810F66
:1025C0000E948F12288739874A875B876C877D87AF
:1025D0008E8780917D04815080937D0408C0809116
:1025E0004106909142068E159F0508F4A9CF87E019
:1025F000FE013896DE01119601900D928A95E1F761
:1026000029813A814B815C816D817E818F8190E04F
:102610002E960FB6F894DEBF0FBECDBFDF91CF91DF
:102620001F910F91FF90EF900895CF93DF93CDB757
:10263000DEB72E970FB6F894DEBF0FBECDBF609108
:10264000410670914206CE0108960E94391287E039
:10265000FE013896DE01119601900D928A95E1F700
:1026600029813A814B815C816D817E818F8190E0EF
:102670002E960FB6F894DEBF0FBECDBFDF91CF917F
:102680000895CF93DF9300D000D01F92CDB7DEB76F
:102690006091410670914206CE0101960E94391266
:1026A0002981322F32953F709A81892F81708295CE
:1026B000807F832B96959F732F702A3028F4883162
:1026C00018F481E09C3308F080E091E08927279698
:1026D0000FB6F894DEBF0FBECDBFDF91CF91089546
:1026E000CF93DF9300D000D01F92CDB7DEB76091BB
:1026F0003F0670914006CE0101960E943912298151
:10270000322F32953F709A81892F81708295807F18
:10271000832B96959F732F702A3028F4883118F4F4
:1027200081E09C3308F080E027960FB6F894DEBF76
:102730000FBECDBFDF91CF910895AF92BF92CF92E0
:10274000DF92EF92FF920F931F93CF93DF9300D00E
:1027500000D01F92CDB7DEB7A62EC42E89012091DE
:102760003F06309140062017310708F485C02091BC
:102770004106309142060217130708F47DC0F12C80
:10278000972F9170D92ED29490EFD922962F9295AF
:102790009F70D92A972F96959F73B92E771F772709
:1027A000771F8F71E82EEE0CE72A80913F069091FB
:1027B000400680179107C8F1F7FC37C0B801CE0179
:1027C00001960E943912882379F0883051F40E94D2
:1027D0004113882331F00091410610914206CC202C
:1027E00021F10FEF1FEF21C02981322F32953F7069
:1027F0008A81982F91709295907F932B482F4695C0
:102800004F73FD2CF91AD9F5FB2CF41AC1F5382FAA
:10281000331F3327331F8B818F71880F832BFE2C3F
:10282000F81AC11014C0F7FE18C0C80127960FB6D9
:10283000F894DEBF0FBECDBFDF91CF911F910F91F6
:10284000FF90EF90DF90CF90BF90AF900895F11080
:1028500004C0822F8A258F7041F32F702A3018F020
:10286000CC2019F3BECF9831D8F74C33C8F7C80144
:102870000E9418128C0199CF04E010E0D6CFCC2032
:1028800091F2EBCF0F931F93CF93DF93CDB7DEB7CA
:102890002E970FB6F894DEBF0FBECDBF28873987BD
:1028A0004A875B876C877D878E87980168857985E5
:1028B0008A8541E00E949D138C010F3F100771F43F
:1028C0000FEF1FEFC8012E960FB6F894DEBF0FBEB4
:1028D000CDBFDF91CF911F910F91089580913F0659
:1028E000909140068017910758F38091410690918E
:1028F00042060817190720F3B801CE0101960E947D
:102900003912BE01685F7F4FCE0101960E94C5114A
:102910008111D8CFC8010E9418120817190780F634
:102920008C01288539854A855B856C857D858E85FA
:102930000E9442148C01C6CF2F923F924F925F9219
:102940006F927F928F929F92AF92BF92CF92DF92BF
:10295000EF92FF920F931F93CF93DF93CDB7DEB724
:102960002F970FB6F894DEBF0FBECDBFF62EE72E21
:10297000A82E262F2F70B22E87E0E6E0F2E0DE01CF
:10298000189601900D928A95E1F720910602822F08
:102990008F708A3078F422952F7080910702982FDB
:1029A00091709295907F922B983120F486958F7339
:1029B0008C33E0F0209141063091420640E06F2DCB
:1029C0007E2D8A2D0E949D13BC018B2D0E948F129B
:1029D00020930602309307024093080250930902A5
:1029E00060930A0270930B0280930C02812C3B2DA2
:1029F0003F703F878A2D8F71C82ECC0C8E2D881F7B
:102A00008827881FC82A8E2D8170582E529480EFF7
:102A1000582200910602802F8F7002950F709091BE
:102A20000702292F21702295207F022B192F16953E
:102A30001F738A3008F0F8C0083108F0F5C01C3365
:102A400008F0F2C0EF2DE07FFE2EFF85FF2A991FD0
:102A50009927991FD09008022D2D2F71D22EDD0CB1
:102A6000D92A2E2D26952F739F2D92959F709529EB
:102A7000302F391B932F29F4912F921B11F49D2D88
:102A80009C1919160CF4D0C06B2D0E94A011982E21
:102A9000882309F4C9C080913406982F9F259F7020
:102AA000F9F490913506492F46954F73392F331F0E
:102AB0003327331F209136062F71220F232B382FF7
:102AC00032953F70892F81708295807F832B801B88
:102AD00029F4842F811B11F4822F8D1987FFA4C044
:102AE000209106023091070240910802509109029C
:102AF00060910A0270910B0280910C020E94E01119
:102B00000091410610914206209106023091070281
:102B1000409108025091090260910A0270910B02E3
:102B200080910C020E9442140E941812BC018B2D4D
:102B30000E948F12722ED32E842E252E362E472ED3
:102B4000682E29833A834B835C836D837E838F83D6
:102B5000BE016F5F7F4F86E092E00E94C511811138
:102B600062C02D2D21702295207F872D82958F7038
:102B7000282B90910602392F32953F7080910702E1
:102B8000982F91709295907F932B291759F087E099
:102B9000FE013196A6E0B2E001900D928A95E1F730
:102BA000892C37CF2D2D26952F73982F96959F73AF
:102BB0002913EDCF982D9F71990F2D2D221F2227BC
:102BC000221F922B282F221F2227221F80910802CA
:102BD0008F71880F822B9813DACF009141061091E4
:102BE0004206272D3D2D482D522D632D742D862D07
:102BF0000E9442143C01009141061091420620912E
:102C0000060230910702409108025091090260913A
:102C10000A0270910B0280910C020E9442148615E8
:102C2000970508F4B4CF892C8F2D807FF82EEF857F
:102C3000FE2AF0923406E0923506A0923606009104
:102C400037061091380601151105C1F066E072E0F3
:102C5000CE0108960E94C511811110C02091060274
:102C600030910702409108025091090260910A02D6
:102C700070910B0280910C02F8011995882D2F9606
:102C80000FB6F894DEBF0FBECDBFDF91CF911F917D
:102C90000F91FF90EF90DF90CF90BF90AF909F90FB
:102CA0008F907F906F905F904F903F902F900895FE
:102CB000E0913D06F0913E061995609334067093BD
:102CC00035068093360686E092E00E94D611609128
:102CD000340670913506809136060C949C140F933F
:102CE0001F93CF93DF93CDB7DEB765970FB6F894F8
:102CF000DEBF0FBECDBF2F87388B498B5A8B6B8BB6
:102D00007C8B8D8B0E944113811150C00091410634
:102D1000109142062F85388949895A896B897C89A7
:102D20008D890E9442148F3F980721F10E9418124A
:102D3000BC01CE0108960E943912811113C028856A
:102D4000822F8F708A3070F422952F708985982F8A
:102D500091709295907F922B983120F486958F7385
:102D60008C3340F06091410670914206CE01089686
:102D70000E94391287E0FE013896DE01119601901B
:102D80000D928A95E1F729813A814B815C816D81B1
:102D90007E818F8190E065960FB6F894DEBF0FBEFE
:102DA000CDBFDF91CF911F910F910895CE0108966D
:102DB0000E94D611DFCFCF92DF92EF92FF920F9356
:102DC0001F93CF93DF93CDB7DEB768970FB6F89414
:102DD000DEBF0FBECDBF20913F06309140062617C3
:102DE000370708F476C020914106309142066217F9
:102DF000730708F46EC06B018C0187E0F801DE01F7
:102E0000199601900D928A95E1F7C8010E94261249
:102E1000888B88E0FE013996DE01119601900D92B3
:102E20008A95E1F788E0FE013196DE01199601905E
:102E30000D928A95E1F788E0FE013996DE01519600
:102E400001900D928A95E1F788E0F82EE0913B061B
:102E5000F0913C0648E0BE016F5E7F4FC6011995B8
:102E6000E88CE0913906F0913A0648E0BE016F5EC9
:102E70007F4FC6011995BE016F5E7F4FC8010E944A
:102E8000C511882321F081E0988D9E1180E0FA948D
:102E9000FF2021F08823D1F280E00CC08111FCCF0B
:102EA00029893A894B895C896D897E898F890E943D
:102EB0004F1888E068960FB6F894DEBF0FBECDBFFE
:102EC000DF91CF911F910F91FF90EF90DF90CF9006
:102ED000089584E0EFCFAF92BF92CF92DF92EF924E
:102EE000FF920F931F93CF93DF93CDB7DEB7659714
:102EF0000FB6F894DEBF0FBECDBF2F87388B498B3E
:102F00005A8B6B8B7C8B8D8B009141061091420606
:102F10000E944214409141065091420648175907B9
:102F200040F420913F063091400616E08217930747
:102F300018F19F85392F32953F708889982F9170AD
:102F40009295907F932B69F4982F9E7751F4982F48
:102F5000991F9927991F89898F71880F892B17E0ED
:102F600059F06F85788989899A0140E00E949D1304
:102F70008C01019699F411E0812F65960FB6F894B3
:102F8000DEBF0FBECDBFDF91CF911F910F91FF909C
:102F9000EF90DF90CF90BF90AF90089580913F0663
:102FA0009091400608978017910708F476C08091A9
:102FB0004106909142060817190708F46EC00E9456
:102FC00070138111D8CFB801CE0101960E94391239
:102FD000C8010E9418127C01DD24D394B12C87E033
:102FE000A82E80913F0690914006E816F90608F059
:102FF00042C0DD2009F43FC08B2D90E00196817026
:103000009927A89E6001A99ED00C112481E090E030
:103010008C0F9D1FC80ED91EB701C6010E94391220
:10302000B7018B2D8170E1E0F0E0EC0FFD1F8A9D70
:10303000E00DF11D1124CF010E94DB16F601208165
:10304000322F32953F708181982F91709295907FA9
:10305000932B86958F732F702A3030F4983120F49B
:10306000DD24D3948C3308F0D12CB394C7010E9493
:1030700018127C01B6CFB801CE010F960E94DB1664
:10308000182F811179CF80913D0690913E06892BB2
:1030900009F472CF0E9458166FCF15E06DCFFF92E2
:1030A0000F931F93CF93DF93CDB7DEB72E970FB655
:1030B000F894DEBF0FBECDBF288739874A875B876C
:1030C0006C877D878E8700914106109142060E9491
:1030D000421400913F06109140060817190708F4A2
:1030E0005BC00E9418120817190708F462C02091EB
:1030F0004106309142068217930708F45AC08C01AA
:1031000008501109FF24F39480913F0690914006E6
:103110000817190750F5FF20A1F1C8010E941812E5
:10312000BC01CE0101960E943912B801CE01019670
:103130000E94DB162981322F32953F708A81982FA9
:1031400091709295907F932B86958F732F702A3074
:1031500030F4983120F4FF24F3948C3308F0F12CF0
:10316000C8010E9418128C01CFCF8017910749F433
:10317000CE0101960E94D611B801CE0101960E949F
:10318000DB1666E072E0CE0108960E94C51181113F
:103190000E94581680E001C082E02E960FB6F89487
:1031A000DEBF0FBECDBFDF91CF911F910F91FF907A
:1031B000089585E0F2CFAF92BF92CF92DF92EF9267
:1031C000FF920F931F93CF93DF93CDB7DEB72E9768
:1031D0000FB6F894DEBF0FBECDBF0091410610912F
:1031E0004206C8010E9418127C0180913F0690910E
:1031F00040068E159F0508F457C0B801CE01019610
:103200000E943912182FB701CE0108960E94391278
:10321000111177C0811175C08981982F9F709A30E4
:1032200008F081C082958F70AA801A2D11701295B6
:10323000107F182B183108F076C0BA2CB6948B2D5D
:103240008F73B82E8BE38B1508F46DC00885802F23
:103250008F708A3008F067C002950F70D9848D2D69
:1032600081708295807F082B083108F05CC0CD2CDE
:10327000C6948C2D8F73C82E8BE38C1508F453C025
:10328000BE01685F7F4FCE0101960E94C511882361
:1032900069F028853D2D4A855B856C857D858E8509
:1032A0000E944F180E94DB1881E02CC0AA1CAA249F
:1032B000AA1C2B812F71220F2A29DD1CDD24DD1C85
:1032C0009A859F71990F9D29812F801B29F48B2D41
:1032D0008C1911F4822F891B18162CF52885398535
:1032E0004A855B856C857D858E850E944F18288573
:1032F00039854A855B856C857D858E850E946B1737
:10330000D1CF80E02E960FB6F894DEBF0FBECDBFB2
:10331000DF91CF911F910F91FF90EF90DF90CF90B1
:10332000BF90AF900895C7010E94181287015CCF2B
:1033300097E6899F90011124232F26952695922F99
:10334000990F920F990F890F0895EF92FF920F93A3
:103350001F93CF93DF937C0108E010E0C0E0D1E041
:10336000C7010E94F00B8111CD2BDD0F0150110917
:10337000B9F78C2FDF91CF911F910F91FF90EF90B4
:103380000895EF92FF920F931F93CF93DF938C01D9
:103390007B0140E065E50E94430CE70188E0E80E10
:1033A000F11C699140E0C8010E94430CCE15DF0575
:1033B000C1F7DF91CF911F910F91FF90EF9008958A
:1033C000EF92FF920F931F93CF93DF93EC018B014A
:1033D0007A018D819E810E94770CB8018D819E813A
:1033E0000E94C11940E06EE48D819E810E94430CD1
:1033F00040E0F70162818D819E810E94430C40E094
:10340000F70163818D819E810E94430CF8018081C8
:10341000803139F040E0F70164818D819E810E9406
:10342000430C8D819E810E94770CB8018D819E8115
:103430000E94C119488168E48D819E810E94430CDD
:103440008881882331F06AE070E080E090E00E949B
:1034500007108D819E81DF91CF911F910F91FF9079
:10346000EF900C94770CCF92DF92EF92FF920F9334
:103470001F93CF93DF93EC017B018A018D819E81A5
:103480000E94770C811102C090E029C0B7018D81A4
:103490009E810E94C11940E06EEB8D819E810E9449
:1034A000430C7801680189E0C80ED11C8D819E8192
:1034B0000E94A519F70181937F01CE16DF06B1F7AF
:1034C0008D819E810E94770C8130F1F668E0C80101
:1034D0000E94E00B91E0F80120852813D5CF892FB9
:1034E000DF91CF911F910F91FF90EF90DF90CF90E0
:1034F0000895CF93DF9300D000D000D0CDB7DEB7D2
:10350000FB012081203199F0AE014F5F5F4F0E9497
:10351000331A882331F08D818F33A9F020F48F3155
:10352000A1F080E007C08F3521F08F37D1F78CE014
:1035300001C08BE029960FB6F894DEBF0FBECDBF59
:10354000DF91CF9108958AE0F5CF89E0F3CFAF9274
:10355000BF92CF92DF92EF92FF920F931F93CF9380
:10356000DF9300D000D000D0CDB7DEB77C01062FAE
:10357000142F6C018EE0C80ED11C5701E1E2AE0E93
:10358000B11CAE014F5F5F4FB501C6010E94331AF7
:103590008823B9F0602F093C0CF469EC6E370CF00D
:1035A0006DE76C83412F193C0CF449EC4E370CF05D
:1035B0004DE74B83AE014F5F5F4FB501C6010E94DF
:1035C000E019AE014F5F5F4FB501C6010E94331A8B
:1035D000882301F18B81F70184ABAE014F5F5F4F10
:1035E000B501C6010E94331A8823B1F08C81F7011E
:1035F00083AB29960FB6F894DEBF0FBECDBFDF9127
:10360000CF911F910F91FF90EF90DF90CF90BF90DF
:10361000AF90089581E8DFCF81E8E9CFCF92DF92C4
:10362000EF92FF920F931F93CF93DF93EC017B01F7
:103630008A010E94770CB701CE010E94C11940E0B7
:103640006EEBCE010E94430C7801680189E0C80E40
:10365000D11CCE010E94A519F70181937F01EC15C1
:10366000FD05B9F769E0C8010E94E00B91E0811106
:1036700090E0892FDF91CF911F910F91FF90EF90F4
:10368000DF90CF9008953F924F925F926F927F921A
:103690008F929F92AF92BF92CF92DF92EF92FF9262
:1036A0000F931F93CF93DF93FC013680A32DB0E0DF
:1036B00020E833E341EE51E00E94B4834B015C010A
:1036C000D0E0C0E09D0184E6C82ED12C90E9E92E1F
:1036D000FF24F394C217D307C4F14580512C2E5810
:1036E0003E4FC90164E670E00E9441837C01C9013C
:1036F00060E971E00E9441836C010CE113E0C1E0DC
:10370000D0E0832D8170382E3901A3E06A2277241E
:10371000C415D5050CF047C0C230D105A9F531104C
:1037200033C06114710481F5E114F10419F4C1147A
:10373000D10451F5A0E88A0EABE39A1EA6E2AA1EB8
:10374000B11C21960F5F1F4FE3CFC0FD1BC08E0140
:103750000E581E4FC80183709927892B99F4C80110
:10376000B6010E944183892B31F4C801B7010E9440
:103770004183892B39F480E8880E81E5981E81E029
:10378000A81EB11C2196A6CFD8018C91A82FB0E01D
:1037900020E831E541E050E00E94B483860E971E98
:1037A000A81EB91ECECF228130E0A0E1BEE00E946B
:1037B0009E836B017C01218130E0ACE3B0E00E948C
:1037C0009E83C60ED71EE81EF91E8081C80ED11C2E
:1037D000E11CF11CA481A150BB0B20E831E541E0C4
:1037E00050E00E94BF836C0D7D1D8E1D9F1D680DD6
:1037F000791D8A1D9B1DDF91CF911F910F91FF9025
:10380000EF90DF90CF90BF90AF909F908F907F9080
:103810006F905F904F903F9008957F928F929F920C
:10382000AF92BF92CF92DF92EF92FF920F931F93CE
:10383000CF93DF936B017C01EA018CE3882E912CFE
:10384000A12CB12CC701A50194010E945583688366
:10385000CA01B901A50194010E9455836983C7017A
:10386000B60120E13EE040E050E00E945583CA01ED
:10387000B90128E130E040E050E00E9455836A83BE
:10388000C701B60120E831E541E050E00E945583D0
:1038900049015A01CA01B9016C5F7F4F8F4F9F4F99
:1038A00027E030E040E050E00E9455836F5F6B837B
:1038B000F0E0E0E0712C94E6E92EF12C20E9C22E34
:1038C000DD24D394272D30E0472D417070FC1DC0BE
:1038D00089010E581E4FC80183709927892BA9F4BE
:1038E000C801B7010E944183892B31F4C801B60198
:1038F0000E944183892B49F48EE691E0E80FF91F7D
:103900008E169F0628F07394DDCF8DE691E0F6CFFA
:103910007E822E583E4FC90164E670E00E944183CA
:103920008C01C90160E971E00E94418341110AC024
:10393000B90163707727672B29F401151105E9F4A4
:103940000097D9F06DE671E0E61BF70B8E1A9F0A1F
:10395000A108B108ECE1F3E060E0237033276130A7
:1039600079F4411133C02115310581F50115110597
:1039700011F4009759F55DE104C06EE671E0E4CF03
:103980005081C52ED12CF12CE12C51E0560F8C1416
:103990009D04AE04BF0440F08C189D08AE08BF081B
:1039A0003196652F5C30D9F66F5F6D8383948C827E
:1039B000DF91CF911F910F91FF90EF90DF90CF900B
:1039C000BF90AF909F908F907F9008955CE1D9CF8A
:1039D000CF92DF92EF92FF92C0907404D090750462
:1039E000E0907604F0907704C616D706E806F9064C
:1039F00071F06B017C014DE654E00E940D1CC092F9
:103A00007404D0927504E0927604F0927704FF90EB
:103A1000EF90DF90CF900895CF92DF92EF92FF92D8
:103A20000F931F93CF93DF93EC01FB0180818031D3
:103A300008F080E01882982F3FE0A92FB0E03A9F6D
:103A4000F0013B9FF00D1124E258FB4F50814111D2
:103A500008C0511109C0211131C09923B9F1915009
:103A600030C0E881E517B8F73A9F80013B9F100D01
:103A7000112402581B4FF801DE01532F01900D92C3
:103A80005A95E1F7FB019083F801C384D484E5845F
:103A9000F684FB01C182D282E382F4824111DBCF42
:103AA00081E09881911101C080E0DF91CF911F9159
:103AB0000F91FF90EF90DF90CF9008959F5F90312E
:103AC00018F48913BACFECCF90E0FBCF9FE0F9CF89
:103AD000FB0120812F5F208321E041E00C940C1D2D
:103AE0000F931F93DC01EC91E031B0F48FE0E89F7D
:103AF000F0011124E258FB4F11960D911D912D916B
:103B00003C91149743855485658576850417150780
:103B10002607370709F410828FEF8C931F910F91BE
:103B20000895CF92DF92EF92FF92CF93DF93E091CF
:103B30004707F09148070680F781E02D40815181C9
:103B400070E060E08091450790914607892B21F451
:103B5000440F551F661F771F809143070E94C50CB5
:103B60006C01F12CE12C8091690490916A04A09180
:103B70006B04B0916C048C0D9D1DAE1DBF1D809318
:103B8000690490936A04A0936B04B0936C048091D1
:103B90006E058F3F09F463C0A0916E0587E0A89F72
:103BA000D0011124A159BA4F11964D915D916D919B
:103BB0007C911497C416D506E606F706C0F5119653
:103BC0004D915D916D917C9114974C195D096E0931
:103BD0007F0911964D935D936D937C931497119685
:103BE0004D915D916D917C911497DEEFC7E0411589
:103BF000510561057105B9F58C9180936E05159697
:103C0000ED91FC911697DC93199580916E058F3F8D
:103C100031F1A0916E05AC9FD0011124A159BA4F8A
:103C200011964D915D916D917C911497E0CF40E09C
:103C300050E0BA01DACF9A01AB0144275527A8EE2C
:103C4000B3E00E94B483AB01BC018FE397E0DF9146
:103C5000CF91FF90EF90DF90CF900C94A70D40E6AE
:103C600050E160E070E0C416D506E606F70619F7E5
:103C7000DF91CF91FF90EF90DF90CF900895CF929A
:103C8000DF92EF92FF926B017C01E0914707F09188
:103C900048070684F785E02D8081816080830E943B
:103CA000F10C4091690450916A0460916B04709129
:103CB0006C04480F591F611D711D40936904509396
:103CC0006A0460936B0470936C04E0914707F09171
:103CD00048070480F581E02D11821082C114D104BF
:103CE000E104F10421F4C12CD12C7601C394A70185
:103CF000960144275527A8EEB3E00E94B483AB0198
:103D0000BC018FE397E0FF90EF90DF90CF900C9491
:103D1000A70DEF92FF920F931F93CF93DF938C0128
:103D2000D62FC0916E0561110E94BA0C87E0CF3F7B
:103D3000A9F18C9FD0011124A159BA4FEC9015968E
:103D40002D913C91169720173107B1F59EEF9C936A
:103D500090916E059C1333C0E0926E05A0916E05A4
:103D60008A9FD0011124A159BA4F11964D915D91AE
:103D70006D917C9114978E9DF0011124E159FA4FB9
:103D800081819281A381B4818A019B01080F191F4F
:103D90002A1F3B1FC901B8010E943F1ED1110E947A
:103DA000AF0C81E0CF3F09F480E0DF91CF911F910C
:103DB0000F91FF90EF900895FC2ECE2DB8CF8F9DE0
:103DC0009001112421593A4FF901E082FFEFEF16DB
:103DD00029F311964D915D916D917C9114978E9D73
:103DE000F0011124E159FA4F81819281A381B481BC
:103DF000840F951FA61FB71F81839283A383B4836B
:103E0000CDCF8F929F92AF92BF92DF92EF92FF92AF
:103E10000F931F93CF93DF937C014A015B01D22E56
:103E200021110E94BA0C10E000E0E7E0602FE09F53
:103E3000D001E19FB00D1124A159BA4FDC91DE3FB2
:103E400009F47BC00F5F1F4F0831110579F7D110BE
:103E50000E94AF0C81E0DE3F09F080E0DF91CF915E
:103E60001F910F91FF90EF90DF90BF90AF909F90C8
:103E70008F900895EC9FF0011124E159FA4F818150
:103E80009281A381B481EC2F70E047E02C2F30E0C9
:103E900088159905AA05BB0560F188199909AA0931
:103EA000BB09E7E0E29FA001E39F500D11244159B7
:103EB0005A4FFA0181839283A383B483E72F8091C1
:103EC0006E058C1332C060936E05C501B4010E946B
:103ED0003F1E87E0809FF001819FF00D1124E15982
:103EE000FA4FC08381829282A382B482F682E582F5
:103EF000AECF881A990AAA0ABB0A429FD001439FF3
:103F0000B00D1124A159BA4FCC914C9FD00111246E
:103F1000A159BA4F11968D919D910D90BC91A02DF4
:103F20007E2FCF3F61F2EC2FB1CF87E0E89FF00109
:103F30001124E159FA4F6083CCCFC0916E05CF3F79
:103F400009F098CFE0E0BBCFCF93DF9300D000D053
:103F50001F92CDB7DEB7811123C060E08BE298E2FB
:103F60000E94891E8091AC0684FF09C020E04CE4C9
:103F70005DE160E070E08BE298E20E94011F8091B9
:103F8000AC0683FF0DC05C8150786091B0067091E3
:103F9000B10629813A814B818091B2060E94E011DD
:103FA00080E092E027960FB6F894DEBF0FBECDBF3B
:103FB000DF91CF910C94701D8F929F92AF92BF9220
:103FC000CF92DF92EF92FF920E94F10CC0906904B1
:103FD000D0906A04E0906B04F0906C04C80ED91E77
:103FE000E11CF11C8090690490906A04A0906B041D
:103FF000B0906C040E94F10C880E991E8C149D04E4
:1040000019F7C701B601FF90EF90DF90CF90BF90F6
:10401000AF909F908F90089560931F067093200635
:104020008093210690932206645D7E4F8F4F9F4FB1
:1040300060931B0670931C0680931D0690931E06CA
:1040400082E080937C040E94DC1F6093780470936C
:10405000790480937A0490937B0408950F931F93BF
:104060000E94DC1F8B019C014091780450917904DF
:1040700060917A0470917B0480911F0690912006D4
:10408000A0912106B0912206041B150B260B370BBD
:10409000083E134021053105C0F00196A11DB11D58
:1040A00080931F0690932006A0932106B0932206CA
:1040B00048515C4F6F4F7F4F409378045093790481
:1040C00060937A0470937B04CBCF40911B06509190
:1040D0001C0660911D0670911E0684179507A607A1
:1040E000B70770F0E0912306F0912406309741F075
:1040F0001995611571058105910569F00E940C20E3
:1041000060911F06709120068091210690912206F1
:104110001F910F91089580911F0690912006A09104
:104120002106B0912206845D9E4FAF4FBF4F809312
:104130001B0690931C06A0931D06B0931E0681E0FB
:1041400090917C04911101C080E080937C04D8CFD1
:1041500020914604260F3327331F21323105ECF41A
:1041600020911507FC0190E080E0243069F082E0A6
:104170000895A09146042191AC014A5D5B4FA40FC4
:10418000B52FB11D2C930196861798F380914604A4
:10419000680F6093460480E0089581E008951092CE
:1041A000150781E0809314071092EF0661E084E127
:1041B0000E944C0F61E085E10E944C0FE9EBF0E0BA
:1041C00080818E7F808380818D7F808388E480934F
:1041D000B80085E48093BC000895CF93DF9391E00D
:1041E000909325048823B9F0C091B800D091BA000B
:1041F0008091BC008A7B8093BC0060E084E10E94D7
:104200004C0F60E085E10E944C0F0E94CF20D093BC
:10421000BA00C093B800DF91CF910895CF92DF929A
:10422000EF92FF920F931F93CF93DF93D0913E07AE
:1042300081E0D13208F09CC0C0913D070E94E20F9E
:104240006B017C018091150781116CC082E0809325
:10425000150781E0809314078FEF80931307109266
:104260001207D0931107ADE1B7E0E1EFF6E080E08F
:10427000D8138DC01092F0068091F006CC0FC82B99
:10428000C093F0068091EF06813009F084C010924F
:10429000EF060E94E20F6B017C018091F006809393
:1042A000BB008091170790911807A0911907B09152
:1042B0001A07892B8A2B8B2BA1F00E94E20F009109
:1042C0001707109118072091190730911A076C19D8
:1042D0007D098E099F09061717072807390708F473
:1042E00042C08091BC0083FDD8CF85EC8093BC0098
:1042F0000E94E20F6B017C0180911507823009F466
:104300004CC0809113078F3F09F469C08091130757
:10431000803209F466C080911307803309F463C0CA
:1043200084E026C08091170790911807A091190783
:10433000B0911A07892B8A2B8B2B09F483CF0E940B
:10434000E20F00911707109118072091190730917B
:104350001A076C197D098E099F0906171707280788
:10436000390708F06FCF809116070E94ED2085E095
:1043700010921C0710923E0710921B07DF91CF91FD
:104380001F910F91FF90EF90DF90CF9008959D9136
:1043900091938F5F6DCF85EEA9CF80911707909194
:1043A0001807A0911907B0911A07892B8A2B8B2B1C
:1043B00009F4A2CF0E94E20F00911707109118078D
:1043C0002091190730911A076C197D098E099F09F0
:1043D000061717072807390708F08ECFC4CF80E0EB
:1043E000C7CF82E0C5CF83E0C3CF0F931F93CF9396
:1043F000C1E00E94E20F009115081091160820916B
:10440000170830911808601B710B820B930B6938E9
:1044100073418105910570F480911908C0931B07C1
:1044200080933D0710921C0710923E070E940E21B8
:104430008111DFCFCF911F910F910895CF92DF921D
:10444000EF92FF920F931F93CF93DF93D82FC62F36
:10445000613208F098C00E94E20F6B017C018091EC
:10446000150781116BC081E08093150780931407B5
:104470009FEF90931307109212079C0F90931107D0
:104480008093F0068091F006DD0FD82BD093F006D4
:104490008091EF06813009F078C01092EF060E94FB
:1044A000E20F6B017C018091F0068093BB0080914C
:1044B000170790911807A0911907B0911A07892B37
:1044C0008A2B8B2BA1F00E94E20F0091170710910D
:1044D00018072091190730911A076C197D098E0968
:1044E0009F09061717072807390708F448C0809165
:1044F000BC0083FDD8CF85EC8093BC000E94E20F06
:104500006B017C0180911507813009F440C08091D6
:1045100012078C1710F4C0911207E1EFF6E0AFEC30
:10452000B6E080E08C1355C08C2FDF91CF911F91A6
:104530000F91FF90EF90DF90CF9008958091170733
:1045400090911807A0911907B0911A07892B8A2B0F
:104550008B2B09F484CF0E94E20F00911707109172
:1045600018072091190730911A076C197D098E09D7
:104570009F09061717072807390708F070CF8091A1
:1045800016070E94ED20C0E0CFCF85EEB5CF809119
:10459000170790911807A0911907B0911A07892B56
:1045A0008A2B8B2B09F4AECF0E94E20F00911707E4
:1045B000109118072091190730911A076C197D097D
:1045C0008E099F09061717072807390708F09ACFA1
:1045D000D6CF91919D938F5FA5CFE091CE0680912C
:1045E000CD06E81730F4F0E0E153F94F808190E018
:1045F00008958FEF9FEF08959091CE068091CD069C
:104600002FEF3FEF981748F4E92FF0E0E153F94F0F
:10461000208130E09F5F9093CE06C901089580917C
:10462000CD069091CE06891B990B0895CF92DF920B
:10463000EF92FF920F931F93CF93DF937C01CB01F7
:104640008A0120911B07222389F0EB016B01C40E24
:10465000D51ECC15DD0569F06991D701ED91FC916E
:104660000190F081E02DC7011995F3CF642F0E94CE
:10467000A820C801DF91CF911F910F91FF90EF907B
:10468000DF90CF900895CF93DF931F92CDB7DEB721
:10469000698320911B072223F9F020913E072032E5
:1046A00058F021E030E0FC013383228390E080E089
:1046B0000F90DF91CF91089580911C07E82FF0E0D3
:1046C000E35EF84F998190838F5F80931C078093FE
:1046D0003E0781E090E0ECCF61E0CE0101960E94C0
:1046E000A820F7CFCF93C62F91E090931B0798E6B1
:1046F00090933D0710921C0710923E07682F89E0A7
:1047000098E00E9443236C2F89E098E00E944323A5
:10471000CF910C940E21FC01808190ED980F9A307E
:1047200038F09FEB980F81E09A3118F080E00895FF
:1047300081E008954E962091290630912A0682172D
:10474000930720F080912B0690912C060895FF92FC
:104750000F931F93CF93DF938C01C0912B06D091C1
:104760002C06E0912506F0912606B801CE01199598
:10477000C8010E948B23F82ECE010E949A23EC01DF
:10478000F1100EC080912B0690912C068C179D077E
:1047900040F382E0DF91CF911F910F91FF90089538
:1047A00080E0F8CFCF92DF92EF92FF920F931F93AA
:1047B000CF93DF93EB01E82EF12C20912B06309163
:1047C0002C064EE1849FC00111248217930778F1D3
:1047D0000091290610912A06C801821B930B6EE1F5
:1047E00070E00E942D83E616F70608F58EE1C82ECC
:1047F000D12CC901B6010E942D836E157F0540F4AE
:1048000020173107A0F4C9010E949A239C01F1CF1F
:104810002017310760F4E0912506F0912606BE01CD
:10482000C9011995CE010E948B2381110AC082E033
:10483000DF91CF911F910F91FF90EF90DF90CF907C
:10484000089580E0F5CFAF92BF92CF92DF92EF92C2
:10485000FF920F931F93CF93DF93CDB7DEB76E9781
:104860000FB6F894DEBF0FBECDBF6C017B018B018C
:104870005C0188E0A80EB11CE0912506F0912606A7
:10488000BE016F5F7F4FC8011995DE011196F601D9
:104890009D918191981751F0C8010E949A238C0133
:1048A000E816F90649F70FEF1FEF03C0EA15FB05FD
:1048B00079F7C8016E960FB6F894DEBF0FBECDBF74
:1048C000DF91CF911F910F91FF90EF90DF90CF90EC
:1048D000BF90AF900895CF93DF93EB0160912B06CB
:1048E00070912C060E9423248F3F980779F0209125
:1048F0002B0630912C06821B930B6EE170E00E9418
:104900002D83688380E0DF91CF91089582E0FBCF13
:104910008F738A3010F4805D0895843210F4895CBE
:1049200008958E3310F4835C08958E3311F080E285
:1049300008958FE50895982F80ED890F8A3090F0C3
:104940008FEB890F8A3118F489EC890F08958FE96C
:10495000890F8A3110F483ECF8CF9F3511F08FE383
:1049600008958EE30895089590E080E00895462F1D
:10497000E82FF0E0E25DFC4F608184ED860F83302C
:1049800020F48FEF97E00C942C0D8EEF860F823081
:1049900018F48BEE97E0F7CF85EF860F823018F48E
:1049A00085EF97E0F0CF08952F923F924F925F925C
:1049B0006F927F928F929F92AF92BF92CF92DF922F
:1049C000EF92FF920F931F93CF93DF9300D000D00D
:1049D00000D01F92CDB7DEB79A878987DC01169683
:1049E0000D90BC91A02DB887AF839696ED91FC9168
:1049F00080809180C280D380E480F5800681178119
:104A00006085718542855385A484B58466847784E6
:104A10004088518822883388848995899E838D8334
:104A2000A689B789BC83AB83808D918D9A83898356
:104A3000228D338D848D958DAF81B885ED91FC915C
:104A40008082A985BA851696ED91FC911797028010
:104A5000F381E02D90821696ED91FC9117970480DA
:104A6000F581E02DC0821696ED91FC911797068096
:104A7000F781E02DD0821696ED91FC911797008476
:104A8000F185E02DE0821696ED91FC911797028456
:104A9000F385E02DF0821696ED91FC911797048432
:104AA000F585E02D00831696ED91FC91179706840D
:104AB000F785E02D10831696ED91FC91A089B189C0
:104AC0006D937C93A289B3894D935C93A489B58936
:104AD000AD92BC92A689B7896D927C92A08DB18D62
:104AE0004D925C92A28DB38D2D923C92A48DB58D8A
:104AF0004D815E814D935C93A68DB78D4B815C811A
:104B00004D935C93A0A1B1A149815A814D935C93CF
:104B1000A2A1B3A12D933C9304A0F5A1E02D918314
:104B200080832A960FB6F894DEBF0FBECDBFDF910B
:104B3000CF911F910F91FF90EF90DF90CF90BF909A
:104B4000AF909F908F907F906F905F904F903F902D
:104B50002F900895CF93DF93CDB7DEB766970FB64A
:104B6000F894DEBF0FBECDBF463009F441C08F3789
:104B700009F43EC08617E1F14130C1F49091B306CB
:104B8000392F331F3327331F2091B406922F9F7381
:104B9000990F932B98132EC080E066960FB6F89469
:104BA000DEBF0FBECDBFDF91CF91089596E1E7E262
:104BB000F2E0DE01119601900D929A95E1F7FE0167
:104BC00031969E01295E3F4F9191981729F3E21784
:104BD000F307D1F7423091F69091B3069F7789178A
:104BE000D9F2453029F52091B706922F987799F59B
:104BF00081E0D3CF322F3295369536953370909130
:104C0000B506292F2F71220F220F232B281721F2EF
:104C1000292F2295269527709091B6069F70990F9F
:104C2000990F990F922B981709F4B6CF4330A1F63C
:104C30009091AB06292F269526959091AC06917000
:104C40009295990F990F907C922B891709F4A4CF14
:104C5000443071F2C8CF9091B606392F32953F702B
:104C6000922F97709295907F932B891708F2269533
:104C7000269526952F70290F3327331F8217130689
:104C80000CF0B6CF89CFFC01D9014150423040F43D
:104C900080818E3749F48181863321F487E38183D3
:104CA00081E0089586E3FBCF8F3479F481818E36DD
:104CB00029F486E6818382831C92F2CF8EE681837B
:104CC00080E2828381E08C93EBCF893541F08E3492
:104CD00061F489E5808385E6818383E7F2CF8EE402
:104CE00080838FE6818380E2E6CF8B3229F08D329C
:104CF00031F48BE28083E0CF8DE28083E3CF883490
:104D000049F480E280838CE481838FE4828387E5A9
:104D10008383D2CF88E4808399E4918397E492835C
:104D20008383D0CFCF93C82F9091B706692F60951A
:104D3000661F6627661F8091B606282F22952F7062
:104D4000892F87708295807F822B8C0F0E944C0F59
:104D500085E08C9FF0011124E65AF94F9081903143
:104D600020F4CF01CF910C94701DCF9108958AB596
:104D7000877F8ABD0895CF93DF93CDB7DEB766975F
:104D80000FB6F894DEBF0FBECDBF982F8F37B9F0A6
:104D900086E1E7E2F2E0DE01119601900D928A953C
:104DA000E1F7FE0131969E01295E3F4F81919817F0
:104DB00041F0E217F307D1F781E0963418F480E070
:104DC00001C081E066960FB6F894DEBF0FBECDBF7E
:104DD000DF91CF910895F2980895F29A61E08BEEF9
:104DE00096E20E94891E61E081E097E20E94891E9E
:104DF00021E040E355E760E070E08BEE96E20C9432
:104E0000011F60E08AE00E944C0FF0980895CF9255
:104E1000DF92EF92FF92F2992DC0F49902C0F59BB8
:104E200029C00E94DC1F6B018091ED039091EE037D
:104E30009601281B390BC9018D3D9540D8F0F09B98
:104E400013C00E940127D092EE03C092ED0321E02F
:104E50004CED55E060E070E087E097E2FF90EF9066
:104E6000DF90CF900C94011F61E08AE00E944C0F0C
:104E7000F09AE9CFFF90EF90DF90CF900895F79AE6
:104E80000895CF92DF92EF92FF92CF93682F8AB569
:104E900060FB84F98ABDF79B21C0F7988091B30627
:104EA0008F778F3741F09091AC0696FD02C091E06C
:104EB00069270E944C0F61E08FE397E20E94891EF0
:104EC00021E040E65AEE60E070E08FE397E2CF9198
:104ED000FF90EF90DF90CF900C94011FC0916E0572
:104EE000611137C00E94BA0CC12CD12C760127E089
:104EF000CF3F39F12C9FF0011124E159FA4FC081C5
:104F000081819281A381B481C80ED91EEA1EFB1E45
:104F1000858196818D5D974259F70E94AF0CCD280F
:104F2000CE28CF2809F043C061E081E297E40E94D7
:104F3000891E21E040E355E760E070E08DED97E2E7
:104F4000C6CFC12CD12C7601E8CFC12CD12C760153
:104F50001BC00E94BA0CC12CD12C760187E0CF3F38
:104F6000A1F38C9FF0011124E159FA4FC0814181D6
:104F7000528163817481C40ED51EE61EF71E258101
:104F800036812152374459F70E94AF0CCD28CE28E4
:104F9000CF2869F461E08DED97E20E94891E21E03F
:104FA00040E355E760E070E081E297E490CFCF9175
:104FB000FF90EF90DF90CF90089588EE93E00E94ED
:104FC000701D80E00C944127CF92DF92EF92FF9208
:104FD0000F931F93CF93DF930E942E206B017C01D0
:104FE0000E94E81CE0917004E150D0E0E73020F42A
:104FF000F0E0EC51FD4FD081C701B6010E94E81CE2
:1050000000916F04C02FCF71C701B6010E94E81C48
:1050100010916E041F73C701B6010E94E81C9091A5
:105020006D04892F8F73602F6295607FDF706D2B09
:10503000110F7C2F72957F70979599279795712BFB
:10504000792B8695DF91CF911F910F91FF90EF9073
:10505000DF90CF900895FF920F931F93CF93DF932C
:10506000D091AA06D695D1700EE213E0F801C19155
:105070008F0184ED8C0F8330D0F46C2F8FEF97E08D
:105080000E94000D50E040E0D81711F040E050E2DF
:105090006C2F8FEF97E00E94720D83E005331807A5
:1050A00029F7DF91CF911F910F91FF9008958EEF17
:1050B000F82EFC0EF1E06C2F8BEE97E0FF1530F42C
:1050C00085EF8C0F823088F485EF97E00E94000D09
:1050D00040E050E2D81302C050E040E0E1E06C2F25
:1050E0008BEE97E0EF15B8F604C040E050E2DD2308
:1050F00099F385EF8C0F823080F66C2F85EF97E067
:10510000CACF0F931F93CF93DF932091AB06E22F6B
:10511000E695E6952091AC0621702295220F220F8C
:10512000207C2E2B8FE7820F8F77853470F0809153
:105130004D0790914E0723E0969587952A95E1F7C4
:10514000DF91CF911F910F91089530E0F901E75958
:10515000F94E8491F901E15FF84E0491F901E753AA
:10516000F94E1491112301F181110E94E50EE12FF6
:10517000F0E0EE0FFF1FE155F94EA591B491EC91CF
:105180000E2331E020E009F430E0832F922F2091AC
:10519000AC0626952170C22F20E0D22FC817D90760
:1051A00009F4C5CF80E0CCCF90E080E0F0CFFC01E7
:1051B0008081811108C089E898E06181428164178B
:1051C00028F40C94A71A82E598E0F7CF0895CF93BE
:1051D000C0E08C2F0E949226CF5FC031D1F7CF91D3
:1051E00008950C94E7288FE00C9492268EE00C949E
:1051F00092268DE00C9492268CE00C9492268BE003
:105200000C9492268AE00C94922689E00C949226C3
:1052100088E00C94922687E00C94922686E00C9409
:10522000922685E00C94922684E00C94922683E0EA
:105230000C94922682E00C94922681E00C949226A3
:1052400080E00C9492260F931F93CF93DF93EC0191
:10525000088119818A81811708F436C0812F90E076
:10526000FC01E15FF84E24918753994EFC01849133
:105270008823E9F02223D9F0622F70E0AB0141507E
:10528000510942235723452B91F490E0880F991F31
:10529000FC01EB5CF94E45915491FC01E15BF94E48
:1052A000A591B491FA018081282329F48C9161E0C1
:1052B000812F0E947A0F61E0011101C060E0812F0F
:1052C0000E944C0F1F5FC6CFDF91CF911F910F91AE
:1052D0000895EF92FF920F931F93CF93DF93CDB773
:1052E000DEB76E970FB6F894DEBF0FBECDBFDC0100
:1052F000EC91E250ED32B8F5F0E0E151FD4F108154
:10530000173088F511968C91119701E012969C91B7
:10531000911101C000E0E12EF12CF701ED5AF94F97
:10532000282F2F71220F220F90819378922B00FB50
:1053300090F99083BE016F5F7F4F0E94D22381114D
:1053400012C086E18E9DD0018F9DB00D1124AF5A01
:10535000B84FFE01399601900D928A95E1F7602FC2
:10536000812F0E94B7246E960FB6F894DEBF0FBE51
:10537000CDBFDF91CF911F910F91FF90EF900895D6
:10538000AF92BF92CF92DF92EF92FF920F931F9353
:10539000CF93DF937B01C42ED12C8C01BB24B3941B
:1053A0001C141D040CF046C00E94F521C6012FE11B
:1053B000C216D10414F08EE190E0E801C07EA02E68
:1053C000AE01405E5F4F9C01200F311FC01BC05ECD
:1053D000421753070CF0C82F80911908B0921B0791
:1053E00080933D0710921C0710923E07612F89E0C1
:1053F00098E00E9443236A2D89E098E00E944323AD
:10540000D0E0AE01B70189E098E00E9416230E9427
:105410000E210E94E20F6093150870931608809386
:10542000170890931808CC1ADD0A0C0F1D1FEC0EFC
:10543000FD1EB6CFDF91CF911F910F91FF90EF909E
:10544000DF90CF90BF90AF900895CF93E091E703A6
:10545000E150E83090F5F0E0E655FD4FC081CF3FD8
:1054600061F18091E603811110C081E08093E60331
:1054700044EF51E060E070E020E085E29AE20E94B3
:10548000011FC0930502CF910895853040F48F5FCE
:105490008093E6034DE451E060E070E0EDCF4BE433
:1054A00050E060E070E08C3038F78F5F8093E60367
:1054B00046EA50E060E070E0DFCF1092E603E3CF11
:1054C0001F93CF93DF93EC0181E080931B0788E665
:1054D00080933D0710921C0710923E0760E089E020
:1054E00098E00E9443230E940E21182F811180C052
:1054F00067E088E60E941E221092CE068093CD06B9
:1055000089E098E00E94FC228F77282F30E094E019
:10551000359527959A95E1F7922F990F990F291BA9
:10552000220F820F888389E098E00E94FC229C0170
:1055300044E0359527954A95E1F72F703327922F50
:10554000990F990F291B220F820F898389E098E018
:105550000E94FC228F7B282F30E054E03595279560
:105560005A95E1F7922F990F990F291B220F820F5D
:105570008A8389E098E00E94FC228B8389E098E08E
:105580000E94FC229C0164E0359527956A95E1F71D
:105590002F703327922F990F990F291B220F820FFB
:1055A0008C8389E098E00E94FC228F77282F30E0DE
:1055B00074E0359527957A95E1F7922F990F990F19
:1055C000291B220F820F8D8389E098E00E94FC2224
:1055D0009C01E4E035952795EA95E1F72F70332794
:1055E000922F990F990F291B220F825E280F2E836D
:1055F000812FDF91CF911F910895CF92DF92EF928B
:10560000FF921F93CF93DF93CDB7DEB72E970FB6E0
:10561000F894DEBF0FBECDBF18E0CE0101960E9408
:10562000602A8111FACFCE0108960E94602A81116A
:10563000F4CFCE0101960E94431B6B017C01CE0189
:1056400008960E94431B6C157D058E059F0529F069
:10565000115019F760E070E0CB012E960FB6F89468
:10566000DEBF0FBECDBFDF91CF911F91FF90EF90B6
:10567000DF90CF900895CF9391E090931B0798E629
:1056800090933D0710921C0710923E07682F89E007
:1056900098E00E9443230E940E2181110DC061E019
:1056A00088E60E941E221092CE068093CD0689E0E5
:1056B00098E00E94FC22C82F8C2FCF910895CF93A1
:1056C000DF93D82F8FE00E943B2B2D2F2150330BDF
:1056D000A90121E030E001C0220F4A95EAF7982F96
:1056E0009223A1F02095C22FC823D8E06C2F8FE021
:1056F0000E947223D15021F481E0DF91CF9108956F
:105700008FE00E943B2BC81789F3F6CF80E0F5CFDE
:10571000CF9382E10E943B2BC82F81E10E943B2B5B
:105720002C2F382F37FF02C0215C3F4FC90126E0E4
:10573000959587952A95E1F7CF910895DF92EF929D
:10574000FF920F931F93CF93DF9300D000D01F924F
:10575000CDB7DEB729833A834B835C836D837E8329
:105760008F83822F8F708A3008F05CC0822F8295E1
:105770008F70032F01700295007F082B083108F00D
:1057800051C0F32EF6948F2D8F73F82E8BE38F1567
:1057900008F448C0832F881F8827881F142F1F7183
:1057A000110F182BF69A0E942E200E94E81CE09000
:1057B0007004812F0E949819D82E8F2D0E9498195D
:1057C000F82E802F0E949819082F8E2D0E9498196C
:1057D000E82E6894E7F818E06D2D87E00E947223A8
:1057E0006F2D88E00E947223602F89E00E9472234F
:1057F0006E2D8AE00E9472238AE00E943B2BE816FD
:1058000011F090E00BC089E00E943B2B0813F9CF08
:1058100088E00E943B2B91E0F812F3CF115081F009
:105820009923D1F227960FB6F894DEBF0FBECDBFF5
:10583000DF91CF911F910F91FF90EF90DF9008952E
:105840009111F0CF88E027960FB6F894DEBF0FBE17
:10585000CDBFDF91CF911F910F91FF90EF90DF901F
:105860000C945F2BBF92CF92DF92EF92FF920F9337
:105870001F93CF93DF93EC01B62EC72EED84E1107A
:1058800004C00E94770C81110EC01B861D861C86E9
:1058900080E0DF91CF911F910F91FF90EF90DF900B
:1058A000CF90BF90089540E060EFCE010E94430C7E
:1058B000D12C01E011E0CE010E94F00BF82ECE01B8
:1058C0000E94F00B91E0F91218C0813099F5113463
:1058D000E0F2EB86E11002C081E08D878B818823A6
:1058E000A1F22396EB2DFC2DCF010896299121934F
:1058F000E817F907D9F781E0CCCFED2DF0E0F812E9
:105900000FC08B851817A0F4DE01AE0FBF1F1396D2
:105910008C91802379F4F12C193008F41C87E12E46
:10592000EC0FFD1F8381902F9095892383830AC0FC
:105930008113F1CFFE01ED0DF11D8381802B838357
:10594000FF24F3946F2DCE010E94140C1F5F000FF3
:1059500011F4D39401E087E08D1508F0ACCFB7CFF8
:10596000EF92FF920F931F93CF93DF937C018B01F4
:10597000D42FDC011596ED91FC91138615861486C3
:10598000128611861086178216821582148213825F
:10599000C0E0B801F701858196810E94322C8823EE
:1059A00029F0DC1759F0CF5FDC1798F780E0DF9122
:1059B000CF911F910F91FF90EF90089567E0C8017C
:1059C0000E94E00BD80117969C918913ECCF81E0DF
:1059D000EECFBF92CF92DF92EF92FF920F931F9381
:1059E000CF93DF93CDB7DEB761970FB6F894DEBFE4
:1059F0000FBECDBF8C016B01F42E8CE08417D8F460
:105A00009CE0F92EB601C8010E94791A8F1119C0C5
:105A1000BB24B3948B2D61960FB6F894DEBF0FBEF6
:105A2000CDBFDF91CF911F910F91FF90EF90DF904D
:105A3000CF90BF900895E9E04E1720F789E0F82E47
:105A4000E1CFAE014F5F5F4FB601C8010E94331A2C
:105A5000B82E8823F9F2F60180818031C9F2FBE08B
:105A60008FE5FF1651F08CE0F81631F0EAE08FE197
:105A7000FE1203C08FE301C08FE78D83AE014F5F3D
:105A80005F4FB601C8010E94E019F80181818F15AE
:105A900008F48F2DF801F81610F08183B9CFF18248
:105AA000F12CE12CF80184818E151F0409F00CF40F
:105AB000B1CF4E2DBE01665F7F4FC8010E94B02C52
:105AC000F801D180BE01665F7F4FC8010E94791A3C
:105AD0008D1540F4F8018181F8018183FFEFEF1A01
:105AE000FF0AE0CFBE01665F7F4FC8010E94791AAE
:105AF000F3CF7F928F929F92AF92BF92CF92DF921D
:105B0000EF92FF920F931F93CF93DF93CDB7DEB742
:105B1000A4970FB6F894DEBF0FBECDBF8C016C0109
:105B200081E2C80ED11C4801EEE08E0E911CB60138
:105B3000C4010E94791A782E68E0C6010E94E00B29
:105B400021E030E0811102C030E020E07901F8016D
:105B500087A1811106C086A1811103C081A188326D
:105B600021F07901FFEFEF1AFF0AAE014F5F5F4F9F
:105B7000B601C8010E940E1B811107C0AE014F5F24
:105B80005F4FB601C8010E940E1B69E0CE0101966D
:105B90000E94E00B811111C08E818F3F19F08FEFB1
:105BA000E81AF80A8F819FEF980F903160F599817C
:105BB000903509F52A81253019F587EF870D843056
:105BC00028F4472DB601C4010E94E92C8E2DA4961D
:105BD0000FB6F894DEBF0FBECDBFDF91CF911F91FE
:105BE0000F91FF90EF90DF90CF90BF90AF909F907C
:105BF0008F907F9008959F3F19F42A812730E9F212
:105C0000890F8F70D1F28885803109F0A3C0EFEF42
:105C1000EE1AFE0AC8010E94770CB601C8010E9464
:105C2000C11940E06EE4C8010E94430C6B8160958D
:105C300040E0C8010E94430C6C81609540E0C801BF
:105C40000E94430C40E06FE3C8010E94430CC8016E
:105C50000E94770CAE01465F5F4FB601C8010E94FB
:105C60000E1B811107C0AE01465F5F4FB601C80130
:105C70000E940E1B8B8180959C85981305C08C819A
:105C800080959D85981719F08FEFE81AF80A8E8590
:105C90008F3319F0EFEFEE1AFE0A9F858E8198136D
:105CA00008C098898F81981304C0998988859817AE
:105CB00019F0FFEFEF1AFF0AC8010E94770CB60136
:105CC000C8010E94C11940E06EE4C8010E94430C63
:105CD00040E06B81C8010E94430C40E06C81C80128
:105CE0000E94430C40E06FE7C8010E94430CC801CA
:105CF0000E94770CAE014D5E5F4FB601C8010E9455
:105D00000E1B811107C0AE014D5E5F4FB601C80189
:105D10000E940E1B8F898F3719F08FEFE81AF80A4F
:105D2000998D288D8F85281307C08889891304C011
:105D30002A8D8989281719F0EFEFEE1AFE0A8B8950
:105D4000803561F48C89853009F037CF913108F0C6
:105D500034CF12C0F2E0EF0EF11C5CCF8F3F29F47C
:105D60008C89873009F029CFF1CF9C3009F025CFFD
:105D7000845F8F7009F021CF86E0A82EB12CF1E06E
:105D8000AF1AB10809F419CFC8010E94770CB60107
:105D9000C8010E94C11940E064E4C8010E94430C9C
:105DA0006EEE72E080E090E00E940710A895AE01D0
:105DB000445E5F4FB601C8010E940E1B811107C0EF
:105DC000AE01445E5F4FB601C8010E940E1B8C8D70
:105DD000803569F49D8D953091F29AA19C3069F4DB
:105DE000845F8F7061F28FEFE81AF80AE6CE8F3F7A
:105DF000A1F79D8D973089F7C2CF890F8F7099F7E2
:105E0000DCCE2F923F924F925F926F927F928F9251
:105E10009F92AF92BF92CF92DF92EF92FF920F9339
:105E20001F93CF93DF9300D000D000D0CDB7DEB763
:105E30008C010E94DC1F4B015C01F80182A593A537
:105E4000A4A5B5A524013501481A590A6A0A7B0A96
:105E500086A9882309F452C0F8EE4F16F3E05F06D6
:105E60006104710408F44AC0C8010E94770C8823B9
:105E700021F140E06CECC8010E94430C40E06EEB65
:105E8000C8010E94430C9E012F5F3F4F79016E01B4
:105E90003AE0C30ED11C1701C8010E94A519D70111
:105EA0008D937D01CA16DB06B9F768E0C1010E9437
:105EB000E00B9985891709F4D3C0F80186A58F5F97
:105EC00086A7D12C833008F49AC07801FEE0EF0E4B
:105ED000F11C680121E2C20ED11C40E0B601C701ED
:105EE0000E94B02C882309F4A4C0D80199964C9143
:105EF000B601C7010E94E92CF80116A6F801D0A846
:105F0000DD2009F4C0C0E1A5E9508EEE92E0E33057
:105F100038F4F0E0EE0FFF1FE85DFC4F80819181C7
:105F2000B0E0A0E0481659066A067B0608F4ABC04C
:105F3000D80153968D919C910E94F00BF80196A583
:105F4000813009F0C7C058013EE0A30EB11C9F5F2D
:105F5000D8019E969C939E97D0961C924801B1E2E0
:105F60008B0E911CAE014F5F5F4FB401C5010E94C3
:105F7000331AC82E882391F1EA80F12CFE2CEE24EE
:105F8000FF0CFF0CFF0C8981E8E08E9FC0011124FB
:105F9000E82AF92AD80191968C918031C9F4688554
:105FA00070E08F81FB01E81BF109CF019695982FD6
:105FB0008827979587950E94418360517109E3E096
:105FC000EE0CFF1CEA95E1F7F0E8EF22E60EF71E73
:105FD00021E8E21624EEF2060CF090C0D8019E965D
:105FE0001C929E9781E0D6968C93D69780E8D196A6
:105FF0008C93D197D2961C92D297D5961C928D2DC8
:1060000029960FB6F894DEBF0FBECDBFDF91CF91BA
:106010001F910F91FF90EF90DF90CF90BF90AF90C6
:106020009F908F907F906F905F904F903F902F90B8
:10603000089581E0D801D6968C93D69780E8D196C2
:106040008C93D197D2961C92D297D5961C92F80138
:1060500082A693A6A4A6B5A610AADD24D394CFCF7A
:10606000D8019E961C929E97D6968C91D697813099
:1060700009F044CFD0961C92B8EE4B2EB3E05B2EC5
:10608000612C712C3BCFF8EE4F16F3E05F066104F4
:10609000710418F3F80116A6838994890E94770C7D
:1060A00040E06CECD80153968D919C910E94430C7A
:1060B000F801468564E4838994890E94430CD801E1
:1060C0009A968D929D92AD92BC929D9781E0D096CA
:1060D0008C93C3CF28EE421623E05206610471046C
:1060E00008F031CF933008F4B8CF82E086AB80E877
:1060F00081AB12AA15AA10AA16A681CFF80116A67E
:10610000C701880F892F881F990B81AB97012F77C3
:10611000332744E6429FC001439F900D1124880F0E
:10612000892F881F990B82AB83A9823874F4AE0142
:106130004F5F5F4FB401C5010E94331A882309F4F1
:1061400044C08C81D801D3968C93F801D3A884A93C
:1061500082386CF4AE014F5F5F4FB401C5010E94FD
:10616000331A8823A1F18B81D801D4968C93F8013E
:1061700064A96D1531F184E0F594E7948A95E1F70F
:10618000FD2D28E0F202E018F108112424E62E9DEE
:10619000C0012F9D900D1124062E000C770B6D1958
:1061A0007109D7FC739523E0660F771F2A95E1F7F5
:1061B0000E9441836038710564F08FE7D801D5965D
:1061C0008C93F80116AADC2C1ACF81E8BBCF81E8AA
:1061D000CBCF6038BFEF7B0724F480E8F80185ABB4
:1061E000F0CFD801D5966C93ECCFCF92DF92EF929F
:1061F000FF920F931F93CF93DF9300D000D01F9295
:106200001F92CDB7DEB7FC0167A76F37A9F480E80E
:1062100081AB12AA15AA81E086AB28960FB6F89436
:10622000DEBF0FBECDBFDF91CF911F910F91FF90C9
:10623000EF90DF90CF9008958C010E94B60F780107
:106240008EE0E80EF11CD8015396ED91FC91549725
:10625000138615861486128611861086178216827A
:1062600015821482138252961C92DD24D394BE01AF
:106270006F5F7F4FF801838994890E94322C8823B5
:1062800009F452C067E0CE0101960E94E00B9885A8
:106290008913EDCFD8011E968C911E97811125C0D0
:1062A00053968D919C910E94770CBE016F5F7F4F3A
:1062B000F801838994890E94C11940E064EBD801F8
:1062C00053968D919C910E94430CF8018389948987
:1062D0000E94F00BC82ED80153968D919C910E947C
:1062E000770CC11002C0F801D686D8011F96CC9059
:1062F000BE016F5F7F4FC7010E94791A8C1568F449
:10630000F8018785D8011F968C931F9752968C9120
:1063100052978F5F52968C93AACFBE016F5F7F4FCB
:10632000C7010E94791AEECF6801B1E2CB0ED11CF1
:1063300040E0B601C7010E94B02CF80141A5B601AA
:10634000C7010E94E92CD80150961C925097D6960E
:106350001C92D697D0961C92F80112A613A614A6EA
:1063600015A65BCFCF93DF93EC016FE70E94B60FCA
:106370008FED9BE098A38F8FDC8BCB8B1A8A1E86C8
:1063800089E08F8781E0888B898B1EA618AA90E808
:106390009BAB9CAB1DAA2AE029A72FE72FA799AB9F
:1063A0001AAA8EABDF91CF910895FF920F931F939E
:1063B000CF93DF93EC01F62E8A01262F660F330B65
:1063C000E885F985828982171306F9F461E00E9455
:1063D0007A0FE885F9850190F081E02D8081806851
:1063E0008083A8016F2DCE010E94720DE885F9858A
:1063F0000280F381E02D80819C81892B8083DF9155
:10640000CF911F910F91FF900895838982171306F2
:1064100059F461E00E947A0FE885F9850190F081D6
:10642000E02D80818062DCCF848982171306C9F653
:1064300061E00E947A0FE885F9850190F081E02DF6
:1064400080818860CDCF2F923F925F926F927F9232
:106450008F929F92AF92BF92CF92DF92EF92FF9274
:106460000F931F93CF93DF938091CC06882309F479
:10647000F8C01092CC068091CB06811125C0E09126
:10648000C906F091CA063097F9F02091490730917A
:106490004A0740914B0750914C07C0914F07D0914C
:1064A0005007A3E2B0E00E94B48335E1969587954A
:1064B000779567953A95D1F79E0143E036952795F4
:1064C0004A95E1F7822F19958091490790914A07E3
:1064D000A0914B07B0914C07892B8A2B8B2B41F451
:1064E00080914F079091500790934E0780934D07EE
:1064F000E0904D07F0904E07C701B3E09695879561
:10650000BA95E1F727E6289F3001299F700C1124E6
:10651000672C77246694669420E5269DC001279D0C
:10652000900D11249701281B390BADECB0E00E94AF
:106530009E834B015C010EE213E0C9E4D7E085E3E2
:10654000282E83E0382E63018FEFC81AD80ACC0CAE
:10655000DD1C660C771CF80151908F01F0E2EF16FC
:10656000F3E0FF0609F08FC04C8D5D8D84ED850D45
:10657000833008F0AAC0652D8FEF97E00E94D531D7
:1065800066962016310639F720914D0730914E0757
:1065900080914F07909150072817390709F4B6C02A
:1065A0008091CB06811139C06091490770914A07EB
:1065B00080914B0790914C0720914F0730915007E5
:1065C00040914D0750914E074217530708F08EC077
:1065D00020914F073091500740914F07509150073D
:1065E000E0914D07F0914E074E175F0708F083C00A
:1065F00040914F0750915007241B350B50E040E06D
:106600000E94558320931D0230931E0240931F0267
:106610005093200281E08093CB0640911D0250915F
:106620001E0260911F027091200221E08091C70636
:106630009091C8060E94011F20914D0730914E078E
:1066400080914F07909150072817390708F058C0DC
:1066500080914D0790914E07019690934E0780933D
:106660004D07DF91CF911F910F91FF90EF90DF9039
:10667000CF90BF90AF909F908F907F906F905F90E2
:106680003F902F900895FE01E60DF71D0084F185DF
:10669000E02DDE01AC0DBD1D18960D90BC91A02D16
:1066A000AE1BBF0BA50194010E94B483AB01BC01DA
:1066B000505E6F4F7F4FAEE0769567955795479543
:1066C000AA95D1F74E0F5F1F51CF8EEF850D823007
:1066D00020F4652D8BEE97E051CF85EF850D82304C
:1066E00008F04ECF652D85EF97E048CF20914D07FC
:1066F00030914E0771CF40914D0750914E077CCF9E
:1067000080914D0790914E070197A7CF1092CB062D
:10671000E091C506F091C606309709F4A2CF20910A
:10672000490730914A0740914B0750914C07C0915F
:106730004F07D0915007A3E2B0E00E94B48325E157
:1067400096958795779567952A95D1F79E0143E0B1
:10675000369527954A95E1F7822FDF91CF911F91CA
:106760000F91FF90EF90DF90CF90BF90AF909F90F0
:106770008F907F906F905F903F902F901994853607
:1067800008F084E628E0829FC0011124909350070E
:1067900080934F0781E08093CC06109249071092B6
:1067A0004A0710924B0710924C070C942332CF9358
:1067B000C82F0E9481288C0F853618F4CF910C9435
:1067C000BF33CF91089581E08093CC060C9423329F
:1067D000CF93DF93EC011092CB061092CC0661E0D0
:1067E0008091C7069091C8060E94891E0E94812848
:1067F0000E94BF332A8130E0A0E6BAEE0E949E8359
:106800006093490770934A0780934B0790934C0716
:1068100081E08093CC068881853608F084E628E004
:10682000829FC00111249093500780934F07DF91FE
:10683000CF910C942332CF93DF93EC0160E08E81F3
:106840000E944C0F61E08E810E944C0F60E08E81AF
:106850000E944C0F8BE891E00197F1F7DF91CF9107
:106860000895CF92DF92EF92FF920F931F93CF93F1
:10687000DF936C017C0187E0E80EF11CD0E0C0E002
:10688000062F10E0B8010C2E02C0759567950A948A
:10689000E2F76170F70181917F010E944C0F219610
:1068A000C430D10579F7C601DF91CF911F910F91C7
:1068B000FF90EF90DF90CF900C941B34CF92DF923B
:1068C000EF92FF920F931F93CF93DF93EC01F62E7D
:1068D000642F8C810E944C0F8D818F3F19F060E0F6
:1068E0000E944C0F0F2D10E08F8584FF25C06E0194
:1068F00087E0C80ED11CF12CE12CB8010E2C02C08F
:10690000759567950A94E2F76170F60181916F01C0
:106910000E944C0FFFEFEF1AFF0A88E0E816F1041F
:1069200061F7CE01DF91CF911F910F91FF90EF9012
:10693000DF90CF900C941B34B80184E07595679577
:106940008A95E1F7CE010E9431346F2DCE01DF919F
:10695000CF911F910F91FF90EF90DF90CF900C940B
:10696000313440E0682F80EC98E00C945E34643061
:1069700008F063E09091D308691710F06FEF690F8A
:10698000E62FF0E0E054F74F9489890F80680C946B
:10699000B1340C94B734CF93DF93823029F49091C3
:1069A000CF0898609093CF088093D3081092D408B2
:1069B00080E48093D50880E18093D60880E58093B9
:1069C000D70861E08091C4080E947A0F8091C508C1
:1069D0008F3F19F061E00E947A0F61E08091C60854
:1069E0000E947A0FC0ECD8E09E01205C3840809174
:1069F000CF0884FD0BC084E090E02196281739076A
:106A000044F461E08E810E947A0FEECF88E090E03E
:106A1000F4CF8BE39DE00197F1F760E08091C4082B
:106A20000E944C0F60E08091C6080E944C0F80913C
:106A3000C5088F3F19F060E00E944C0F8091CF088D
:106A400084FD39C063E080EC98E00E943134CBE4EF
:106A5000D6E4CE010197F1F763E080EC98E00E9464
:106A600031342197F1F763E080EC98E00E943134F3
:106A700083E592E00197F1F762E080EC98E00E94F4
:106A800031348091CF0880620E94B13484E08093D9
:106A9000D0088CE00E94B13481E00E94B1348BE3D5
:106AA0009FE10197F1F782E08093D10886E0DF91C2
:106AB000CF910C94B13480620E94B1348BE496E49F
:106AC0000197F1F78091CF0880620E94B13483E58D
:106AD00092E00197F1F78091CF0880620E94B13473
:106AE000D0CF81E00E94B1348BE39FE10197F1F7B1
:106AF000089541E00E945E3481E090E008950F9394
:106B00001F93CF93DF938B0128E0829FC001112454
:106B100080640E94B134E801085F1F4F699180ECE6
:106B200098E00E947935C017D107C1F7DF91CF9166
:106B30001F910F9108956F927F928F929F92AF92C3
:106B4000BF92CF92DF92EF92FF920F931F93CF935A
:106B5000DF936B01C42FD0E08C010E94F521B12C92
:106B6000A12C77247394209709F443C0F09019085E
:106B700070921B07F0923D0710921C0710923E077F
:106B8000612F89E098E00E944323602F89E098E01C
:106B90000E9443230E940E216C2FC138D1050CF0B6
:106BA00060E8613208F060E28F2D0E941E22682E9C
:106BB0001092CE068093CD067601EA0CFB1C0C19D0
:106BC0001D0948018A189B0884010E0D1F1D5701DD
:106BD000AC18BD088091CE06681629F2209719F2EC
:106BE00089E098E00E94FC22F70181937F012197C0
:106BF000EBCFDF91CF911F910F91FF90EF90DF903E
:106C0000CF90BF90AF909F908F907F906F9008959E
:106C1000009769F0FC0101900020E9F73197AF017E
:106C2000481B590BBC0180EC98E00C94441090E098
:106C300080E00895AF92BF92CF92DF92EF92FF92E1
:106C40000F931F93CF93DF936C0110E0A12C00E012
:106C5000C12FD0E07601EC0EFD1EF701B080C60119
:106C60008A0D911DBB20D9F0FEE7BF1216C02196F8
:106C7000CC0DDD1D28812E3781F0F70110820E9496
:106C8000083682E0A82EA10EF701B0826881605319
:106C900080EC98E00E94793501501F5FD9CF0E94A7
:106CA0000836802FDF91CF911F910F91FF90EF90C9
:106CB000DF90CF90BF90AF900895CF93DF93EC011A
:106CC0008FEF840F823008F055C0D9018C91FB0101
:106CD000DB0161E09D91992321F09C37D9F76F5F2B
:106CE000F9CF4130A1F490E0019670E00E94418319
:106CF000D9018C9390E09F01DF014D91981770F4BA
:106D0000442399F04C3709F49F5FFD01F4CF8111C2
:106D100003C08FEF860FECCF8150EACFDF019D01DA
:106D20008D918C3711F08111FACFDE010D9000208A
:106D3000E9F7CD0101978C1B9D0B2E1B3F0B821792
:106D4000930708F49C01DE01AC01421B530B4C0F6E
:106D50005D1F60E2A417B50741F42E0F3F1FE21735
:106D6000F30729F041914D93FACF6D93F3CFC80FFC
:106D7000D91F188281E0DF91CF9108959C01CB014A
:106D80004EE150E0B9010C94DF82CF93DF9300D045
:106D900000D0CDB7DEB790912D06492F50E060911D
:106DA0002E0670912F06899F600D711D1124CE0152
:106DB00001960E94DF82FE013196CE010796219155
:106DC0002F3F69F4E817F907D1F780E026960FB650
:106DD000F894DEBF0FBECDBFDF91CF91089581E063
:106DE000F5CFEF92FF920F931F93CF93DF9300D0D5
:106DF00000D0CDB7DEB790913006891780F0FB0147
:106E0000108280E026960FB6F894DEBF0FBECDBF8D
:106E1000DF91CF911F910F91FF90EF9008958B011B
:106E200090912D06492F50E060912E0670912F060B
:106E3000899F600D711D1124CE0101960E94DF8291
:106E4000E9808E2D0E948824F8018083FA80F4E086
:106E5000FF9EC00111248C73E294E694E69493E0C3
:106E6000E9228E290E948824F8018183EB80F0E1D9
:106E7000EF9EC00111248073F2942FE0F2228F293B
:106E80000E948824F80182838E2D869586950E9423
:106E90008824F8018383EC808E2D0E948824F801D9
:106EA0008483FD80F4E0FF9EC00111248C73E29482
:106EB000E694E69433E0E3228E290E948824F801C8
:106EC0008583EE80F0E1EF9EC00111248073F2947F
:106ED0004FE0F4228F290E948824F80186838E2DAA
:106EE000869586950E948824F80187831086FE0186
:106EF0003196CE01079621912F3F21F4E817F9072B
:106F0000D1F77FCF81E07ECFCF93DF9300D000D049
:106F1000CDB7DEB7FB01418150E090819F739A01AC
:106F200066E0220F331F6A95E1F7922B9983228145
:106F300030E055954795559547954F70B901A4E0B8
:106F4000660F771FAA95E1F7462B4A83B4E0359583
:106F50002795BA95E1F72370438194E0499FA001FA
:106F60001124242B2B83458150E094819F739A0137
:106F700066E0220F331F6A95E1F7922B9C832681EE
:106F800030E055954795559547954F70B901A4E068
:106F9000660F771FAA95E1F7462B4D83B4E0359530
:106FA0002795BA95E1F72370478194E0499FA001A6
:106FB0001124242B2E8390912D06492F50E06091AF
:106FC0002E0670912F06899F600D711D1124CE0130
:106FD00001960E94EF8226960FB6F894DEBF0FBE90
:106FE000CDBFDF91CF9108959F92AF92BF92CF9284
:106FF000DF92EF92FF920F931F93CF93DF9300D016
:1070000000D01F921F92CDB7DEB7B82E6B018FE371
:1070100089838A838B838C838D838E838F838887F8
:10702000CE0101967C0110E000E0982EAF2CF60115
:10703000E00FF11F8491882351F00E949B24F701F7
:1070400081937F010F5F1F4F0830110581F7692D74
:107050007A2D8B2D0E94843728960FB6F894DEBFC8
:107060000FBECDBFDF91CF911F910F91FF90EF9099
:10707000DF90CF90BF90AF909F9008950F931F9394
:10708000CF938F37B1F08B01C82F80913006C8178E
:1070900058F080913006C81760F4B8018C2FCF915A
:1070A0001F910F910C94F4378C2F0E94C5368823C2
:1070B00081F3CF911F910F910895EF92FF920F935B
:1070C0001F93CF93DF9300D000D000D0CDB7DEB7B1
:1070D000611165C0FC01A681B781ED91FC9111970A
:1070E000E081E250ED3208F05AC0F0E0E151FD4F8E
:1070F000E080E7FC54C08C010E2C000CFF081296B7
:107100006D917C91C7018D5A994F7C01DC018C9166
:10711000869586958F710E94D223882341F0D801ED
:107120001696ED91FC91828193810E94A723F7012D
:10713000F080F0FAFF24F0F8D8011696ED91FC915A
:10714000A481B58181E08F258C930280F381E02DAD
:1071500088E0DE01119601900D928A95E1F719867B
:10716000AE014F5F5F4F61E0C8010E94A81049EA7D
:1071700053E0FF2011F040EB53E062E0C8010E94B1
:10718000A81081E029960FB6F894DEBF0FBECDBFE0
:10719000DF91CF911F910F91FF90EF90089580E0C4
:1071A000F1CFCF92DF92EF92FF920F931F93CF9385
:1071B000DF9300D000D000D0CDB7DEB7D82EC92ED7
:1071C0008901F90180814130A9F5853488F58F5F07
:1071D000F8018083CE0101967C01BC01F801808119
:1071E0000E94F136FF92EF92F80180811F928F93F7
:1071F0008CE897E09F938F931F9280E18F93CF92BB
:10720000DF920E94C37F0FB6F894DEBF0FBECDBFE2
:1072100081E029960FB6F894DEBF0FBECDBFDF9197
:10722000CF911F910F91FF90EF90DF90CF90089535
:1072300080E0CECF423071F6882311F08150C8CF64
:1072400085E4C6CFCF92DF92EF92FF920F931F9308
:10725000CF93DF93CDB7DEB72C970FB6F894DEBF90
:107260000FBECDBF7C01D62EC72EFC0180818E01C2
:10727000085F1F4F823009F462C0833009F462C096
:10728000813089F48BE297E09F938F931F9285E082
:107290008F931F930F930E94C37F0F900F900F90B7
:1072A0000F900F900F90F701638574858585968503
:1072B000AE014F5F5F4F0E940D1C97012F5F3F4F44
:1072C000F7018081823008F040C084E03F932F9323
:1072D0001F930F931F928F938A811F928F938B819D
:1072E0001F928F931F9283E08F938D811F928F93B4
:1072F0008E811F928F938F818E51990B9F938F93C5
:1073000089EF96E09F938F931F9284E28F93CF92A1
:10731000DF920E94C37F0FB6F894DEBF0FBECDBFD1
:107320002C960FB6F894DEBF0FBECDBFDF91CF9184
:107330001F910F91FF90EF90DF90CF90089586E21C
:1073400097E0A2CF82E297E09FCF85E0BFCF0F9377
:107350001F93CF93DF93CDB7DEB72F970FB6F89477
:10736000DEBF0FBECDBF5FEF540F5230B8F4F9014E
:10737000092F182F20814230E9F42F5F208321E06C
:1073800040E0BF01CE0101960E940C1D8823D9F078
:10739000612F702FCE0101960E94223981E02F9635
:1073A0000FB6F894DEBF0FBECDBFDF91CF911F9116
:1073B0000F910895211104C08FE0808320E0E0CF79
:1073C00021502083FBCF80E397E09F938F931F9200
:1073D00080E28F930F931F930E94C37F0F900F90B3
:1073E0000F900F900F900F90D9CFCF92DF92EF9226
:1073F000FF920F931F93CF93DF93D82EC92E122F96
:10740000032F413009F063C060912B0670912C0668
:10741000822F932F0E9423248F3F9807C9F1EC01FC
:107420006E978091290690912A06C817D90738F4DB
:1074300020912B0630912C06C217D30710F4EC01D3
:107440006E977E01E0912506F0912606612F702F40
:10745000C7011995812F902F0E948B23811118C08D
:107460008EE1E81AF1088091290690912A06E81623
:10747000F90638F420912B0630912C06E216F3061B
:1074800020F47C012EE1E21AF108CE15DF05D1F6D9
:107490000F931F9389EE96E09F938F931F9289E03D
:1074A0008F93CF92DF920E94C37F8DB79EB70896CD
:1074B0000FB6F8949EBF0FBE8DBF81E0DF91CF91D4
:1074C0001F910F91FF90EF90DF90CF900895423081
:1074D000F9F660912B0670912C06822F932F0E9453
:1074E00023248F3F9807A1F20E949A237C01EC018C
:1074F000E0912506F0912606612F702FCE01199597
:10750000812F902F0E948B238111C2CFCE010E9428
:107510009A23EC01E816F90659F7BACFCF92DF9219
:10752000EF92FF920F931F93CF93DF9300D000D081
:1075300000D0CDB7DEB7D82EC92E89018FEF840FCA
:107540008230F0F4F90180818C3009F458C060F485
:10755000833009F44BC08B3009F44CC0823081F485
:107560004130F1F583E00AC08D32C1F18E32D1F1A4
:107570008C3231F4413009F040C08DE2F801808353
:10758000CE0101967C01BC01F80180810E94F13698
:10759000FF92EF92F80180811F928F938FED96E01A
:1075A0009F938F931F928CE08F93CF92DF920E94D4
:1075B000C37F0FB6F894DEBF0FBECDBF81E0299622
:1075C0000FB6F894DEBF0FBECDBFDF91CF911F91F4
:1075D0000F91FF90EF90DF90CF900895413089F4A4
:1075E0008EE2CCCF413049F682E0C8CF4130E1F79E
:1075F0008BE0C4CF413009F0B5CF8CE0BFCF413034
:10760000B9F78CE2BBCF0F931F93CF93DF93D82FA3
:107610008B018091B706982F9695969596959F70B9
:107620002D2F30E092171306ACF0DD2399F0C091B6
:10763000B6069C2F92959F70C82FC770C295C07FC9
:10764000C92BC150CD0F44E06FE78C2F0E94AA25B3
:10765000811117C080EE95E09F938F931F928DE06C
:107660008F931F930F930E94C37F0F900F900F90E3
:107670000F900F900F90C801DF91CF911F910F9144
:107680000895B8016C5F7F4F8C2F0E94F13680E522
:10769000F801808381E3DA3008F480E3F801818324
:1076A0008D2F6AE00E942183905D92838AE3838319
:1076B000E2CFEF92FF920F931F93CF93DF937C0162
:1076C000D42F89019091B60692959F70C091B7060C
:1076D0008C2F87708295807F44E06FE7892B0E9412
:1076E000AA25882359F18C2F887741F1F8018081F0
:1076F000D130C1F4C695C695C695CF708C1780F46D
:107700008F5FF8018083B701F80180810E94033BFD
:1077100081E0DF91CF911F910F91FF90EF9008953D
:1077200081E0EFCFD23079F7823030F48C2F86951C
:10773000869586958F70E5CF8150E3CFB7018FE7AF
:10774000E5CFCF92DF92FF920F931F93CF93DF93FA
:1077500000D000D000D0CDB7DEB7F82E8B018FE778
:10776000F81220C08AEC95E09F938F931F928CE0D3
:107770008F931F936F930E94C37F0F900F900F9072
:107780000F900F900F90C80129960FB6F894DEBFA6
:107790000FBECDBFDF91CF911F910F91FF90DF9072
:1077A000CF900895CE0101966C01BC018F2D0E94EF
:1077B000F136DF92CF921F92FF9286ED95E09F9374
:1077C0008F931F928CE08F931F930F930E94C37F20
:1077D0000FB6F894DEBF0FBECDBFD5CF0F931F936A
:1077E000CF93DF93CDB7DEB72C970FB6F894DEBFFB
:1077F0000FBECDBF8C0161110EC0FC01A681B78107
:107800008D919C911197FC0180818130A1F128F02C
:10781000823009F441C080E023C012960D90BC91E3
:10782000A02D9091B306892F881F8827881F9091DB
:10783000B4069F73990F982B9C93D8011696ED91DF
:10784000FC910280F381E02DBE016F5F7F4F80814C
:107850000E94A13BAC0161E0C8010E94A81081E038
:107860002C960FB6F894DEBF0FBECDBFDF91CF913F
:107870001F910F91089512960D90BC91A02D90919B
:10788000B406892F82958695869583709091B5066A
:107890009F71990F990FCFCF12960D90BC91A02D8B
:1078A0009091B506892F8295869587709091B6063E
:1078B0009F70990F990F990FBECF81508930C0F4F6
:1078C000E82FF0E0EE0FFF1FEE52FD4F8081918117
:1078D0009F938F931F9283E08F937F936F930E9468
:1078E000C37F0F900F900F900F900F900F900895FF
:1078F0008EE795E0EDCF0F931F93CF93FC018901A5
:107900009081933561F1A4F49634E1F0C1E09D34A7
:10791000D1F0413089F5C0E0CF5FBF018C2F0E94CC
:107920005D3CF801C08381E0CF911F910F910895D4
:10793000943579F0973569F78181C8E0853619F477
:10794000C3E001C0C5E0413039F3423031F7C150E6
:10795000E4CF8181C4E08537B1F7C2E0F4CF818103
:10796000813621F0853721F4C7E0EDCFC6E0EBCFBB
:10797000413029F0C9E0E9CFC9E0423071F2C0E0FE
:10798000CCCF4F925F926F927F928F929F92AF92E5
:10799000BF92CF92DF92EF92FF920F931F93CF93FC
:1079A000DF93CDB7DEB7CE54D1090FB6F894DEBF62
:1079B0000FBECDBF8C014B01DC013C91832F8F703A
:1079C0008A3008F09AC032953F7011969C91292F09
:1079D00021702295207F232B283108F08EC09695A8
:1079E0009F739C3308F089C05E01BCE4AB0EB11CF0
:1079F000B5010E945D3CF80183818F779E012B5B6E
:107A00003F4F7901823009F497C1C8F5882309F402
:107A10009DC0813009F46DC1D80111968C911197E8
:107A2000982F96959F732C9122952F708170829537
:107A3000807F822B13962C9127FF1EC227E0AE0178
:107A4000415E5F4F5F934F93FF92EF921F929F9320
:107A50001F928F93BF92AF921F922F938BE196E06C
:107A60009F938F931F9283E28F939F928F920E9496
:107A7000C37F0FB6F894DEBF0FBECDBF4FC0DE018F
:107A80005F966D01833009F4C4C1843029F68EE31A
:107A900096E09F938F931F9287E08F93FF922F938F
:107AA0000E94C37FBE016F5F7F4FD80115968C91F6
:107AB0000E94D22388E0FE013196DE01DC9601901F
:107AC0000D928A95E1F725961FAE2597BE01605D60
:107AD0007F4FF80184810E94A13B9F938F93CE0139
:107AE000CC969F938F9385E396E09F938F931F92FD
:107AF00081E18F93DF92CF921CC180EC96E09F933F
:107B00008F931F9283E28F939F928F920E94C37FE5
:107B10000F900F900F900F900F900F90C25BDF4F60
:107B20000FB6F894DEBF0FBECDBFDF91CF911F918E
:107B30000F91FF90EF90DF90CF90BF90AF909F900C
:107B40008F907F906F905F904F9008958581968180
:107B50009E012F5F3F4F6901981330C0B901892FF3
:107B60000E94A13BD80114968C91882321F187EAC9
:107B700093E09F938F938DEB96E09F938F931F924B
:107B800087E08F93FF92EF920E94C37FDF92CF92A4
:107B900085EB96E09F938F931F9281E18F93CE01A7
:107BA0004F969F938F930E94C37F0FB6F894DEBFCA
:107BB0000FBECDBF31CF8EEA93E0DBCFBE01605D5B
:107BC0007F4F0E94A13BB601D80116968C910E946E
:107BD000A13BF8018481882321F187EA93E09F93F8
:107BE0008F9382EB96E09F938F931F9287E08F9302
:107BF000FF92EF920E94C37F0FB6F894DEBF0FBED4
:107C0000CDBF612C80E0E0E3F0E0EC0FFD1FE80F5A
:107C1000F11D9081992399F08F5F9032A1F3682E26
:107C2000F2CF8EEA93E0DBCF782EF601E80FF11D5C
:107C30009081992339F08F5F9032B1F7F6CF712C94
:107C400080E0F3CF662D670D6031E0F041EF460F25
:107C500070E0262D671408F4272D30E0220F331F23
:107C6000429FC001439F900D1124860F971F0E94D1
:107C70002D836F5F70E075956795461B7614C0F491
:107C8000661A741ADE015F96FE01F09630E020E07D
:107C9000AD01862D90E066246394620E28173907A3
:107CA00054F46191662339F06D932F5F3F4FF3CF0A
:107CB000641A761AE7CF240F351F8DE2D9018C9311
:107CC000F601672D70E0862D90E09F012C193D098B
:107CD000261737074CF42191222331F06394840F47
:107CE000951FDC012C93EFCF480F591FFA0110822A
:107CF00093CE8EEA96E09F938F931F9287E08F93A7
:107D0000FF922F930E94C37FD80116968C911697ED
:107D10001F928F9314968C911F928F938CE996E00B
:107D20009F938F931F9281E18F93CE014F969F93E4
:107D30008F930E94C37F39CF8091B606982F92957A
:107D40009F708091B70687708295807F892B8150C4
:107D50009481FE0131963F01BF01890F0E94F136E7
:107D6000D80115969C91492E46944694937029E12A
:107D7000929F502C1124FE017F966F01882331F1D0
:107D80007F926F9286E996E09F938F931F9287E090
:107D90008F93FF92EF920E94C37FD80116968C9129
:107DA0001F928F931F925F921F924F92CE01079660
:107DB0009F938F938DE796E09F938F931F9281E11E
:107DC0008F93DF92CF920E94C37FEFCE86E796E03B
:107DD0009F938F931F9287E08F93FF92EF920E9461
:107DE000C37FD80116968C9116971F928F931F927E
:107DF0005F921F924F9214968C911F928F938DE5F4
:107E000096E09F938F931F9281E18F93DF92CF92A1
:107E1000DACF87E596E09F938F931F9287E08F9349
:107E2000FF922F930E94C37FD80116963C9116971C
:107E300015962C9115970F900F900F900F900F9013
:107E40000F9014968C918823A1F085EB93E01F92FC
:107E50003F931F922F939F938F9384E496E09F9379
:107E60008F931F9281E18F93DF92CF920E94C37F05
:107E70009CCE8AEB93E0EBCF26E0E1CDCF92DF9270
:107E8000EF92FF920F931F93CF93DF93CDB7DEB79F
:107E900065970FB6F894DEBF0FBECDBF6C017901B8
:107EA000F9012081822F8F708A3008F07EC03181E5
:107EB000832F81708295807F922F92959F70892B5E
:107EC000883108F072C0832F86958F738C3308F049
:107ED0006CC0413009F0A2C087E0DE011F9601901E
:107EE0000D928A95E1F70E944113811192C0009191
:107EF0004106109142062F85388949895A896B8934
:107F00007C898D890E9442148C0180914106909158
:107F100042060817190709F069C0C8010E94181223
:107F20008C01BC01CE0108960E94391240913F0697
:107F300050914006811116C02885322F32953F702E
:107F40008985982F91709295907F932B86958F734A
:107F50002F702A3038F4983128F48C3318F4041731
:107F60001507D8F20417150709F040C087E0FE0195
:107F70003896DE01119601900D928A95E1F787E01F
:107F8000FE013196DE01189601900D928A95E1F777
:107F900087E0FE013896D70101900D928A95E1F7AE
:107FA000B601C7010E94C13C11C08FEC96E09F93BF
:107FB0008F931F9280E18F93DF92CF920E94C37FB5
:107FC0000F900F900F900F900F900F9081E065969B
:107FD0000FB6F894DEBF0FBECDBFDF91CF911F91DA
:107FE0000F91FF90EF90DF90CF9008958091410620
:107FF00090914206B801685071098017910720F0EE
:1080000060913F0670914006CE0108960E94391299
:10801000ADCFCE0108960E94D611A8CF423009F00C
:10802000BFCF428153816481758186810E946F1622
:10803000F70120833183428353836483758386836E
:10804000AFCF2F923F924F925F926F927F928F921B
:108050009F92AF92BF92CF92DF92EF92FF920F93D7
:108060001F93CF93DF9300D01F92CDB7DEB77C83F1
:108070006B83342E3A8329834DB65EB62FEF240FDF
:10808000223008F0C1C0FB0101900020E9F72E2F3B
:10809000261B225040E0912C60E0022E000C330B96
:1080A000A42FB0E02A173B07C4F00B811C810A0FF4
:1080B0001B1FF8015081442319F0A217B30731F4B4
:1080C0005D3209F0D8C093944F5FEACF6D3219F05A
:1080D0005D3209F09394652FF7CF492D50E07A0176
:1080E000F1E0EF1AF108BA01660F771FADB7BEB71E
:1080F000A61BB70B0FB6F894BEBF0FBEADBFEDB752
:10810000FEB73196AB81BC816C90BDE2792C88249E
:1081100083946B1219C077247A94790C8701112704
:10812000BF01600F711FAFE5DA2EDB01DC92BF01EA
:10813000640F751F600F711FDB01DC92AB81BC8186
:1081400011966C90B2E08B2E5F01A40EB51E082D27
:1081500010E020173107A4F48F01DC016C9170E06E
:108160009716B9F1D8012D918D0162173CF09D0150
:108170002E0D3F1DD9012C91261764F57F5FF0CF9E
:108180007A94672D70E0AB81BC810A0F1B1FD80168
:108190002C906F01C60ED71EBDE22B1213C0D60164
:1081A0006C926A0D7B1DD80111961C91DB011C930A
:1081B000839483946B817C81680D711DDB016C90CD
:1081C0008394C5CFD6016C926A0D7B1DDB016C9246
:1081D000F1CF70E0272F30E0B1E03B1239C0DF0172
:1081E000A40FB51FA20FB31F7C9176132DC02F5F74
:1081F0003F4F241735072CF12081FC012083FC011F
:108200008081A981BA818C9381E00FB6F8945EBE1B
:108210000FBE4DBE0F900F900F900F90DF91CF913A
:108220001F910F91FF90EF90DF90CF90BF90AF9094
:108230009F908F907F906F905F904F903F902F9086
:108240000895E20FF31FD8CF6F5FDC016C93D7CF97
:10825000DF01A20FB31FAC91A6130BC0E40FF51FF3
:10826000711103C0EE0DFF1DC7CFE20FF31F319751
:10827000C3CF6150EACF6D3209F02CCF2CCF2F92B3
:108280003F924F925F926F927F928F929F92AF92A6
:10829000BF92CF92DF92EF92FF920F931F93CF93F3
:1082A000DF93CDB7DEB7E3970FB6F894DEBF0FBE0E
:1082B000CDBFA98EBA8ECB8EDC8EED8EFE8E0F8F4B
:1082C00018A329A33AA34BA35CA36DA37EA38FA3FA
:1082D0002DB73EB73BAB2AAB2A8D3B8D812C80E07E
:1082E0002115310579F0F901E80FF11D90819923ED
:1082F00049F0943229F49181943211F08F5F839484
:108300008F5FEECF482D4150550B5FA74EA78CE0F5
:10831000889EB001112479AB68AB912C16E05CE02B
:10832000752EE0914906F0914A0619958AEF810F62
:10833000823008F08CC1ADB7BEB7BDA7ACA7EDB712
:10834000FEB728A939A9E21BF30B0FB6F894FEBFBC
:108350000FBEEDBF4DB75EB74F5F5F4F59A748A740
:10836000E0914906F0914A061995512C412C312C87
:1083700090E0612C4A8D5B8D062D10E0FA01E00F34
:10838000F11FF080292F30E0FF2009F4B6C05AE039
:10839000F51204C03394512C6394ECCF539464E2EF
:1083A000F612FACF81818432B9F3639410828A8DF8
:1083B0009B8D820F931F0E944C11580E8A8D9B8DAE
:1083C000080F191FD801FC92442D50E0E8A5F9A52B
:1083D000749CE00DF11D11248FEF850D828733868B
:1083E0002A8D3B8D80E8F901E60DF11D108190ED9D
:1083F000910F9A3058F487FD07C0BAE08B9F802D0B
:108400001124890F6394EFCF80E0FBCF87FD14C068
:10841000749EF001759EF00D112468A579A5E60FF4
:10842000F71F880F990B6F8D78A1860F971FDC01BE
:108430008D919C9191878087749EF001759EF00DBF
:10844000112448A559A5E40FF51FA12F110FBB0B4F
:10845000A156B048AA0FBB1F8091510690915206B9
:10846000A80FB91F8D919C9191838083639463942D
:10847000260D311D35832483BF016C5F7F4F7BA7A1
:108480006AA75F0172E0A70EB11C0A8D1B8D91E0F7
:10849000960DE92EF12CF801EE0DFF1D2080D8017C
:1084A000A60DB11D8C918D3731F18CE2281221C0BF
:1084B000AAA5BBA5CD90DC901082C6010E944C11EC
:1084C000970121503109020F131F0C191D09080FC4
:1084D000500E8A8D9B8DE80EF91EF7012082639461
:1084E00063948A8D9B8D860D911DD5018D939C93F0
:1084F000CCCF692ECCCF43944FCFCA01820F931FAC
:108500000E944C1190E19519981B19164CF50DB766
:108510001EB7E92F092E000CFF0B9F012F5F3F4F65
:108520004DB75EB7421B530B0FB6F8945EBF0FBE3C
:108530004DBF2DB73EB72F5F3F4F422FD90150E2BD
:108540005D938A2F841B8917DCF3E20FF31F1082DF
:10855000C9010E944C110FB6F8941EBF0FBE0DBF8B
:10856000882009F4C3C0512C9CE2492E08A519A506
:10857000579C000D111D1124E0914706F09148060B
:10858000D8011B966C911B971A968C911995E091C6
:108590004D06F0914E061995682EBFEF8B1709F422
:1085A0009AC0F801E480F58080E05701A80EB11C64
:1085B000D5019C919C3211F08F5FF7CFF5011082AD
:1085C000D8011296CD90DC9080E01601280E311C67
:1085D000F101F081FAA7FD3711F08F5FF6CFD101DD
:1085E0001C9247E150E0B701CE0101960E945D88E0
:1085F000188EF801208531850190F081E02D462DFF
:10860000B601C7011995182FB701CE0101960E9436
:108610005488892B09F449C08EA19FA1892B09F4A4
:1086200044C0D5014C922AA5F1012083EEA1FFA1FF
:10863000652DCE0149961995882399F187E04CA5BF
:108640005DA50FB6F8945EBF0FBE4DBF182F143056
:1086500009F4A3C0153009F44FC0111112C0ECA1E8
:10866000FDA1309719F0CE014996199589A1811184
:108670004AC0E0914506F0914606CE01499619950B
:108680001FEF8CEF810F843008F44BCE123009F4C9
:108690005CC0133009F47FC0113009F057C015E0F9
:1086A00055C0D5011C92F1011082C7010E944C11E6
:1086B000112331F0F3E06F1210C0552019F05A94D5
:1086C00086E0682ED5014C922DE7F101208336E03B
:1086D000631609F44BCF862DB2CF6110F1CF2EA5D2
:1086E0003FA55216130674F75394EACFE0914D0656
:1086F000F0914E061995A3CF9A9489A1891518F483
:1087000099249A94980EAAA1BBA1A90DB11DE0913C
:108710004306F0914406AE01475E5F4F6C91CE0177
:1087200001961995A980BA80CB80DC80ED80FE800F
:108730000F81188529853A854B855C856D857E85F9
:108740008F850E943F41182F9CCF14E0CE0149969F
:108750000E94F610812F6AA97BA90FB6F8947EBFFC
:108760000FBE6DBFE3960FB6F894DEBF0FBECDBF50
:10877000DF91CF911F910F91FF90EF90DF90CF90FD
:10878000BF90AF909F908F907F906F905F904F9031
:108790003F902F90089516E0D9CF939489A1981611
:1087A00008F4B1CF912CAFCF4F925F926F927F922E
:1087B0008F929F92AF92BF92CF92DF92EF92FF92F1
:1087C0001F93CF93DF9300D01F921F92CDB7DEB7D8
:1087D000388DC98CDA8CEB8CFC8CEEE7F4E01FEF63
:1087E00040E050E0BA0190E080E02081432E421A40
:1087F00094150CF051C04385548565857685360106
:108800004701641A750A860A970AB401A301182F52
:10881000942D8F5F3F96803141F71F3FD9F02FE0B5
:10882000129FC0011124AC0142585B4F5A01FA015A
:1088300030839E01215E3F4F4D8D5E8D6AE070E07A
:1088400081589B4F0E940080F5011286C386D48612
:10885000E586F6861983CA82DB82EC82FD823C2D96
:108860004B815C816D81212F70E080E090E00F9062
:108870000F900F900F900F90DF91CF911F91FF906D
:10888000EF90DF90CF90BF90AF909F908F907F90B0
:108890006F905F904F9008954912BBCF838494846A
:1088A000A584B68426013701481859086A087B0850
:1088B00053014201481559056A057B0508F0A9CF07
:1088C000182FB301A201A5CF1F93CF93DF9300D040
:1088D00000D01F92CDB7DEB7182F8091AC0682FF73
:1088E0000DC05C8150786091AD067091AE06298113
:1088F0003A814B818091AF060E94E01160E08BE2EB
:1089000098E20E94891E80E092E00E94701D0E9401
:108910002E201F921F9324E735E03F932F939F93C0
:108920008F937F936F9381E08F930E94D443209322
:1089300000023093010240930202509303026093BD
:1089400004020FB6F894DEBF0FBECDBF27960FB658
:10895000F894DEBF0FBECDBFDF91CF911F91089578
:108960008F929F92AF92BF92DF92EF92FF920F93FE
:108970001F93CF93DF9300D01F921F92CDB7DEB726
:108980007C0189014150423008F06DC061E081EF07
:1089900098E20E94891EF70181818633B9F40E9412
:1089A000E7280E94DC1FF80181809280A380B480B8
:1089B000681979098A099B09618372838383948387
:1089C00087E3F7018183DD24D39429C021E040E3CC
:1089D00055E760E070E081EF98E20E94011FD82E19
:1089E0000E94DC1FF8016183728383839483DD20FE
:1089F00041F19091B706692F661F6627661F809127
:108A0000B60682958F7097709295907F982B9150B3
:108A10008081890F0E944C0F86E3F70181838D2DA1
:108A20000F900F900F900F900F90DF91CF911F91AB
:108A30000F91FF90EF90DF90BF90AF909F908F903D
:108A400008952EEE36E03F932F939F938F937F935D
:108A50006F9383E08F930E94D4430FB6F894DEBFE8
:108A60000FBECDBFB0CFFC018181863329F441E038
:108A7000C7010E94B044A7CFDD24D394873379F691
:108A8000F90181819281A381B481892B8A2B8B2B5F
:108A900031F6D12CC4CFEF92FF920F931F93CF9357
:108AA000DF9300D01F921F92CDB7DEB7FC018B0180
:108AB000DB0113968C91309709F496C021813281A5
:108AC0002115310509F490C0D9010D900020E9F776
:108AD0001197A21BB30B169708F486C091E0D90139
:108AE00015962C91273309F090E090FB87F9D80177
:108AF00013968C93A681B78112960D90BC91A02DF0
:108B00008C918F70D8019C91907F982B9C93A6811B
:108B1000B78114962D913C91D9018C918295807FDB
:108B20009F70982BD8019C93D9019C9194FB882726
:108B300080F9D80111969C9111979E7F982B1196E0
:108B40009C93A681B78116960D90BC91A02D8C9117
:108B50008F73880F9170982BD80111969C93119761
:108B600012968C911297807E12968C93E380F480FB
:108B7000D701EC91E43109F06BC01396ED91FC91B3
:108B80000680F781E02D0190F081E02D83818F77C1
:108B9000823009F4C5C050F5882309F47FC08130C4
:108BA00009F4A0C0C8010E94D6110E942E2021E124
:108BB00036E03F932F939F938F937F936F9383E040
:108BC0008F930E94D4430FB6F894DEBF0FBECDBF83
:108BD0000F900F900F900F900F90DF91CF911F91FA
:108BE0000F91FF90EF9008958F7781CF833009F434
:108BF000C8C08430B9F6D80113968C911397807849
:108C0000846013968C93D7011696ED91FC9117977B
:108C10000190F081E02D8081F801848319821696FD
:108C2000ED91FC91BE016F5F7F4F828193810E9425
:108C30006B248981D80115968C93D7011696ED91F6
:108C4000FC910480F581E02D808191E0892796C018
:108C5000E850EB3108F0BCCFF0E08827ED5CF94B31
:108C60008F4F0C94968372464E469046C146E84517
:108C7000FB45E845E845E845E845E845E845E84579
:108C8000E845E845E845E845E8457246E8454E468A
:108C9000E8459046E845C146E845FB45D8011396AE
:108CA0008C911397807813968C93D7011696ED913B
:108CB000FC9117970190F081E02D8081F801848369
:108CC0001696ED91FC910280F381E02D8081D80110
:108CD00015968C93D7011696ED91FC910480F58141
:108CE000E02D4BC0D80113968C911397807881604A
:108CF00013968C93D7011696ED91FC9117970190DE
:108D0000F081E02D8081F80184831696ED91FC912D
:108D10000280F381E02D8081D80116968C9358CF84
:108D2000F8018381807882608383D7011696ED9164
:108D3000FC9117970190F081E02D8081F8018483E8
:108D40001696ED91FC91A481B5818C9129E2829FC8
:108D5000C0011124969596950280F381E02D8081C3
:108D6000880F880F890FD80115968C93D701169616
:108D7000ED91FC910680F781E02D8081F8018683DA
:108D800027CFD80113968C911397807883608BCF6F
:108D9000EF92FF920F931F93CF93DF93182F062F1D
:108DA000F72EEA01E22E8881803118F4CA010E9470
:108DB000701D8FE7E816F9F0113021F50E942E2082
:108DC000FF920F9329E835E03F932F939F938F9362
:108DD0007F936F9382E08F930E94D44328833983DB
:108DE0004A835B836C838DB79EB709960FB6F89460
:108DF0009EBF0FBE8DBFDF91CF911F910F91FF904E
:108E0000EF9008951230B9F70E942E20FF920F9331
:108E100021E935E03F932F939F938F937F936F9337
:108E20001F930E94D443288339834A835B836C83D6
:108E30008DB79EB709960FB6F8949EBF0FBE8DBF33
:108E4000DACF88EE93E00E94701D0AB401FE25C0BF
:108E50008091B3068F778F3701F10E942E2021E891
:108E600035E03F932F939F938F937F936F9381E090
:108E70008F930E94D4432093E8033093E9034093F7
:108E8000EA035093EB036093EC038DB79EB707960C
:108E90000FB6F8949EBF0FBE8DBF81E00C944127A2
:108EA0004F925F926F927F928F929F92AF92BF92FA
:108EB000CF92DF92EF92FF920F931F93CF93DF93A6
:108EC000CDB7DEB7A7970FB6F894DEBF0FBECDBF04
:108ED000A895EEE7F4E08EE695E0DF012C912330D3
:108EE00009F499C01F968A179B07C1F720E020FD5F
:108EF000F59A20FFF5982081223009F48EC03F9624
:108F00008E179F07C1F780E080FDF49A80FFF498E8
:108F10000AB403FE84C0F6980E94DC1F6093F3033A
:108F20007093F4038093F5039093F603E0913D066C
:108F3000F0913E0619950E949C14811109C187E0A9
:108F4000E6E0F2E0DE01919601900D928A95E1F75C
:108F500087E0FE01B196DE01529601900D928A954E
:108F6000E1F78A898F708A3008F002C109A1902F39
:108F700092959F708AA1082F01700295007F092B9E
:108F8000083108F0F5C0182F16951F731C3308F030
:108F9000EFC0881F8827881F9BA0292D2F71922E34
:108FA000990C982A0E942E20AE014F5F5F4F0E94BD
:108FB0000D1C9B81802F891B091708F4885E9A81FC
:108FC000212F291B330BD9013CE3839FA00DB11D39
:108FD00011242CE330E00E94AD832B013C018981F8
:108FE000292D281B330BC901092E000CAA0BBB0B22
:108FF000A3019201280F391F4A1F5B1FA8EEB3E09F
:109000000E94B4836093EF037093F0038093F103A5
:109010009093F20322C021E06ACF81E075CFF699E8
:109020007ACF0E94DC1F0091F3031091F40320918A
:10903000F5033091F603601B710B820B930B0091CB
:10904000EF031091F0032091F1033091F203061722
:1090500017072807390708F45ECF0E942332809152
:10906000BF0890910C049817A9F02091B306922F95
:10907000991F9927991F2091B4062F73220F292B2E
:1090800048EF53E06FEB73E00E94C8468091BF0841
:1090900080930C048091880890910D049817B9F082
:1090A0002091B406922F9295969596959370209163
:1090B000B5062F71220F220F292B4DEF53E064ECE0
:1090C00073E00E94C8468091880880930D048091C7
:1090D000510890910E049817B9F02091B506922F7F
:1090E0009295969597702091B6062F70220F220FB9
:1090F000220F292B42E054E069EC73E00E94C8463D
:109100008091510880930E042091BF082223E9F139
:10911000809188088823C9F18AB58B7F8ABD8AB57A
:109120008D7F8ABD8AB58E7F8ABD87E094E00E94DC
:10913000701D0E94DD2703E01091F703113009F440
:1091400079C108F45EC0123009F47CC180E062C0CD
:109150000AB403FEF4CE81E00E945F2B21E042E3DB
:1091600050E060E070E087EB96E20E94011FE7CEDE
:1091700080E09CE5A0E0B0E08093EF039093F003E3
:10918000A093F103B093F20368CF9091BE08943698
:109190000CF0F3C18091870884360CF0EEC12111E8
:1091A00001C0892F87FF16C20AB401FCC4CF87E033
:1091B00094E00E94701D0E942E2023EA35E03F9328
:1091C0002F939F938F937F936F9382E08F930E944F
:1091D000D443209307043093080440930904509328
:1091E0000A0460930B048AB582608ABD8AB58B7FBE
:1091F0008ABD0E9421470FB6F894DEBF0FBECDBFD7
:109200009ACF8091B8088F3709F4A0CF89E898E009
:109210000E94012F1F5F133008F01CC11093F70349
:10922000811103C0015009F087CFF09912C08091DD
:1092300005028F3F71F0809105028F3F19F08FEF8B
:10924000809305020E94ED2661E08AE00E944C0FA7
:10925000F09AF19946C1F09B44C110910502CE01EC
:1092600001964C011F3F09F448C08FEF809305021F
:109270000E94ED26113009F4FEC0123009F4FFC03F
:1092800011113BC0F19AE0914306F091440650E081
:1092900040E060E0C4011995712CAA85BB85A70D3B
:1092A000B11DE0914306F0914406A4016C91CE01FA
:1092B00042961995AA88BB88CC88DD88EE88FF88FD
:1092C000088D198D2A8D3B8D4C8D5D8D6E8D7F8D1A
:1092D00088A10E943F41843009F0BFC073949985F2
:1092E000791608F0C6C09CEF980F9230B0F2873024
:1092F000A1F2C4010E94F610F1980E94DC1F209197
:10930000230430912404621B730B603A7F40B0F059
:1093100080911E04803108F0B4C08F5F80931E04DA
:1093200021E040E06EE174E08FE094E00E940C1DCB
:109330000E94DC1F70932404609323040E942E205B
:109340002B013C018091D0088D7F8093D0088860EC
:109350000E94B1348091D0088E7F8093D0088860BD
:109360000E94B13460E080E00E94B734C301B201D2
:109370000E94E81CE0917004E15080E0E73020F4A6
:10938000F0E0EC51FD4F8081B4010E945D3CC401CE
:109390000E94083663E080EC98E00E947935D09016
:1093A000BB08ED2C0D2C000CFF08E090BA080E2D28
:1093B0000E2C000C110BC301B2010E94E81C00919D
:1093C0006E04C301B2010E94E81CFF92DF921F935A
:1093D000EF921F920F9380916F041F928F9387EBF0
:1093E00095E09F938F931F928DE08F939F928F9222
:1093F0000E94C37FC4010E94083660E080EC98E0C0
:109400000E94793561E080E00E94B73400910F043A
:1094100011E00FB6F894DEBF0FBECDBF0023C1F13F
:1094200010E065E0013009F464E080EC98E00E940F
:10943000793530C0809181088F3709F487CE82E575
:1094400098E0E6CE80914A088F3709F47FCE8BE111
:1094500098E0DECE1092F703E3CE853009F043CFDB
:109460007A949985971508F03ECF77247A94790EEF
:109470003ACF712C38CF81E00E94D7333ECF8FEFA7
:10948000FBCF6EE174E08FE094E00E94681D50CF46
:1094900080E289830E94812820E134E0011102C02A
:1094A00021EE33E01F928F933F932F938CEA95E048
:1094B0009F938F931F928FE08F93C401810F911D13
:1094C0009F938F930E94C37FC4010E94083661E07E
:1094D00080EC98E00E9479350FB6F894DEBF0FBE9D
:1094E000CDBFF29905C0F49903C0F59B0E940127F6
:1094F0000E94072750E040E06DE085EF97E00E9472
:10950000720D809164008062809364008091640099
:1095100080688093640083B7816083BF889583B738
:109520008E7F83BF809164008F7D809364008091E3
:1095300064008F778093640085EF97E00E943F0E70
:10954000AB016DE085EF97E00E94720DA7960FB614
:10955000F894DEBF0FBECDBFDF91CF911F910F9169
:10956000FF90EF90DF90CF90BF90AF909F908F9043
:109570007F906F905F904F9008950AB402FC24C0D2
:1095800087E094E00E94701D0E942E2029E935E0BA
:109590003F932F939F938F937F936F9382E08F934B
:1095A0000E94D44320930704309308044093090495
:1095B00050930A0460930B048AB584608ABD0FB689
:1095C000F894DEBF0FBECDBF0E94DD278AB58D7F28
:1095D0008ABDB1CD882329F08091AC0687FF0E9417
:1095E000DD278091AC0687FF04C00AB404FE0E9408
:1095F00021478AB58B7F8ABD8AB58D7F8ABD87E07A
:1096000094E00E94701D97CDCF938091D008982F41
:1096100091609093D00889600E94B134F19B19C089
:10962000F29B17C0C0910502CF3F19F40E9450472A
:10963000F5CF8FEF809305020E94ED268091D00830
:109640008E7F8093D00888600E94B1348C2FCF9198
:109650000895CFEFF1CF8F929F92AF92BF92EF928A
:10966000FF920F931F93CF93DF9300D000D000D0D1
:10967000CDB7DEB7FC011081112309F483C09091AE
:10968000B7069695969596959F70911708F47AC0AF
:109690001150E12EF12C8180912CB12CA12CB82CF1
:1096A000AA2499248824A281B0E020E030E043E29B
:1096B00050E00E94B4839B01AC019BE05695479516
:1096C000379527959A95D1F7C501B4010E94558326
:1096D000BA01A901F701EE0FFF1FEE54FD4F20E084
:1096E000808191810E94011F882309F45CC0009150
:1096F000B606802F82958F706091B706062F07708F
:109700000295007F082B010F661F6627661F802FBA
:109710000E944C0FCE0101965C01BC01802F0E947B
:10972000F13685E08E9DF0018F9DF00D1124E65AF3
:10973000F94F9081903118F4CF010E94701D0E9462
:109740002E2025E02E9D80012F9D100D1124065AFC
:10975000194FBF92AF922FE635E03F932F939F931F
:109760008F937F936F9381E08F930E94D443F8018E
:10977000208331834283538364830FB6F894DEBF22
:109780000FBECDBF29960FB6F894DEBF0FBECDBF7A
:10979000DF91CF911F910F91FF90EF90BF90AF900D
:1097A0009F908F9008950E942E201F921F9327E66E
:1097B00035E03F932F939F938F937F936F9383E035
:1097C0008F930E94D443D9CFEF92FF920F931F93B0
:1097D000CF93DF93CDB7DEB7A3970FB6F894DEBF74
:1097E0000FBECDBF7C018B014EE150E0BC01C80132
:1097F0000E94EF82BE016F5F7F4FC7010E94BE369D
:10980000DE011196A801485F5F4FC801FC0131914C
:10981000CF012D91321791F180E0FA01DE01199606
:10982000025E1F4F882351F0E017F107D1F021911C
:1098300031918D919D9128173907B1F30E942E2007
:109840002DE535E03F932F939F938F937F936F93F5
:1098500083E08F930E94D4430FB6F894DEBF0FBE0F
:10986000CDBFA3960FB6F894DEBF0FBECDBFDF917C
:10987000CF911F910F91FF90EF9008958417950756
:1098800029F681E0CACFAF92BF92CF92DF92EF92DA
:10989000FF920F931F93CF93DF93CDB7DEB7CE0127
:1098A0000E96FC01A190B1907F019F01A50170E08F
:1098B00060E090E080E00E9400808E5F082F10E062
:1098C000C8010E9428876C019701A501B8010E9478
:1098D0000080C601DF91CF911F910F91FF90EF9013
:1098E000DF90CF90BF90AF900895CF92DF92EF922C
:1098F000FF920F931F93CF93DF9300D000D000D03F
:10990000CDB7DEB72E96EEACFFAC2E9729968FAD75
:10991000299782388CF4AE014F5F5F4FBE016A5CBD
:109920007F4FCE0183960E94331A882309F471C0B9
:109930008C8129968FAF299729960FAD29972A9662
:109940008FAD2A9782388CF4AE014F5F5F4FBE0116
:109950006A5C7F4FCE0183960E94331A882309F4F4
:109960005AC08B812A968FAF2A972A961FAD2A97C5
:1099700081EF800F853108F004E180EF810F89319C
:1099800008F01EE1812F012E000C990B9F931F936D
:10999000802F002E000C990B9F930F9386E497E085
:1099A0009F938F930E94434CF7019283818382E0BF
:1099B000858384E090E00E9428876C01F7019783FB
:1099C000868381E090E00E9428877C01F6019183E4
:1099D000808381E090E00E942887F6019383828350
:1099E000F7010083FC0110830F900F900F900F90F0
:1099F0000F900F9029960FB6F894DEBF0FBECDBF23
:109A0000DF91CF911F910F91FF90EF90DF90CF905A
:109A1000089581E88ECF81E8A5CF85ED8093BC00C5
:109A20008091170790911807A0911907B0911A0714
:109A30000796A11DB11D23E0B695A795979587952B
:109A40002A95D1F72091BC0024FD03C01092150780
:109A50000895409117075091180760911907709168
:109A60001A07452B462B472B69F30097A105B10533
:109A700041F02AE22A95F1F700C00197A109B10946
:109A8000E1CF809116070C94ED204F925F926F9278
:109A90007F928F929F92AF92BF92CF92DF92EF927E
:109AA000FF920F931F93CF93DF93CDB7DEB7C755C8
:109AB000D1090FB6F894DEBF0FBECDBF4C01DC015B
:109AC0008C918B3309F413C408F091C1803209F4EE
:109AD000A7C608F079C0883109F4A6C608F054C0BA
:109AE0008E3009F4B9C6813109F44BC6873009F0CC
:109AF000A3C0BE016F5F7F4FC4010E944B45998197
:109B0000292F22952F708A81982F91709295907F9E
:109B1000922B89F4982F9E7771F42B81922F9F714D
:109B2000990F382F331F3327331F932B21F480686D
:109B30008A83207E2B83D4011396ED91FC91808142
:109B4000843109F07FC60380F481E02D0680F7811F
:109B5000E02D0190F081E02DA980BA80CB80DC80DF
:109B6000ED80FE800F8120813181428153816481AB
:109B7000758186810E94F674882309F45DC00E9475
:109B80002E202CEF34E10AC48C3109F411C68E3139
:109B900009F426C68A3109F04FC05C8150785160C3
:109BA0005C831696ED91FC91A081B1816C916D83DF
:109BB0000280F381E02D80818F8329813A814B815E
:109BC0007E810E94E01138C08B3209F45AC668F5D4
:109BD000863209F409C28A3209F444C6823261F538
:109BE0008C81807884608C831696ED91FC91A081A5
:109BF000B1818C918D83BE01615E7F4F82819381A3
:109C00000E946B247F8D7E83D4011696ED91FC918A
:109C10000480F581E02D808191E089278F8329815F
:109C20003A814B815C816D81CCCF813309F4EDC6E3
:109C3000D8F48D3209F432C6C95ADF4F0FB6F89402
:109C4000DEBF0FBECDBFDF91CF911F910F91FF906F
:109C5000EF90DF90CF90BF90AF909F908F907F90CC
:109C60006F905F904F900895833309F4EEC286336E
:109C700019F71696ED91FC91A081B1811196CD90C6
:109C8000DD90ED90FC9014970280F381E02D20810F
:109C9000C114D104E104F10479F2222369F230E025
:109CA000A0E6BAEE0E949E83A70196010E9455830A
:109CB000122F0E9415132EA73FA748AB59AB6AABD2
:109CC0007BAB8CAB922F92959F70832F8170829586
:109CD000807F892B36953F732F702A3008F0ACCFE8
:109CE000883108F0A9CF3C3308F0A6CF87E0FE0109
:109CF000BE96DE01979601900D928A95E1F787E076
:109D0000FE01B796DE015F9601900D928A95E1F70C
:109D10002F8D38A149A15AA16BA17CA18DA10E94D0
:109D20006F162FA338A749A75AA76BA77CA78DA7A3
:109D30008AA18F778230D1F5D4011396ED91FC91F1
:109D40000680F781E02D0190F081E02D9BA18081BC
:109D500098132CC087E0FE017F96DE0111960190DA
:109D60000D928A95E1F71F83A980BA80CB80DC80B1
:109D7000ED80FE80012F2F8D38A149A15AA16BA142
:109D80007CA18DA10E94F674BE01625D7F4FCE0161
:109D90004F960E94C511882349F087E0FE01319655
:109DA000DE019E9601900D928A95E1F72FA1822FF8
:109DB0008F708A3008F040CF22952F7088A5982F99
:109DC00091709295907F922B983108F035CF8695BF
:109DD0008F738C3308F030CFBE01625D7F4FCE01B0
:109DE00087960E94C511882309F489CF25CF8B342B
:109DF00009F45BC608F07EC0833409F4CFC108F0D3
:109E00004FC08F3309F45CC2813409F487C18D33AC
:109E100009F012CF1696ED91FC910190F081E02DA2
:109E2000808191816DE770E00E942D831FEF160FF6
:109E3000912F9770990F990F8091AA06837E892B95
:109E40008093AA064EE050E060E078E08AEA96E06F
:109E50000E94EF8280E00E94BF33212F30E02F5F0D
:109E60003F4F032E000C440B550B60E47FE180E074
:109E700090E00E94778369017A01BA01A9018FEF0E
:109E800097E00E94A70DB701A6018BEE97E00E9414
:109E9000A70DB701A60185EF97E00E94A70DCCCED4
:109EA000863409F4EEC1E0F4853409F0C5CE809122
:109EB000AC0684608093AC061696ED91FC91A0816F
:109EC000B1818C918093AD06A281B3818C918093F6
:109ED000AE060480F581E02D80818093AF0653C1EA
:109EE000883409F4D4C1893409F0A6CE8091AC0637
:109EF000877FCAC1823609F460C308F053C0843535
:109F000009F461C28C3509F4BDC28F3409F094CED6
:109F10001396ED91FC9114970680F781E02D019046
:109F2000F081E02DF0801696ED91FC918E010F5F8F
:109F30001F4FCF014096A80121913191D9012C9159
:109F4000DA012D93AD018E179F07B1F71986809125
:109F50003006F81608F070CE8FE38F8F88A389A3A0
:109F60008AA38BA38CA38DA38EA35E01BFE1AB0E4E
:109F7000B11C6801E8E0CE0ED11C9A2CEB2CD80164
:109F80008D918D01882341F00E949B24F5018193DE
:109F90005F010C151D0599F7692D7E2D8F2D0E94EF
:109FA00084374ACE863709F4CEC360F4843609F08C
:109FB00043CE0E94DB1881113FCE0E94DC1F26E0B9
:109FC00035E1ECC1873709F4C9C3893709F034CECC
:109FD000A89588E19CE00FB6F894A895809360005E
:109FE0000FBE90936000FFCF1696ED91FC91A0817B
:109FF000B1818C918BA3A281B3818C918CA3A4811C
:10A00000B5818C918DA3A681B7819C9199A3008481
:10A01000F185E02D908198A31F8E825E8DA30E9412
:10A02000FD2A6B017C01CE014F960E94431B4B0120
:10A030005C01AE014F5F5F4F0E940D1C81E0809379
:10A040001B0788E680933D0710921C0710923E077D
:10A0500060E089E098E00E94432389810E9498197A
:10A06000682F89E098E00E9443238A810E94981912
:10A07000682F89E098E00E9443238B810E94981901
:10A08000682F89E098E00E9443236C8189E098E082
:10A090000E9443238D810E949819682F89E098E0DF
:10A0A0000E9443238E810E949819682F89E098E0CE
:10A0B0000E9443238F818E510E949819682F89E056
:10A0C00098E00E9443230E940E218FE00E943B2BC8
:10A0D000682F6F778FE00E947223C501B4010E9440
:10A0E0000C200E9458168091B8069091B906A09154
:10A0F000BA06B091BB06880D991DAA1DBB1D4C0167
:10A100005D018C189D08AE08BF088092B806909239
:10A11000B906A092BA06B092BB068ECD1696ED9106
:10A12000FC91A481B5818C91B3E08B9F90011124A7
:10A1300056E0359527955A95E1F7A281B3818C9128
:10A14000880F880F820F880F880F880F8595859557
:10A1500085950190F081E02D30812091AA069091A3
:10A16000AB06311119C0382F3295330F307E2F7165
:10A17000232B2093AA0686958695869583709C7FCF
:10A18000892B8093AB064EE050E060E078E08AEAED
:10A1900096E00E94EF8250CD8195E5CF1696ED9125
:10A1A000FC91A081B1818C912091AB06322F369524
:10A1B00036959091AC06292F21702295220F220FFF
:10A1C000207C232B482F50E024171506E1F5A281AF
:10A1D000B381969591702C919227382F330F330FBE
:10A1E0002091AB062370232B2093AB0686FB2227FE
:10A1F00020F98091AC068E7F822B8093AC06028082
:10A20000F381E02D208120FB81F98093AC06992316
:10A2100009F412CD4EE050E060E078E08AEA96E082
:10A220000E94EF829091AB06969596958091AC0630
:10A2300081708295880F880F807C62E775E1892B99
:10A240000E943E38F9CC91E0C8CF1696ED91FC9172
:10A25000A081B1819C90A281B381FC900480F581A2
:10A26000E02D008110E01F1509F436C444E06FE7CB
:10A27000812F890D0E94AA25882309F428C41F5F15
:10A28000F2CF8091AC068B7F8093AC067CCF80911F
:10A29000AC0688608093AC061696ED91FC91A08187
:10A2A000B1818C918093B006A281B3818C9180930F
:10A2B000B1060480F581E02D80818093B20663CFE2
:10A2C0001696ED91FC91A081B1819C918091AC0694
:10A2D00090FB84F98093AC060280F381E02D90819D
:10A2E0008091AA0690FB81F98093AA064CCF139621
:10A2F000ED91FC9114970680F781E02D0190F0819B
:10A30000E02DE081E250ED3208F058C0F0E0E1517C
:10A31000FD4FF080F7FC52C01696ED91FC91008144
:10A3200011810280F381E02DE080BE016F5F7F4FDD
:10A33000C8010E946B2481112DC081E0E8266F2D99
:10A340000F2C000C770BFB01ED5AF94F99819F718F
:10A35000292F220F220F90819378922BE0FA90F907
:10A36000908360527E4F41E050E0CF010E94EF8227
:10A3700086E1EF2DE802D0011124AF5AB84FF80161
:10A38000389601900D928A95E1F76E2D8F2D0E94DF
:10A39000B72452CC0E94DC1F26E535E13F932F9372
:10A3A0009F938F937F936F9383E08F930E94D44307
:10A3B0000FB6F894DEBF0FBECDBF3ECC0E94DC1FAF
:10A3C0002CE435E1EBCF1696ED91FC91BE01615E78
:10A3D0007F4F86A197A10E946B24811131C08E010D
:10A3E0000F5F1F4F86E1F80111928A95E9F749E462
:10A3F00057E090E080E0FC01ED5AF94F2081322FC8
:10A40000369536953F716F8D70E03617170651F40B
:10A410002378208326E1F801DA01189601900D9245
:10A420002A95E1F701964A5E5F4F8730910519F74B
:10A4300047E050E060EE71E083E596E00E94EF8235
:10A4400060912B0670912C06D4011696ED91FC912B
:10A45000808191810E9423248F3F980771F0BE0173
:10A460006F5F7F4F2EE1FB0111922A95E9F7E09192
:10A470002706F09128061995DFCB0E94DC1F22E405
:10A4800035E18CCF1396ED91FC910380F481E02DA2
:10A490000380F481E02D0380F481E02D0380F481BA
:10A4A000E02D0380F481E02D0380F481E02D038111
:10A4B00014814E01B9E08B0E911CFE01319640E1F2
:10A4C000A42EB12CD12C7F01D80116968D919C9190
:10A4D000DC01AA0DBB1D0D90BC91A02D0D90BC916F
:10A4E000A02D25E236E041E050E00E94B483D40183
:10A4F0008D939D934D01B7E0BD1568F0D801169678
:10A500008D919C91DC01AA0DBB1D50970D90BC91C3
:10A51000A02D8C918083D394B2E0AB0EB11C319608
:10A520002BE0D212D1CFD8018C918E3559F4C701CE
:10A530000E948176882309F47FCB0E94DC1F28E3E8
:10A5400035E12CCF833509F077CB1696ED91FC9150
:10A55000B70186A197A10E945576882329F00E9411
:10A56000DC1F2EE235E11ACFBE01615E7F4FC701CD
:10A570000E946B24811160CB49E457E030E020E079
:10A58000F901ED5AF94F8081869586958F716F8D0F
:10A5900070E08617170649F486E1FE013996DA0164
:10A5A000189601900D928A95E1F72F5F3F4F4A5E12
:10A5B0005F4F2730310521F73FCB1396ED91FC918A
:10A5C000E380F480DE01119690E080E0F7012681BF
:10A5D0003781F901E80FF91F0190F081E02D20810A
:10A5E0002D9302968031910589F7D70116960D912A
:10A5F0001C91D8015296ED91FC91608170E090E041
:10A6000080E00E94188520E030E048EC52E40E948F
:10A6100034844B015C01D8015096ED91FC9160812E
:10A6200070E090E080E00E9418859B01AC01C501BC
:10A63000B4010E94C8832B013C011A86198626EBBF
:10A64000822E24E1922E5E01BBE0AB0EB11CCC2425
:10A65000C394D12CCC0EDD1EECE1CE0ED11CF40146
:10A660002591359145915491C301B2010E94918683
:10A670000E94AE8420E030E040E056E40E949186E3
:10A6800020E030E040E05FE30E94C8830E94E7845E
:10A69000D5016D937D935D01B4E08B0E911CAC14DC
:10A6A000BD04E9F680E090E29E8F8D8FF7018081F6
:10A6B0008D3561F4CE0101960E948176882309F4DC
:10A6C000BBCA0E94DC1F24E235E168CE813609F066
:10A6D000B3CABE016F5F7F4FD80154968D919C9194
:10A6E0000E945576882329F00E94DC1F2AE135E17B
:10A6F00055CEBE01615E7F4FCE0101960E946B2454
:10A7000081119ACA49E457E030E020E0F901ED5A9E
:10A71000F94F8081869586958F716F8D70E08617D1
:10A72000170649F486E1FE013996DA011896019080
:10A730000D928A95E1F72F5F3F4F4A5E5F4F2730BA
:10A74000310521F779CA1396ED91FC910680F781C6
:10A75000E02D808191810E94701D6ECA1396ED914B
:10A76000FC910680F781E02D00811181C8010E94D3
:10A77000701DB801CE0101960E94681D8111F6CFAF
:10A780005BCA1696ED91FC910190F081E02D20813D
:10A790003181428153816481758186810E944F1885
:10A7A000882309F449CA0E94DC1F20E135E1F6CD77
:10A7B0005C8150785C83D4011696ED91FC91A08168
:10A7C000B1816C916D83A281B3817C917E83048081
:10A7D000F581E02D80818F8329813A814B81F1C9F8
:10A7E0005C81507852605C831696ED91FC91A0815B
:10A7F000B1816C916D83A481B5818C91B9E28B9FFD
:10A80000C0011124892F86958695A281B3817C9100
:10A81000770F770F780F7E830680F781E02DDACFF0
:10A820005C8150785360C6CF1696ED91FC910190F3
:10A83000F081E02D208131814281538164817581D5
:10A840008681BFC929813A814B815C816D817E817E
:10A850008F810E946B1790C913968D919C910E94D5
:10A86000454DEAC91696ED91FC91A281B381019004
:10A87000F081E02D4C91608189E898E00E94A71A50
:10A88000DBC91696ED91FC91A281B3810190F08114
:10A89000E02D4C91608182E598E0F0CF1696ED9125
:10A8A000FC91A281B3818C910190F081E02D908187
:10A8B000913009F470C0E8F1923009F0BDC92091DF
:10A8C000B506422F4295469547709091B606392FAE
:10A8D0003F70330F330F330F342B482F50E03417B2
:10A8E000150609F4A9C9382F3295330F307E2F7120
:10A8F000232B2093B506282F2695269526952F7075
:10A90000907F922B9093B60661EE74E18F770E9450
:10A910003E386091B506862F829586958770609146
:10A92000B6066F70660F660F660F682B8BE198E0B6
:10A930002FC03091B306432F441F4427441F9091EA
:10A94000B406292F2F73220F242B482F50E02417F1
:10A95000150609F471C980FB37F93093B306282F27
:10A9600026952F73907C922B9093B40663EF74E13D
:10A970008F770E943E386091B306862F881F882704
:10A98000881F6091B4066F73660F682B89E898E0A2
:10A990000E94F530F8CB2091B406422F429546959F
:10A9A000469543709091B506392F3F71330F330FA1
:10A9B000342B482F50E03417150609F43DC9382FC1
:10A9C0003295330F330F307C2F73232B2093B40633
:10A9D000282F269526952F71907E922B9093B50661
:10A9E0006AEE74E18F770E943E386091B406862F3C
:10A9F00082958695869583706091B5066F71660F16
:10AA0000660F682B82E598E0C3CF1696ED91FC9116
:10AA1000A081B1819C918091AC0686FB222720F910
:10AA20002917F1F190FB86F98093AC0621E00280B2
:10AA3000F381E02D90818091AC0687FB332730F9BC
:10AA4000391729F090FB87F98093AC0621E0D401F7
:10AA50001396ED91FC910680F781E02D0190F08135
:10AA6000E02D80819091B306392F3F77482F50E039
:10AA700034171506B9F08F779078982B9093B3061A
:10AA80006AED74E10E943E388091B3068F778F376C
:10AA900009F479CB61E00E947A0F0E94DD2773CB25
:10AAA00020E0C5CF21116FCBC7C81696ED91FC9160
:10AAB0000190F081E02D90818091AC0685FB2227EA
:10AAC00020F990FB85F9291709F4B6C8DDCB0E945F
:10AAD000DC1F2FE535E162CC8091B6068F70992D91
:10AAE0009295907F892B8093B606292D2295277009
:10AAF0008091B7068078912F9F70990F990F990FC9
:10AB0000822B892B00FB87F98093B7064EE050E03B
:10AB100060E078E08AEA96E00E94EF82B12CA12CF6
:10AB200081E008278AE6C82E85E1D82E99E0792EA3
:10AB3000CE0101967C01A11608F07EC8892C8A0CF2
:10AB400061E0882D0E947A0F602F882D0E944C0FA3
:10AB5000BFEFAB1ABB0ABF92AF92DF92CF921F92A8
:10AB60007F92FF92EF920E94C37FB701882D0E94CF
:10AB70003E380FB6F894DEBF0FBECDBFDCCFBF921C
:10AB8000CF92DF92EF92FF920F931F93CF93DF93B9
:10AB900000D000D000D0CDB7DEB7C82EB92ECB0183
:10ABA000142F7901F9010081FB012081D12C22238E
:10ABB00019F00E949D7FD82E1130C9F5102F153441
:10ABC00091F11F3791F11F5F4D2D602F812F0E9452
:10ABD000AA258823A1F3F7011083F70180818F371D
:10ABE000D1F580E897E09F938F931F928CE08F932D
:10ABF000BF92CF920E94C37F0F900F900F900F9043
:10AC00000F900F9081E029960FB6F894DEBF0FBE2B
:10AC1000CDBFDF91CF911F910F91FF90EF90DF900B
:10AC2000CF90BF9008951FE7CFCF10E0CDCF123067
:10AC3000A1F6102F112359F01F3759F011504D2D47
:10AC4000602F812F0E94AA258823A1F3C4CF1FE77C
:10AC5000F6CF15E4F4CF8E010F5F1F4FB8010E94AD
:10AC6000F1361F930F93F70180811F928F9386E730
:10AC700097E09F938F931F928CE08F93BF92CF9218
:10AC80000E94C37F0FB6F894DEBF0FBECDBFBACF10
:10AC90002F923F924F925F926F927F928F929F92EC
:10ACA000AF92BF92CF92DF92EF92FF920F931F93DA
:10ACB000CF93DF9300D0CDB7DEB74C017B01498342
:10ACC000290190E0F401E90FF11D20812F7E20324F
:10ACD00011F49F5FF7CFCF010E949D7F6C011A8214
:10ACE0003A8033948A818E0D9F2D911DDC018C91C9
:10ACF0003A828D32A9F7E32DF0E0FB83EA835F010E
:10AD000021E0A21AB108AE0CBF1CD5011C9290E044
:10AD1000F701E90FF11D20812F7E203211F49F5F92
:10AD2000F7CFCF010E949D7F8C018DE2F5018083DA
:10AD3000832D90E03701680E791ED3012C902220DC
:10AD400009F468C0BCE72B16D9F13394F1CFF9812F
:10AD5000F23039F40C151D0534F486010A191B096B
:10AD600049C0860147C08C0145C0D2010D931C9398
:10AD7000E150F0E03196E80DF91D2AE030E0C8011D
:10AD8000B9010E944183805D82938B018E169F06DC
:10AD9000B1F781E00F900F900F90DF91CF911F914D
:10ADA0000F91FF90EF90DF90CF90BF90AF909F906A
:10ADB0008F907F906F905F904F903F902F9008956D
:10ADC000F301108201968E0D9F1D0E949D7F5C01F4
:10ADD0008A819B818E0D9F1D0E949D7FD3012C92A5
:10ADE000E981E13009F0B3CFC816D9061CF485011A
:10ADF0000C0D1D1DE1E02AE030E0AC01475F5F4F24
:10AE00004331510508F4B1CFB9010E944183CB0110
:10AE1000EF5FF3CF8A819B818E0D9F1D0E949D7FE6
:10AE2000AA24A394B12CDCCFEF92FF920F931F932F
:10AE3000CF93DF931F921F92CDB7DEB7FC017B014A
:10AE40008901D9018D919C9160E570E00E942D836C
:10AE50007A8369839E012F5F3F4FB701CF010E9424
:10AE6000485629813A8140E5429FC001439F900D99
:10AE70001124F8019183808381E00F900F90DF917E
:10AE8000CF911F910F91FF90EF9008950F931F9313
:10AE9000CF93DF931F921F92CDB7DEB789019E013A
:10AEA0002F5F3F4F0E9448568981F801808381E0DF
:10AEB0000F900F90DF91CF911F910F9108952F92D6
:10AEC0003F924F925F926F927F928F929F92AF923A
:10AED000BF92CF92DF92EF92FF920F931F93CF9387
:10AEE000DF93CDB7DEB76E970FB6F894DEBF0FBE17
:10AEF000CDBF8C01DC011696ED91FC910488F5899B
:10AF0000E02D8EE1DE01119601900D928A95E1F718
:10AF1000DE01119690E080E0F80126813781F90189
:10AF2000E80FF91F0190F081E02D2D91208302960A
:10AF30008031910589F75E01FBE0AF0EB11C6DEE2B
:10AF4000862E65E0962E22242394312C2C0E3D1E55
:10AF50008CE1280E311CC12CD12C7601D5016D91CC
:10AF60007D915D016115710511F461E070E090E083
:10AF700080E00E9416850E9415869B01AC01F401B9
:10AF8000459055906590749063EB7CE280E191E48C
:10AF90000E94C78320E030E040E853E40E9491869D
:10AFA0000E94E0849B01AC01C301B2010E941183A5
:10AFB000C60ED71EE81EF91EB4E08B0E911C2A1493
:10AFC0003B0461F6E8E0EE0EF11C84E1F694E794B0
:10AFD000D794C7948A95D1F784E18C9D90018D9D7B
:10AFE000300D112420583F4F232F332746E0220FE6
:10AFF000331F4A95E1F72E5F3F4FA4E3B3E30E946E
:10B000009E83BC0188279927D8011696ED91FC9163
:10B0100017970088F189E02D70831696ED91FC91C9
:10B020000288F389E02D772724E6269FC001279F19
:10B03000900D112480589F4F90836E960FB6F89410
:10B04000DEBF0FBECDBFDF91CF911F910F91FF905B
:10B05000EF90DF90CF90BF90AF909F908F907F90B8
:10B060006F905F904F903F902F9008954F925F9216
:10B070006F927F928F929F92AF92BF92CF92DF9208
:10B08000EF92FF920F931F93CF93DF93CDB7DEB76D
:10B09000C954D1090FB6F894DEBF0FBECDBF4C0125
:10B0A000D62E8A017E0184E3E80EF11C8FE0D701E1
:10B0B0001D928A95E9F76CAB58AF4FABB9E7B6175D
:10B0C00008F495C0E62FF0E08827E659F74A8F4F3D
:10B0D0000C949683E458FC5894675D69616AF26A3F
:10B0E000916BBC680A6A786A096BA86BDD67F467C4
:10B0F000A968F758196C746C7469696C306CB86C19
:10B10000D26CE96C746CAE69156A9769836AC5691B
:10B11000146BF369B36BDC69FF671C5984591267C0
:10B120002967B46D9D6D866DEA6DCD6D076E1E6EDF
:10B13000756EF7588C6EC86E37704E70B270C970ED
:10B14000FB70F758325D4E5D7B5CBE5C355C4B5CE2
:10B15000D85BEE5BA459BA59345A4A5AA45ABD5A1C
:10B16000A95BB45B345BCD5B116F286F6859566F78
:10B170006D6FA56F645DD65D055E1B5E325E0B5F15
:10B18000A05F7460D8603A619161EC614A6290623C
:10B190007D5DE562EF5DFC62F26371638B6927643C
:10B1A00072668966226D396DF758F8640F656E64B2
:10B1B00085641B6536656A659E654864EE6505664F
:10B1C0005A666666EF66066785E08CAF85E090E0BC
:10B1D0000E942887FC019EAF8DAF81E0808385E6C9
:10B1E000818384E7828383E2838388E784838FE09B
:10B1F000FE01F4960C944B6C86E08CAF86E090E0F8
:10B200000E942887FC019EAF8DAF85E1808382E09C
:10B21000818380E1828382E1838388E6848384E67C
:10B22000858380EB94E19F938F930E94434C9EAB68
:10B230008DAB0F900F90DBCF8091B706982F98774A
:10B2400009F443C09091B60692959F7087708295DD
:10B25000807F892B8F37C9F111E087E08CAF90E0B8
:10B260000E9428879EAF8DAF30E020E0112329F0A7
:10B2700024E3FC01208321E030E0FC01E20FF31F16
:10B2800084E280838CE481838DE48283EDADFEAD26
:10B29000E20FF31F82E38383EDADFEADE20FF31FF8
:10B2A0008AE484838DAD9EAD280F391F85E2D901D4
:10B2B00015968C9387EA94E19F938F930E94434C59
:10B2C0009EAB8DAB0F900F9092CF10E086E0C6CF73
:10B2D00084E08CAF84E090E00E942887FC019EAF60
:10B2E0008DAF87E280838CE281838EE2828380E46B
:10B2F000838382E994E19F938F930E94434C9EAB9A
:10B300008DAB0F900F9073CF86E08CAF86E090E00E
:10B310000E942887FC019EAF8DAF88E380838CE379
:10B32000818382E4828384E4838387E484838EE35D
:10B33000858385E894E19F938F930E94434C9EAB55
:10B340008DAB0F900F9053CF81E08CAF81E090E0F8
:10B350000E9428879EAF8DAF21E4FC0120838CE6FC
:10B3600094E19F938F930E94434C9EAB8DAB0F90C3
:10B370000F903DCF83E089AF86E090E00E94288760
:10B380008C019BAF8AAF81E090E00E9428876C011E
:10B39000D8018D939C9381E090E00E9428877C01E6
:10B3A000F8019383828381E090E00E942887D8018E
:10B3B00015969C938E9314972091AA06322F32955E
:10B3C000369537702091AB062370220F220F220F83
:10B3D000232B220F220F220F259525952595022F2D
:10B3E000001F0027001F022E000C330B37FF03C085
:10B3F0003195219531095901B594A794B594A79435
:10B40000237039E1732E279D102D1124F60100833E
:10B41000D701AC92FC0110830E94882B9C013595CA
:10B420002795359527958370879D802D11249DE262
:10B43000011101C09BE21F921F93BF92AF921F9216
:10B440009F931F928F9333273F932F9385E294E12D
:10B450009F938F930E94434C9EAB8DAB0FB6F89495
:10B46000DEBF0FBECDBFC3CE81E08CAF81E090E0E8
:10B470000E9428879EAF8DAF23E4DC012C9386E1E8
:10B4800094E19F938F930E94434C9EAB8DAB0F90A2
:10B490000F90ADCE9091AC0609EA13E091FD02C089
:10B4A00001EB13E08091AB0686958695917092959D
:10B4B000990F990F907CBE016F5F7F4F892B0E947F
:10B4C000A13B1F930F931F9225E02F939F938F9380
:10B4D00083EF93E19F938F930E94434C9EAB8DAB80
:10B4E00082E089AF84E090E00E9428877C019BAFD6
:10B4F0008AAF81E090E00E9428878C01F701918358
:10B50000808381E090E00E942887FC01D701139698
:10B510009C938E9312979091AB06392F3695369562
:10B520002091AC06922F91709295990F990F907C73
:10B53000932BD8019C932695217020830FB6F89405
:10B54000DEBF0FBECDBF53CE82E08CAF82E090E075
:10B550000E9428879EAF8DAF25E4DC012C9326E462
:10B5600011962C9389ED93E19F938F930E94434C06
:10B570009EAB8DAB0F900F903ACE83E089AF86E003
:10B5800090E00E9428878C019BAF8AAF81E090E019
:10B590000E9428876C01F8019183808381E090E00C
:10B5A0000E9428877C01D80113969C938E93129752
:10B5B00081E090E00E942887FC01D80115969C93B9
:10B5C0008E9314978091AC0682FF45C081E09091E4
:10B5D000AD06911101C080E0D6018C938091AE063A
:10B5E000D7018C938091AF068083BE016F5F7F4F40
:10B5F00080810E94A13B182F092FEAADFBAD02808C
:10B60000F381E02DBE016B5D7F4F80810E94A13BE5
:10B61000EAADFBAD0190F081E02D2081222309F1FC
:10B6200029EA33E01F9245E04F930F931F931F9237
:10B630004F939F938F933F932F938FEA93E19F9321
:10B640008F930E94434C9EAB8DAB0FB6F894DEBF38
:10B650000FBECDBFCCCDD6011C9280E2D7018C931A
:10B66000C3CF21EB33E0DECF83E089AF86E090E00B
:10B670000E9428878C019BAF8AAF81E090E00E94F6
:10B6800028876C01D8018D939C9381E090E00E9403
:10B6900028877C01F8019383828381E090E00E94F7
:10B6A0002887FC01D80115969C938E93149780915E
:10B6B000AC0683FF45C081E09091B006911101C0B6
:10B6C00080E0D6018C938091B106D7018C93809154
:10B6D000B2068083BE016F5F7F4F80810E94A13BD5
:10B6E000182F092FEAADFBAD0280F381E02DBE01DA
:10B6F0006B5D7F4F80810E94A13BEAADFBAD019065
:10B70000F081E02D2081222309F129EA33E01F9204
:10B7100045E04F930F931F931F924F939F938F93E7
:10B720003F932F9385E893E19F938F930E94434C1F
:10B730009EAB8DAB0FB6F894DEBF0FBECDBF57CD1D
:10B74000D6011C9280E2D7018C93C3CF21EB33E06A
:10B75000DECF8BE693E19F938F930E94434C9EAB89
:10B760008DAB0F900F9043CD82E08CAF82E090E0E4
:10B770000E9428879EAF8DAF28E4DC012C9329E43A
:10B7800011962C938FE493E19F938F930E94434CE7
:10B790009EAB8DAB0F900F902ACD8FE293E19F93DC
:10B7A0008F930E94434C9EAB8DAB0F900F901FCD9B
:10B7B00081E08CAF81E090E00E9428879EAF8DAF42
:10B7C0002FE3FC0120838DE093E19F938F930E94F0
:10B7D000434C9EAB8DAB0F900F9009CD82E089AFAB
:10B7E00084E090E00E9428878C019BAF8AAF81E0C3
:10B7F00090E00E9428877C01D8018D939C9381E082
:10B8000090E00E942887FC01D80113969C938E93A8
:10B8100012979091AC0692959170D7019C932091CC
:10B82000AA062695217020832223C9F029EA33E055
:10B830009923C1F08EEC93E03F932F939F938F93C6
:10B8400085EE92E19F938F930E94434C9EAB8DAB0C
:10B850000F900F900F900F900F900F90C8CC21EB8E
:10B8600033E0E6CF82ED93E0E7CF81E08CAF81E07B
:10B8700090E00E9428879EAF8DAF2DE3FC012083CE
:10B880008FEC92E19F938F930E94434C9EAB8DABC4
:10B890000F900F90ACCC81E089AF82E090E00E94E5
:10B8A00028878C019BAF8AAF82E090E00E942887B6
:10B8B000D8018D939C932091AA06269526952770F2
:10B8C00030E02F5F3F4F6DE7629FA001639F500DF7
:10B8D0001124FC01518340835F934F9388EA92E1E6
:10B8E0009F938F930E94434C9EAB8DAB0F900F9014
:10B8F0000F900F907CCCCE0101960E94A72381115E
:10B9000032C0BE016B5D7F4F8CE20E94A13B9F93D2
:10B910008F9389E992E19F938F930E94434C9EAB52
:10B920008DAB11E01CAF81E090E00E9428879EAFB4
:10B930008DAF2BE3DC012C9319AF82E090E00E94E5
:10B9400028878C019BAF8AAF81E090E00E94288716
:10B95000F801918380832CE2DC012C930F900F90EF
:10B960000F900F9044CC86E892E19F938F930E94B2
:10B97000434C9EAB8DAB0F900F9039CCDA011696ED
:10B98000ED91FC910190F081E02DE081E2501FEFFC
:10B99000ED3220F4F0E0E151FD4F108182E089AFFB
:10B9A00084E090E00E9428876C019BAF8AAF8EE113
:10B9B00090E00E9428877C01F6019183808381E0DA
:10B9C00090E00E942887D60113969C938E9312973D
:10B9D00017FD43C0E12F110FFF0BED5AF94F808186
:10B9E000182F117086958695B7018F710E94D2230A
:10B9F000882331F0EAADFBAD808191810E94A723BD
:10BA0000EAADFBADA281B38181E081278C930190E7
:10BA1000F081E02D88E09E012F5F3F4FD90101901A
:10BA20000D928A95E1F7198681EB93E0111102C01E
:10BA300089EA93E09F938F933F932F9381E692E15E
:10BA40009F938F930E94434C9EAB8DAB0F900F90B2
:10BA50000F900F900F900F90CACBC7010E94A723A1
:10BA600010E0CECF84E08CAF84E090E00E94288785
:10BA7000FC019EAF8DAF80E5808381E5818382E507
:10BA8000828389E3838382E592E19F938F930E946F
:10BA9000434C9EAB8DAB0F900F90A9CB81E08CAF48
:10BAA00081E090E00E9428879EAF8DAF2AE3FC01E1
:10BAB000208383E392E19F938F930E94434C9EAB3C
:10BAC0008DAB0F900F9093CB82E08CAF82E090E033
:10BAD0000E9428879EAF8DAF2DE5DC012C932EE5CB
:10BAE00011962C9389E292E19F938F930E94434C8D
:10BAF0009EAB8DAB0F900F907ACB81E08CAF81E045
:10BB000090E00E9428879EAF8DAF25E5FC01208341
:10BB100083E189AF86E290E00E9428879BAF8AAFDD
:10BB200010E000E06801CC0CDD1CEAACFBACEC0CD6
:10BB3000FD1C81E090E00E942887D7018D939C93A3
:10BB400081E4011180E2EAADFBADEC0DFD1D019039
:10BB5000F081E02D80830F5F1F4F0830110511F732
:10BB600000E110E0EAACFBACE00EF11E82E090E0F8
:10BB70000E942887F70191838083EAADFBADE00F37
:10BB8000F11F0190F081E02D118210820E5F1F4F96
:10BB90000632110539F785E192E19F938F930E9458
:10BBA000434C9EAB8DAB0F900F9021CB82E08CAFBE
:10BBB00082E090E00E9428879EAF8DAF2FE5DC01E8
:10BBC0002C9320E611962C938AE092E19F938F9319
:10BBD0000E94434C9EAB8DAB0F900F9008CB81E041
:10BBE0008CAF81E090E00E9428879EAF8DAF23E567
:10BBF000FC01208386EF91E19F938F930E94434C39
:10BC00009EAB8DAB0F900F90F2CA81E08CAF81E0BC
:10BC100090E00E9428879EAF8DAF24E5DC012C9335
:10BC200089EE91E19F938F930E94434C9EAB8DAB25
:10BC30000F900F90DCCACE0101960E94A7238111BC
:10BC400011C081E08CAF81E090E00E9428879EAF18
:10BC50008DAF25E5FC01208384ED94E221969FAF12
:10BC60008EAF219784E189AF88E290E00E94288717
:10BC70008C019BAF8AAF81E090E00E942887D801B9
:10BC80008D939C9381E090E00E942887F801938334
:10BC9000828381E090E00E942887D80115969C93CA
:10BCA0008E93149781E090E00E942887F801978393
:10BCB000868381E090E00E942887D80119969C93A2
:10BCC0008E93189781E090E00E942887F80193876F
:10BCD000828781E090E00E942887D8011D969C937E
:10BCE0008E931C9781E090E00E942887F801978747
:10BCF000868782E090E00E942887D80151969C9325
:10BD00008E93509782E090E00E942887F801938BF1
:10BD1000828B82E090E00E942887D80155969C9300
:10BD20008E93549782E090E00E942887F801978BC9
:10BD3000868B82E090E00E942887D80159969C93D8
:10BD40008E93589782E090E00E942887F801938FA5
:10BD5000828F82E090E00E942887D8015D969C93B4
:10BD60008E935C9782E090E00E942887F801978F7D
:10BD7000868F82E090E00E942887D80191969C935C
:10BD80008E93909782E090E00E942887F80193A319
:10BD900082A382E090E00E942887D80195969C9328
:10BDA0008E9394978EE190E00E942887F80197A3E4
:10BDB00086A30E94A723882359F086ED91E19F93E3
:10BDC0008F930E94434C9EAB8DAB0F900F900FCA88
:10BDD000EAADFBAD06A0F7A1E02D28E0CE0101966B
:10BDE000DC0101900D922A95E1F719869F938F93BC
:10BDF0008AEC91E19F938F930E94434C9EAB8DAB55
:10BE00000F900F900F900F90F3E5DF12F0C9C7016C
:10BE10000E94D424ECC981E08CAF81E090E00E94C4
:10BE200028879EAF8DAF26E5DC012C9388E089AF93
:10BE300080E190E00E942887FC019BAF8AAFD80187
:10BE40001696AD90BC90D501CD90DC901197D18223
:10BE5000C08212968D919C9113979383828314963E
:10BE60002D913C9115973583248316964D915C91C5
:10BE700017975783468318966D917C911997718710
:10BE800060871A960D911C911B97138702871C9649
:10BE9000ED90FC901D97F586E4861E96AD90BC90C3
:10BEA000B786A686D501EC91AE2F0E2E000CBB0BEB
:10BEB000BF93EF93D701EC91AE2F0E2E000CBB0B6E
:10BEC000BF93EF93D801EC91AE2F0E2E000CBB0B5D
:10BED000BF93EF93FB016081E62F062E000CFF0B52
:10BEE000FF936F93DA014C91642F042E000C770BB3
:10BEF0007F934F93F9012081422F022E000C550BA6
:10BF00005F932F93DC018C91282F082E000C330BAC
:10BF10003F938F93F6018081282F082E000C330B5E
:10BF20003F938F938FE491E19F938F930E94434CB3
:10BF30009EAB8DAB0FB6F894DEBF0FBECDBF57C919
:10BF4000DA0113960D911C91F80146815781FA018F
:10BF500070964A5D5F4FE190F190D7012D913C9131
:10BF6000AAEFB0E00E949E83672F782F892F992730
:10BF7000D7016D937C934E175F0769F781E08CAF13
:10BF800081E090E00E9428879EAF8DAF27E5FC01FD
:10BF900020838BE089AF86E190E00E942887FC0136
:10BFA0009BAF8AAFD80116968D919C91DC0150967B
:10BFB000ED90FC90F182E082D80116968D919C91D3
:10BFC000DC015296CD90DC90D382C282D8011696C5
:10BFD0008D919C91DC015496AD90BC90B582A48269
:10BFE000D80116968D919C91DC0156962D913C912D
:10BFF00037832683D80116968D919C91DC01589643
:10C000008D919C9191878087D80116968D919C91F6
:10C01000DC015A968D919C9193878287D801169660
:10C020008D919C91DC015C968D919C919587848784
:10C03000D80116968D919C91DC015E968D919C9114
:10C0400097878687D80116968D919C91DC019096F2
:10C050008D919C91918B808BD80116968D919C919E
:10C06000DC0192968D919C91938B828BD8011696D0
:10C070008D919C91DC0194968D919C91958B848BF4
:10C08000F90180819181889620E530E0B9010E9414
:10C090002D837F936F93D5018D919C918896B901E3
:10C0A0000E942D837F936F93F60180819181889602
:10C0B000B9010E942D837F936F93D7018D919C913D
:10C0C0008896B9010E942D837F936F9389EF90E149
:10C0D0009F938F930E94434C9EAB8DAB0FB6F89409
:10C0E000DEBF0FBECDBF83C881E08CAF81E090E0A2
:10C0F0000E9428879EAF8DAF28E5DC012C9384E059
:10C1000089AF88E090E00E942887FC019BAF8AAF4E
:10C11000D80116968D919C91DC0118960D911C9179
:10C120001997118300831A96ED90FC901B97F38268
:10C13000E2821C96CD90DC901D97D582C4821E961B
:10C140008D919C9197838683FC0180819181889653
:10C1500020E530E0B9010E942D837F936F93D601D3
:10C160008D919C918896B9010E942D837F936F9346
:10C17000F701808191818896B9010E942D837F9378
:10C180006F93D8018D919C918896B9010E942D835F
:10C190007F936F9383EA90E19F938F930E94434C28
:10C1A0009EAB8DAB0FB6F894DEBF0FBECDBF1FC8E0
:10C1B00081E08CAF81E090E00E9428879EAF8DAF38
:10C1C00029E5DC012C9383E089AF86E090E00E94B2
:10C1D0002887FC019BAF8AAFD80113962D913C9123
:10C1E000D90116968D919C91DC0150960D911C9170
:10C1F00011830083D90116968D919C91DC01529692
:10C20000ED90FC90F382E282D90116968D919C917B
:10C21000DC0154968D919C9195838483FC018081EF
:10C220009181889620E530E0B9010E942D837F93AB
:10C230006F93D7018D919C918896B9010E942D83AF
:10C240007F936F93F801808191818896B9010E9454
:10C250002D837F936F9381E690E19F938F930E944C
:10C26000434C9EAB8DAB0FB6F894DEBF0FBECDBF77
:10C270000C94F758DA011396ED91FC910381148127
:10C2800081E08CAF81E090E00E9428879EAF8DAF67
:10C290002AE5FC01208383E089AF86E090E00E94DC
:10C2A0002887FC019BAF8AAFD80116968D919C918F
:10C2B000DC016D917C9171836083D80116968D911C
:10C2C0009C91DC0112968D919C9193838283D8017D
:10C2D00016962D913C91D90114962D913C91358360
:10C2E0002483F90141814F9320812F93DC01119622
:10C2F0002C9111972F938C918F93FB0181818F93B8
:10C3000080818F938CE190E19F938F930E94434CA7
:10C310009EAB8DAB0FB6F894DEBF0FBECDBF0C94B5
:10C32000F758DA011396ED91FC910380F481E02D2A
:10C330000381148181E08CAF81E090E00E94288726
:10C340009EAF8DAF2BE5FC01208383E089AF86E0B3
:10C3500090E00E942887FC019BAF8AAFD801169617
:10C360008D919C91DC0116966D917C917183608317
:10C37000D80116968D919C91DC0118968D919C9117
:10C3800093838283D80116962D913C91D9011A96F8
:10C390002D913C9135832483F90141814F93208174
:10C3A0002F93DC0111962C9111972F938C918F93E1
:10C3B000FB0181818F9380818F9387ED9FE09F9315
:10C3C0008F930E94434C9EAB8DAB0FB6F894DEBFAB
:10C3D0000FBECDBF0C94F758DA011396ED91FC9186
:10C3E0000380F481E02D0380F481E02D038114812A
:10C3F00081E08CAF81E090E00E9428879EAF8DAFF6
:10C400002CE5FC01208383E089AF86E090E00E9468
:10C410002887FC019BAF8AAFD80116968D919C911D
:10C42000DC011C966D917C9171836083D801169616
:10C430008D919C91DC011E968D919C9193838283BA
:10C44000D80116962D913C91D90150962D913C9191
:10C4500035832483F90141814F9320812F93DC019F
:10C4600011962C9111972F938C918F93FB018181C1
:10C470008F9380818F9382E99FE09F938F930E9497
:10C48000434C9EAB8DAB0FB6F894DEBF0FBECDBF55
:10C490000C94F758DA011396ED91FC910380F48126
:10C4A000E02D0380F481E02D0380F481E02D0381F1
:10C4B000148182E089AF84E090E00E9428879BAFDE
:10C4C0008AAFD8011696ED91FC911797228933898E
:10C4D000FC01318320831696ED91FC91A489B589E6
:10C4E000FC01B383A28311968C9111978F938C9149
:10C4F0008F93D90111968C9111978F938C918F9373
:10C5000083E69FE09F938F930E94434C9EAB8DAB3D
:10C510000F900F900F900F900F900F900C94F75872
:10C5200081E08CAF81E090E00E9428879EAF8DAFC4
:10C5300023E6FC0120838FE49FE09F938F930E946A
:10C54000434C9EAB8DAB8AE089AF84E190E00E94C2
:10C5500028879BAF8AAF0F900F9010E000E0680132
:10C56000CC0CDD1CEAACFBACEC0CFD1C81E090E0DB
:10C570000E942887D7018D939C9381E4011180E26A
:10C58000EAADFBADEC0DFD1D0190F081E02D808347
:10C590000F5F1F4F0830110511F70AAD1BAD81E089
:10C5A00090E00E942887F801918B808B22E0DC01CB
:10C5B0002C9381E090E00E942887F801938B828B76
:10C5C00024E1DC012C930C94F75881E08CAF81E0DE
:10C5D00090E00E9428879EAF8DAF21E6FC0120836A
:10C5E0008BE39FE09F938F930E94434C9EAB8DAB58
:10C5F0000F900F900C94F7588BE089AF86E190E094
:10C600000E9428879BAF8AAF10E000E0CAACDBAC89
:10C61000C00ED11E81E090E00E942887D6018D9344
:10C620009C930E5F1F4F0031110581F70AAD1BADC2
:10C6300081E090E00E942887F801918B808B81E057
:10C6400090E00E942887D80153969C938E9352972E
:10C650008EE190E00E942887F801958B848B0E94E0
:10C66000A723882361F088E29FE09F938F930E9425
:10C67000434C9EAB8DAB0F900F900C94F75881E01C
:10C680008CAF81E090E00E9428879EAF8DAF23E6BB
:10C69000DC012C938FE597E521969FAF8EAF219714
:10C6A000EAADFBAD0488F589E02D28E0CE010196C6
:10C6B000DC0101900D922A95E1F719869F938F93E3
:10C6C0008CE19FE09F938F930E94434C9EAB8DAB78
:10C6D000C7010E945F570F900F900F900F900C941E
:10C6E000F75881E08CAF81E090E00E9428879EAFF0
:10C6F0008DAF22E6FC01208388E089AF80E190E0E5
:10C700000E9428879BAF8AAF90E080E0D801169600
:10C71000ED91FC91E80FF91F20813181EAADFBAD6D
:10C72000E80FF91F3183208302968031910571F75C
:10C73000EAADFBADA685B7858C91282F082E000C9D
:10C74000330B3F938F93A485B5858C91282F082EAA
:10C75000000C330B3F938F93A285B3858C91282FC8
:10C76000082E000C330B3F938F93A085B1858C91DD
:10C77000282F082E000C330B3F938F93A681B7818F
:10C780008C91282F082E000C330B3F938F93A4819C
:10C79000B5818C91282F082E000C330B3F938F937B
:10C7A000A281B3818C91282F082E000C330B3F936C
:10C7B0008F930190F081E02D8081282F082E000CAE
:10C7C000330B3F938F9381EA9EE09F938F930E9458
:10C7D000434C9EAB8DAB0FB6F894DEBF0FBECDBF02
:10C7E0000C94F758DA0113960D911C9182E089AFF1
:10C7F00084E090E00E9428879BAF8AAFD80116960C
:10C80000ED91FC91179720893189FC0131832083B8
:10C810001696ED91FC91A289B389FC01B383A283A2
:10C820008C911F928F93D9018C911F928F9389E7DE
:10C830009EE09F938F930E94434C9EAB8DAB0F90D5
:10C840000F900F900F900F900F900C94F75886E078
:10C850008CAF86E090E00E942887FC019EAF8DAFF0
:10C860008FE6808388E6818383E7828386E68383FD
:10C870008BE684838DE685838CE69EE09F938F9381
:10C880000E94434C9EAB8DAB0F900F900C94F758C9
:10C890008FEF97E00E943F0E9B01AC0160E47FE1C7
:10C8A00080E090E00E947783215030E02F5F3F4F7F
:10C8B0004DE7429FC001439F900D11249F938F939A
:10C8C00088E59EE09F938F930E94434C9EAB8DAB77
:10C8D0000F900F900F900F900C94F75881E08CAF51
:10C8E00081E090E00E9428879EAF8DAF2EE6FC018C
:10C8F00020838BE49EE09F938F930E94434C9EABDA
:10C900008DAB0F900F900C94F7580E9415132DA328
:10C910003EA34FA358A769A77AA78BA7822F8F7032
:10C920008A3008F062C0822F82958F70232F217089
:10C930002295207F282B283108F057C036953F7369
:10C940003C3308F052C087E0FE01B596DE01119637
:10C9500001900D928A95E1F710E000E00F5F1F4F04
:10C9600029813A814B815C816D817E818F810E941A
:10C970006F1679012983FA824B835C836D837E83F2
:10C980008F83BE016F5F7F4FCE0185960E94C511D8
:10C99000811113C08E2D8F708A3078F4E2947FE07D
:10C9A000E7222F2D21702295207F2E29283128F46F
:10C9B0008F2D86958F738C3388F280E092E0801BF8
:10C9C000910B9F938F931F930F9383E39EE09F930D
:10C9D0008F930E94434C9EAB8DAB0F900F900F90A6
:10C9E0000F900F900F900C94F75810E000E0E5CFF7
:10C9F00081E08CAF81E090E00E9428879EAF8DAFF0
:10CA00002CE6DC012C938BE29EE09F938F930E9497
:10CA1000434C9EAB8DAB0F900F900C94F75880E178
:10CA20009EE09F938F930E94434C9EAB8DAB0F90E3
:10CA30000F900C94F75883E08CAF83E090E00E9455
:10CA40002887FC019EAF8DAF80E7808381E78183DB
:10CA500082E782838CEF9DE09F938F930E94434CEB
:10CA60009EAB8DAB0F900F900C94F7581091BE08B1
:10CA7000E12E012E000CFF0889E898E00E94792D34
:10CA8000811125C081EE93E0FF921F939F938F93B6
:10CA90008091BB08282F082E000C330B3F938F93F7
:10CAA0008091BA08282F082E000C330B3F938F93E8
:10CAB00088ED9DE09F938F930E94434C9EAB8DAB7E
:10CAC0000FB6F894DEBF0FBECDBF0C94F75885EDBE
:10CAD00093E0DACF10918708E12E012E000CFF08B9
:10CAE00082E598E00E94792D811125C081EE93E0C6
:10CAF000FF921F939F938F9380918408282F082E75
:10CB0000000C330B3F938F9380918308282F082EBE
:10CB1000000C330B3F938F9384EB9DE09F938F9397
:10CB20000E94434C9EAB8DAB0FB6F894DEBF0FBE98
:10CB3000CDBF0C94F75885ED93E0DACF20914C08E7
:10CB4000121604F5122F00914D088BE198E00E9417
:10CB5000792D81113EC081EE93E09F938F931F92B8
:10CB60000F931F921F938DE99DE09F938F930E94D7
:10CB7000434C9EAB8DAB0FB6F894DEBF0FBECDBF5E
:10CB80000C94F7580E94882B2091AA06322F3295D8
:10CB9000369537702091AB062370220F220F220F9B
:10CBA000232B220F220F220F259525952595820FE5
:10CBB000911D27FD9A959C013595279535952795CB
:10CBC000122F837009E1809F002D11248AED93E0DC
:10CBD000C4CF8130D9F785ED93E0BFCF81E08CAF32
:10CBE00081E090E00E9428879EAF8DAF25E7FC0191
:10CBF000208384E99DE09F938F930E94434C9EABDA
:10CC00008DAB0F900F900C94F758BE016D5B7F4F6A
:10CC1000CE0185960E94681D882309F43FC08E01CD
:10CC20000F5F1F4FB801CE0185960E94223982E026
:10CC30008CAF82E090E00E9428879EAF8DAF26E700
:10CC4000DC012C9327E711962C931F930F938BE80D
:10CC50009DE09F938F930E94434C9EAB8DAB81E0F0
:10CC600089AF82E090E00E9428878C019BAF8AAF59
:10CC700085E090E00E942887DC01F80191838083A1
:10CC800095E0FE01ED5BFF4F01900D929A95E1F763
:10CC90000F900F900F900F900C94F75885E79DE040
:10CCA0009F938F930E94434C9EAB8DAB0F900F9040
:10CCB0000C94F75886E69DE09F938F930E94434C17
:10CCC0009EAB8DAB0F900F900C94F75882E59DE0D2
:10CCD0009F938F930E94434C9EAB8DAB0F900F9010
:10CCE0000C94F75881E08CAF81E090E00E94288797
:10CCF0009EAF8DAF27E6DC012C938BE49DE09F93E4
:10CD00008F930E94434C9EAB8DAB0F900F900C9471
:10CD1000F7586091B8067091B9068091BA06909163
:10CD2000BB06AE014F5F5F4F0E940D1C0E942E207C
:10CD30000091B8061091B9062091BA063091BB0651
:10CD40006B017C01C01AD10AE20AF30A5CE3452EAA
:10CD5000512C612C712CC701B601A30192010E94D4
:10CD60005583CA01B901A30192010E9455837F93A3
:10CD70006F93C701B60120E13EE040E050E00E9421
:10CD80005583CA01B90128E130E040E050E00E943B
:10CD900055837F936F93C701B60120E831E541E0E9
:10CDA00050E00E9455833F932F938D811F928F9364
:10CDB0008E811F928F938F818E51990B9F938F93AA
:10CDC00081E29DE09F938F930E94434C9EAB8DAB7D
:10CDD0000FB6F894DEBF0FBECDBF0C94F75881E0BC
:10CDE0008CAF81E090E00E9428879EAF8DAF29E74D
:10CDF000DC012C9389E19DE09F938F930E94434C2B
:10CE00009EAB8DAB0F900F900C94F75886E09DE091
:10CE10009F938F930E94434C9EAB8DAB0F900F90CE
:10CE20000C94F75881E08CAF81E090E00E94288755
:10CE30009EAF8DAF26E2FC0120838DEF9CE09F9397
:10CE40008F930E94434C9EAB8DAB0F900F900C9430
:10CE5000F7580E942E20AE014F5F5F4F0E940D1CBD
:10CE60008F818E518436D8F58F831CAE8A811F92B4
:10CE70008F938B811F928F938D811F928F938E81C1
:10CE80001F928F938F811F928F9381EA9CE09F93D3
:10CE90008F930E94434C9EAB8DAB85E089AF8AE0B7
:10CEA00090E00E9428879BAF8AAF0FB6F894DEBF50
:10CEB0000FBECDBFF12C0AAD1BAD89ADF81688F4BD
:10CEC00081E090E00E9428872F2D30E0220F331F51
:10CED000020F131FD8018D939C93F394ECCF83E63C
:10CEE000C3CFD801ED91FC918D818083EAADFBAD7C
:10CEF0000280F381E02D8E818083EAADFBAD04805A
:10CF0000F581E02D8F818083EAADFBAD0680F7814E
:10CF1000E02D8B818083EAADFBAD0084F185E02DAF
:10CF20008A8180830C94F7580E947013182F8823ED
:10CF300061F082E89CE09F938F930E94434C9EABEC
:10CF40008DAB0F900F900C94F7588091B706982FE7
:10CF5000987789F19091B60692959F708770829527
:10CF6000807F892B8F3739F111E085E08CAF90E01D
:10CF70000E942887FC019EAF8DAF83E0808384E010
:10CF8000818382E090E0112321F085E0828383E0B9
:10CF900090E0E80FF91F86E080838CE0818389E7C9
:10CFA0009CE09F938F930E94434C9EAB8DAB0F9060
:10CFB0000F900C94F75884E0D9CF81E08CAF81E0DA
:10CFC00090E00E9428879EAF8DAF2DE0FC0120836A
:10CFD0008AE69CE09F938F930E94434C9EAB8DAB5F
:10CFE0000F900F900C94F75881E08CAF81E090E0A7
:10CFF0000E9428879EAF8DAF27E0DC012C9383E051
:10D0000089AF86E090E00E9428877C019BAF8AAFC1
:10D0100081E090E00E9428875C01F7019183808382
:10D020008EE190E00E9428876C01D70113969C93B3
:10D030008E93129781E090E00E942887F7019583F4
:10D0400084830115110521F0D8018C918331E9F019
:10D050008CE2F50180838091530686958695B60112
:10D060008F710E94D223882331F0EAADFBAD82811B
:10D0700093810E94A723EAADFBAD0480F581E02DEA
:10D08000809153068095817020C01696ED91FC9199
:10D0900000811181F8018481D5018C93B6018581CD
:10D0A0000E94D223882331F0EAADFBAD82819381C7
:10D0B0000E94A723EAADFBAD0480F581E02D81E05D
:10D0C000D80116969C91911180E080838DE598E3BC
:10D0D00023969FAF8EAF23978AAD9BAD8E010B5DDC
:10D0E0001F4FDC011296ED91FC9128E0D8010190D0
:10D0F0000D922A95E1F71DA6DC011496ED91FC91A5
:10D10000208138EAE32E33E0F32E211104C020EB16
:10D11000E22E23E0F22EDC01ED91FC91BE016F5F67
:10D120007F4F80810E94A13BFF92EF921F930F934C
:10D130009F938F9386E49CE09F938F930E94434C30
:10D140009EAB8DAB0FB6F894DEBF0FBECDBF0C9477
:10D15000F758BE016F5F7F4FCA010E944B4583E2C3
:10D1600090E00E9428879EAB8DABBC01CE0101965A
:10D170000E94C13C0C94F75881E08CAF81E090E0B4
:10D180000E9428879EAF8DAF2EE0DC012C9384E0B7
:10D1900089AF88E090E00E9428877C019BAF8AAF2E
:10D1A00081E090E00E9428875C01F70191838083F1
:10D1B00081E090E00E9428876C01D70113969C9330
:10D1C0008E93129781E090E00E9428873C01F7013E
:10D1D0009583848381E090E00E9428879C01D70199
:10D1E00017969C938E9316970115110521F0F8015F
:10D1F00080818431C1F1D5011C92F60110828CE04E
:10D20000D3018C93F90110828E010F5F1F4FB8017B
:10D21000F60180810E945D3CEAADFBADA681B7813D
:10D220002C91A481B5819C910190F081E02D8081A9
:10D23000882309F440C087E31F922F931F929F9386
:10D240001F930F931F928F938CEF9BE09F938F936D
:10D250000E94434C9EAB8DAB0FB6F894DEBF0FBE61
:10D26000CDBF0C94F7580380F481E02DA681B781DF
:10D270000D90BC91A02D13968C91139787FB882756
:10D2800080F9F50180838C918F70F60180839C91E9
:10D29000892F82958F7011969C911197917092951C
:10D2A000907F982BF301908311969C9196959F7394
:10D2B000D9019C93A9CF86E3BFCF81E08CAF81E0F9
:10D2C00090E00E9428879EAF8DAF28E0DC012C9370
:10D2D00082EF9BE09F938F930E94434C9EAB8DAB5C
:10D2E0000F900F900C94F75881E08CAF81E090E0A4
:10D2F0000E9428879EAF8DAF23E1FC01208388EE3A
:10D300009BE09F938F930E94434C9EAB8DAB0F90FD
:10D310000F900C94F7588AED9BE09F938F930E9497
:10D32000434C9EAB8DAB0F900F900C94F75881E05F
:10D330008CAF81E090E00E9428879EAF8DAF2CE1FA
:10D34000DC012C938DEC9BE09F938F930E94434CC8
:10D350009EAB8DAB0F900F900C94F75881E08CAF83
:10D3600081E090E00E9428879EAF8DAF2AE1FC010A
:10D37000208383EC9BE09F938F930E94434C9EAB52
:10D380008DAB0F900F900C94F75881E08CAF81E03B
:10D3900090E00E9428879EAF8DAF2EE1DC012C9398
:10D3A00089EB9BE09F938F930E94434C9EAB8DAB88
:10D3B0000F900F900C94F75881E08CAF81E090E0D3
:10D3C0000E9428879EAF8DAF22E2FC0120838AEA6B
:10D3D0009BE09F938F930E94434C9EAB8DAB0F902D
:10D3E0000F900C94F75881E08CAF81E090E00E94A0
:10D3F00028879EAF8DAF20E2DC012C9387E99BE06C
:10D400009F938F930E94434C9EAB8DAB0F900F90D8
:10D410000C94F75881E08CAF81E090E00E9428875F
:10D420009EAF8DAF27E0FC01208382E089AF84E0CE
:10D4300090E00E9428876C019BAF8AAF81E090E06A
:10D440000E9428877C01D6018D939C9381E090E017
:10D450000E942887FC01D60113969C938E93129705
:10D460000115110521F0D8018C918331D1F0D7013C
:10D470001C92108280811F928F93F70180811F92EE
:10D480008F9383E69BE09F938F930E94434C9EABC8
:10D490008DAB0F900F900F900F900F900F900C94FA
:10D4A000F75816968D919C91DC012D913C91D901F4
:10D4B00014968C91D7018C93D90116968C91808308
:10D4C000D9CF81E08CAF81E090E00E9428879EAFA9
:10D4D0008DAF29E0DC012C9386E59BE09F938F9331
:10D4E0000E94434C9EAB8DAB0F900F900C94F7585D
:10D4F00081E08CAF81E090E00E9428879EAF8DAFE5
:10D5000027E0FC01208383E089AF86E090E00E9461
:10D5100028877C019BAF8AAF81E090E00E9428873A
:10D520005C01D7018D939C9381E090E00E94288755
:10D530006C01F7019383828381E090E00E94288749
:10D54000FC01D70115969C938E9314970115110534
:10D5500021F0D8018C91833169F1D5011C9288E2C8
:10D56000D6018C938083BE016B5D7F4F80810E94CA
:10D57000A13B182F092FEAADFBAD0280F381E02D0E
:10D58000BE016F5F7F4F80810E94A13B0F931F936D
:10D590009F938F9380E39BE09F938F930E94434CD4
:10D5A0009EAB8DAB0F900F900F900F900F900F9040
:10D5B0000C94F75816968D919C91DC012D913C911D
:10D5C00081E0D90114969C91911101C080E0D501B0
:10D5D0008C93D90115968C91D6018C93D90116960E
:10D5E0008C91C0CF81E08CAF81E090E00E942887D1
:10D5F0009EAF8DAF2AE0FC01208386E29BE09F93E3
:10D600008F930E94434C9EAB8DAB0F900F900C9468
:10D61000F75881E08CAF81E090E00E9428879EAFB0
:10D620008DAF27E0DC012C9384E089AF88E090E0A7
:10D630000E9428877C019BAF8AAF81E090E00E9426
:10D6400028873C01F7019183808381E090E00E946C
:10D6500028876C01D70113969C938E93129781E0D3
:10D6600090E00E9428875C01F7019583848381E024
:10D6700090E00E942887FC01D70117969C938E9317
:10D6800016970115110521F0D8018C91833159F1BC
:10D6900081E0D3018C93D6011C92D5011C9280832A
:10D6A000F080F5010081D6011C91BE016F5F7F4FB4
:10D6B000F30180810E94033B1F92FF921F920F9300
:10D6C0001F921F939F938F9382EE9AE09F938F9365
:10D6D0000E94434C9EAB8DAB0FB6F894DEBF0FBEDD
:10D6E000CDBF0C94F75816968D919C91DC012D912D
:10D6F0003C91D90114968C91D3018C93D901159644
:10D700009C91892F86958695D6018C93937089E19B
:10D71000989F902D1124D5019C93D90116968C9138
:10D72000BECF81E08CAF81E090E00E9428879EAF61
:10D730008DAF2BE0DC012C938FEC9AE09F938F93BD
:10D740000E94434C9EAB8DAB0F900F900C94F758FA
:10D7500081E08CAF81E090E00E9428879EAF8DAF82
:10D7600027E0FC01208383E089AF86E090E00E94FF
:10D7700028875C019BAF8AAF81E090E00E942887F8
:10D780007C01D5018D939C9381E090E00E942887D5
:10D790006C01F5019383828381E090E00E942887E9
:10D7A000FC01D50115969C938E93149701151105D4
:10D7B00021F0D8018C91833129F1D7011C9284E1A9
:10D7C000D6018C9389E180833081F6012081D701D5
:10D7D0008C9181112BC08AEB93E01F923F931F9293
:10D7E0002F939F938F9389E89AE09F938F930E9442
:10D7F000434C9EAB8DAB0FB6F894DEBF0FBECDBFD2
:10D800000C94F75816968D919C91DC012D913C91CA
:10D81000D90114968C91D7018C93D90115968C91CE
:10D82000D6018C93D90116968C91CDCF85EB93E0E0
:10D83000D4CF81E08CAF81E090E00E9428879EAF3A
:10D840008DAF21E1DC012C938DE79AE09F938F93BC
:10D850000E94434C9EAB8DAB0F900F900C94F758E9
:10D86000DA011696ED91FC910190F081E02DE381B3
:10D87000EF77E15069E0E43020F4F0E0E551FD4F4E
:10D880006081A801CE0101960E94365884E1898307
:10D890008FE0FE013196D40101900D928A95E1F757
:10D8A000C401C75BDF4F0FB6F894DEBF0FBECDBF1C
:10D8B000DF91CF911F910F91FF90EF90DF90CF906C
:10D8C000BF90AF909F908F907F906F905F904F90A0
:10D8D000089581E08CAF81E090E00E9428879EAFA0
:10D8E0008DAF24E1FC0120830E944113882361F065
:10D8F0008BE69AE09F938F930E94434C9EAB8DAB37
:10D900000F900F900C94F75881E089AF82E090E07F
:10D910000E9428877C019BAF8AAF87E090E00E943D
:10D9200028878C01D7018D939C930E941513F801D1
:10D93000208331834283538364837583868382E4A7
:10D940009AE09F938F930E94434C9EAB8DABBC019A
:10D950006C5F7F4FEAADFBAD808191810E94C13C3D
:10D96000EDA9FEA98CE286A30F900F900C94F758B6
:10D9700082E08CAF82E090E00E9428879EAF8DAF5E
:10D9800026E1DC012C9327E111962C9385E39AE0A4
:10D990009F938F930E94434C9EAB8DAB0F900F9043
:10D9A0000C94F75881E08CAF81E090E00E942887CA
:10D9B0009EAF8DAF28E1FC01208387E29AE09F9320
:10D9C0008F930E94434C9EAB8DAB0F900F900C94A5
:10D9D000F7588091B706982F987789F19091B606FD
:10D9E00092959F7087708295807F892B8F3739F150
:10D9F00011E085E08CAF90E00E942887FC019EAF8B
:10DA00008DAF89E180838BE1818382E090E01123F7
:10DA100021F08DE1828383E090E0E80FF91F8FE130
:10DA2000808381E2818388E19AE09F938F930E94B3
:10DA3000434C9EAB8DAB0F900F900C94F75810E0B9
:10DA400084E0D8CF81E08CAF81E090E00E9428870D
:10DA50009EAF8DAF29E6DC012C9389E09AE09F937D
:10DA60008F930E94434C9EAB8DAB0F900F900C9404
:10DA7000F75887E0E6E0F2E0DE01119601900D92A2
:10DA80008A95E1F787E0FE013196DE0195960190D7
:10DA90000D928A95E1F787E0FE01B596DE01AD5B58
:10DAA000BF4F01900D928A95E1F724962FAD2497F0
:10DAB000822F8F708A3080F422952F7025968FAD3B
:10DAC0002597982F91709295907F922B983120F402
:10DAD00086958F738C3360F087EF99E09F938F93D7
:10DAE0000E94434C9EAB8DAB0F900F900C94F75857
:10DAF00083E290E00E9428879EAB8DABBC01CE01F3
:10DB00008D5B9F4F0E94C13C0C94F75881E08CAF15
:10DB100081E090E00E9428879EAF8DAF2AE2FC0151
:10DB2000208382EF99E09F938F930E94434C9EAB9A
:10DB30008DAB0F900F900C94F75881E08CAF81E083
:10DB400090E00E9428879EAF8DAF2BE2DC012C93E2
:10DB50008DEE99E09F938F930E94434C9EAB8DABCB
:10DB60000F900F900C94F75882E08CAF82E090E019
:10DB70000E9428879EAF8DAF29E2FC01208328E216
:10DB800021838AED99E09F938F930E94434C9EAB33
:10DB90008DAB0F900F900C94F758FF92EF928DB7CA
:10DBA0009EB7C7970FB6F8949EBF0FBE8DBFADB797
:10DBB000BEB7119687E3E2E5F8E001900D928A95F1
:10DBC000E1F70E94754C0FB6F894DEBF0FBECDBFD3
:10DBD0000C94F758FF92EF92EDB7FEB7F7970FB698
:10DBE000F894FEBF0FBEEDBFADB7BEB7119687E389
:10DBF000E9E8F8E001900D928A95E1F70E94754CF2
:10DC00000FB6F894DEBF0FBECDBF0C94F75881E07D
:10DC10008CAF81E090E00E9428879EAF8DAF2DE20F
:10DC2000DC012C9381EC99E09F938F930E94434CED
:10DC30009EAB8DAB0F900F900C94F75882E089AF9C
:10DC400084E090E00E9428878C019BAF8AAF81E03E
:10DC500090E00E9428876C01F8019183808381E025
:10DC600090E00E9428877C01D80113969C938E93A4
:10DC70001297F60110821091B306812F881F882712
:10DC8000881F1091B4061F73110F182B42E06FE725
:10DC9000812F0E94AA25882321F1D7011C938EEEA3
:10DCA0009BE323969FAF8EAF2397BE016F5F7F4F9D
:10DCB000D7018C910E94A13B1F9222E02F939F934A
:10DCC0008F938EE899E09F938F930E94434C9EAB75
:10DCD0008DAB0F900F900F900F900F900F900C94B2
:10DCE000F7588FE7F7018083DACF81E08CAF81E0CE
:10DCF00090E00E9428879EAF8DAF20E3FC01208337
:10DD00008EE799E09F938F930E94434C9EAB8DAB1F
:10DD10000F900F900C94F75811E01CAF81E090E049
:10DD20000E9428879EAF8DAF21E3DC012C93809168
:10DD3000B306BE016F5F7F4F8F770E94A13B1F929A
:10DD400023E02F939F938F9384E699E09F938F9383
:10DD50000E94434C9EAB8DAB19AF82E090E00E94D5
:10DD600028878C019BAF8AAF81E090E00E942887D2
:10DD7000FC01D8018D939C939091B3069F7790837B
:10DD80000F900F900F900F900F900F900C94F758EA
:10DD90008091AC062EED33E087FD02C022EE33E029
:10DDA00086FF3CC089EA93E03F932F939F938F9324
:10DDB00089E399E09F938F930E94434C9EAB8DAB78
:10DDC00082E089AF84E090E00E9428878C019BAFBD
:10DDD0008AAF81E090E00E9428877C01F80191835E
:10DDE000808381E090E00E942887FC01D80113968F
:10DDF0009C938E9312979091AC0696FB882780F99E
:10DE0000D7018C9397FB992790F990830F900F90EF
:10DE10000F900F900F900F900C94F75880EB93E0B9
:10DE2000C3CF81E08CAF81E090E00E9428879EAF55
:10DE30008DAF2BE4FC01208381E299E09F938F93C7
:10DE40000E94434C9EAB8DAB0F900F900C94F758F3
:10DE500081E089AF82E090E00E9428878C019BAF2F
:10DE60008AAF81E090E00E942887FC01D8018D9361
:10DE70009C939091AC0695FB992790F990839923F8
:10DE800091F08EEC93E09F938F938DEF98E09F93AA
:10DE90008F930E94434C9EAB8DAB0F900F900F90D1
:10DEA0000F900C94F75882ED93E0EDCF81E08CAFAA
:10DEB00081E090E00E9428879EAF8DAF2EE4FC01A8
:10DEC00020838DEE98E09F938F930E94434C9EABEE
:10DED0008DAB0F900F900C94F75811E01CAF81E0C0
:10DEE00090E00E9428879EAF8DAF2FE4DC012C9339
:10DEF00019AF82E090E00E9428878C019BAF8AAF27
:10DF000081E090E00E942887F8019183808320E2DD
:10DF1000DC012C93BE016F5F7F4F80E20E94A13B2A
:10DF20001F9226E02F939F938F9382ED98E09F930B
:10DF30008F930E94434C9EAB8DAB0F900F900F9030
:10DF40000F900F900F900C94F758DA011696ED9100
:10DF5000FC910190F081E02DB080BE016F5F7F4F9A
:10DF60008B2D0E94F13688E089AF80E190E00E941D
:10DF700028879BAF8AAFFE0131967F0110E000E059
:10DF8000CAACDBACC00ED11E81E090E00E942887B5
:10DF9000D6018D939C93EAADFBADE00FF11F01908C
:10DFA000F081E02DD7018D917D0180830E5F1F4FA1
:10DFB0000031110529F7EAADFBADA685B7858C9137
:10DFC000282F082E000C330B3F938F93A485B58523
:10DFD0008C91282F082E000C330B3F938F93A28532
:10DFE000B3858C91282F082E000C330B3F938F9311
:10DFF000A085B1858C91282F082E000C330B3F9300
:10E000008F93A681B7818C91282F082E000C330B9B
:10E010003F938F93A481B5818C91282F082E000CFB
:10E02000330B3F938F93A281B3818C91282F082EBD
:10E03000000C330B3F938F930190F081E02D808192
:10E04000282F082E000C330B3F938F931F92BF9203
:10E0500082E398E09F938F930E94434C9EAB8DABDD
:10E060000FB6F894DEBF0FBECDBF0C94F75881E019
:10E070008CAF81E090E00E9428879EAF8DAF23E3B4
:10E08000DC012C9380E298E09F938F930E94434C95
:10E090009EAB8DAB0F900F900C94F75883E089AF37
:10E0A00086E090E00E9428876C019BAF8AAF81E0F8
:10E0B00090E00E9428877C01F6019183808381E0B3
:10E0C00090E00E9428878C01D60113969C938E9332
:10E0D000129781E090E00E942887FC01D6011596F6
:10E0E0009C938E9314978091B606382F32953F708B
:10E0F0002091B706922F97709295907F892F832B4E
:10E10000D7018C93F22EF694F694F694BF2DBF703F
:10E11000FB2ED801FC92221F2227221F208309EA0E
:10E1200013E0211102C001EB13E0BE016F5F7F4FCE
:10E130000E94A13B1F930F931F92FF921F9224E016
:10E140002F939F938F938AEE97E09F938F930E94D4
:10E15000434C9EAB8DAB0FB6F894DEBF0FBECDBF68
:10E160000C94F75881E08CAF81E090E00E94288702
:10E170009EAF8DAF25E3DC012C9382ED97E09F935A
:10E180008F930E94434C9EAB8DAB0F900F900C94DD
:10E19000F75811E01CAF81E090E00E9428879EAF05
:10E1A0008DAF26E3FC01208319AF82E090E00E944E
:10E1B00028877C019BAF8AAF81E090E00E9428878E
:10E1C000D7018D939C93FC011083BE016F5F7F4F3D
:10E1D00081E00E94033B9F938F9380EC97E09F9395
:10E1E0008F930E94434C9EAB8DAB0F900F900F907E
:10E1F0000F900C94F758DA011696ED91FC9101906E
:10E20000F081E02DD08082E089AF84E090E00E9430
:10E2100028877C019BAF8AAF85E090E00E94288729
:10E220008C01F7019183808381E090E00E94288730
:10E23000D70113969C938E931297F801D082118286
:10E24000128213821482FC011082BE016F5F7F4F25
:10E250008D2D0E94033B1F9227E02F939F938F9356
:10E2600087E997E09F938F930E94434C9EAB8DABC1
:10E270000F900F900F900F900F900F900C94F758F5
:10E280001F920F920FB60F9211240BB60F922F937D
:10E290003F934F935F936F937F938F939F93AF932E
:10E2A000BF93EF93FF93E0913F07F09140073097C2
:10E2B00009F01995FF91EF91BF91AF919F918F91C7
:10E2C0007F916F915F914F913F912F910F900BBE76
:10E2D0000F900FBE0F901F9018951F920F920FB6C0
:10E2E0000F9211242F933F938F939F93AF93BF93DC
:10E2F0008091BD069091BE06A091BF06B091C00668
:10E300003091BC0623E0230F2D3758F50196A11D4F
:10E31000B11D2093BC068093BD069093BE06A093CA
:10E32000BF06B093C0068091C1069091C206A0912D
:10E33000C306B091C4060196A11DB11D8093C1060C
:10E340009093C206A093C306B093C406BF91AF9149
:10E350009F918F913F912F910F900FBE0F901F9023
:10E36000189526E8230F0296A11DB11DD2CF1F924A
:10E370000F920FB60F9211240BB60F922F933F936B
:10E380004F935F936F937F938F939F93AF93BF93BD
:10E39000EF93FF93E0911B02F0911C021995FF91FE
:10E3A000EF91BF91AF919F918F917F916F915F910D
:10E3B0004F913F912F910F900BBE0F900FBE0F907A
:10E3C0001F9018951F920F920FB60F9211240BB643
:10E3D0000F922F933F934F935F936F937F938F93FE
:10E3E0009F93AF93BF93EF93FF93E0911902F09146
:10E3F0001A021995FF91EF91BF91AF919F918F9163
:10E400007F916F915F914F913F912F910F900BBE34
:10E410000F900FBE0F901F9018951F920F920FB67E
:10E420000F9211240BB60F922F933F934F935F934C
:10E430006F937F938F939F93AF93BF93EF93FF93CC
:10E44000E0910F02F09110021995FF91EF91BF91A9
:10E45000AF919F918F917F916F915F914F913F917C
:10E460002F910F900BBE0F900FBE0F901F9018951D
:10E470001F920F920FB60F9211240BB60F922F938B
:10E480003F934F935F936F937F938F939F93AF933C
:10E49000BF93EF93FF93E0910D02F0910E02199557
:10E4A000FF91EF91BF91AF919F918F917F916F916C
:10E4B0005F914F913F912F910F900BBE0F900FBE28
:10E4C0000F901F9018951F920F920FB60F92112464
:10E4D0000BB60F922F933F934F935F936F937F935E
:10E4E0008F939F93AF93BF93EF93FF93E0911702A6
:10E4F000F09118021995FF91EF91BF91AF919F9103
:10E500008F917F916F915F914F913F912F910F90DC
:10E510000BBE0F900FBE0F901F9018951F920F9279
:10E520000FB60F9211240BB60F922F933F934F9378
:10E530005F936F937F938F939F93AF93BF93EF936B
:10E54000FF93E0911502F09116021995FF91EF915A
:10E55000BF91AF919F918F917F916F915F914F91FB
:10E560003F912F910F900BBE0F900FBE0F901F90F9
:10E5700018951F920F920FB60F9211240BB60F929F
:10E580002F933F934F935F936F937F938F939F93BB
:10E59000AF93BF93EF93FF93E0911302F0911402B6
:10E5A0001995FF91EF91BF91AF919F918F917F91BD
:10E5B0006F915F914F913F912F910F900BBE0F90F4
:10E5C0000FBE0F901F9018951F920F920FB60F92CB
:10E5D00011240BB60F922F933F934F935F936F933A
:10E5E0007F938F939F93AF93BF93EF93FF93E091AC
:10E5F0001102F09112021995FF91EF91BF91AF9125
:10E600009F918F917F916F915F914F913F912F914A
:10E610000F900BBE0F900FBE0F901F9018951F927A
:10E620000F920FB60F9211240BB60F922F933F93B8
:10E630004F935F936F937F938F939F93AF93BF930A
:10E64000EF93FF93E091EB07F091EC07309709F01F
:10E650001995FF91EF91BF91AF919F918F917F910C
:10E660006F915F914F913F912F910F900BBE0F9043
:10E670000FBE0F901F9018951F920F920FB60F921A
:10E6800011240BB60F922F933F934F935F936F9389
:10E690007F938F939F93AF93BF93EF93FF93E091FB
:10E6A000F507F091F607309709F01995FF91EF9172
:10E6B000BF91AF919F918F917F916F915F914F919A
:10E6C0003F912F910F900BBE0F900FBE0F901F9098
:10E6D00018951F920F920FB60F9211240BB60F923E
:10E6E0002F933F934F935F936F937F938F939F935A
:10E6F000AF93BF93EF93FF93E091FF07F091000872
:10E70000309709F01995FF91EF91BF91AF919F91CB
:10E710008F917F916F915F914F913F912F910F90CA
:10E720000BBE0F900FBE0F901F9018951F920F9267
:10E730000FB60F9211240BB60F922F933F934F9366
:10E740005F936F937F938F939F93AF93BF93EF9359
:10E75000FF938091B900887F803609F44DC008F09E
:10E7600040C0883209F4A9C028F5803109F49DC061
:10E77000C8F4882309F4FBC0883009F496C0FF91DF
:10E78000EF91BF91AF919F918F917F916F915F9129
:10E790004F913F912F910F900BBE0F900FBE0F9096
:10E7A0001F901895883109F488C0803241F7809312
:10E7B000130714C0803409F49DC040F48033B9F3CA
:10E7C0008833E9F68093130785ECB0C0803509F4EF
:10E7D00085C0883509F496C0883489F60E940D4DAD
:10E7E000CECF883909F48CC038F5883729F050F439
:10E7F000883611F0803719F683E080931507109260
:10E80000680457C0883809F47BC0803919F0803813
:10E8100009F0B5CF80916804803208F071C0E091B2
:10E82000680481E08E0F809368048091BB00F0E063
:10E83000E85BFB4F80833DC0803B39F0E0F4803AD9
:10E8400009F479C0883A09F09ACF84E080931507DB
:10E850001092470410924604E0911906F0911A06AE
:10E8600019958091460481110FC081E08093460480
:10E870001092260409C0803C09F4A6CF883C09F414
:10E88000A3CF883B09F07BCFE091470481E08E0F56
:10E8900080934704F0E0EA5DFB4F80818093BB00EA
:10E8A000909147048091460429C08091F00680939E
:10E8B000BB0085EC8093BC0062CF909112078091E1
:10E8C0001107981758F5E091120781E08E0F809399
:10E8D0001207F0E0EF50F94F8081E9CFE091120785
:10E8E00081E08E0F809312078091BB00F0E0EF5023
:10E8F000F94F808390911207809111079817C8F201
:10E9000085E8D8CFE091120781E08E0F809312073F
:10E910008091BB00F0E0EF50F94F808380911407A5
:10E9200081115CCF81E08093EF0684EA8093BC0084
:10E930001092150724CF85EC8093BC001092150728
:10E9400080916804803230F4E0916804F0E0E85B84
:10E95000FB4F10826091680470E0E0911706F0911F
:10E96000180688E494E019951092680408CF109274
:10E97000130734CF1F920F920FB60F9211240BB6CC
:10E980000F922F933F934F935F936F937F938F9348
:10E990009F93AF93BF93EF93FF9360E085E29AE27A
:10E9A0000E94891E809106018695869580958F70BC
:10E9B0008093E70320E044E150E060E070E085E20E
:10E9C0009AE20E94011FFF91EF91BF91AF919F9139
:10E9D0008F917F916F915F914F913F912F910F9008
:10E9E0000BBE0F900FBE0F901F901895AF92BF9265
:10E9F000CF92DF92EF92FF920F931F93CF93DF930B
:10EA0000CDB7DEB765970FB6F894DEBF0FBECDBFAA
:10EA1000288739874A875B876C877D878E87AF8693
:10EA2000B88AC98ADA8AEB8AFC8A0D8B0091410682
:10EA300010914206822F8A258F7009F062C02295BC
:10EA40002F70932F832F81708295807F282BA29423
:10EA50008FE0A8223B2D31703295307FA32A2A11F6
:10EA600050C0292F2B252E7709F04BC0292F221FAC
:10EA70002227221F942F9F71990F922B2B2D221F3B
:10EA80002227221F8C2D8F71880F822B981339C05B
:10EA9000852F8D258F77A9F5D7FAFF24F0F887E029
:10EAA000FE013896DE01119601900D928A95E1F7EC
:10EAB00029813A814B815C816D817E818F810E94A9
:10EAC0004214BC019C81F0FA97F99C838B898D8359
:10EAD0008C898E838D898F83CE0101960E94DB16EF
:10EAE00065960FB6F894DEBF0FBECDBFDF91CF9114
:10EAF0001F910F91FF90EF90DF90CF90BF90AF905C
:10EB00000895288539854A855B856C857D858E8548
:10EB10000E9442147C018FEFE816F80609F4C3C086
:10EB2000C7010E9418122091410630914206281711
:10EB3000390709F05CC011E080913F0690914006D2
:10EB400020914106309142062E153F0508F048C03D
:10EB5000B701685071096817790709F441C0CE01FF
:10EB600001960E943912882309F48AC08981982F5E
:10EB70009F709A30A8F5982F92959F703A81832FB5
:10EB800081708295807F892B883150F5432F46957F
:10EB90004F734C3328F5932F991F9927991F3B8169
:10EBA0003F71330F392B9889592F56955F73692F11
:10EBB000661F6627661F29892F71220F262B6F85F6
:10EBC00062956F7091709295907F962B891B29F4B6
:10EBD000842F851B11F4832F821B18160CF450C050
:10EBE000112309F44DC0B701CE010F9677CFBC01B8
:10EBF000CE0101960E94391210E0882309F49CCFBF
:10EC00008981982F9F709A3008F095CF982F929510
:10EC10009F703A81832F81708295807F892B883104
:10EC200008F089CF432F46954F734C3308F083CFBC
:10EC3000932F991F9927991F3B813F71330F392BD0
:10EC40009889592F56955F73692F661F6627661F2F
:10EC500029892F71220F262B6F8562956F70917015
:10EC60009295907F962B891B29F4842F851B11F494
:10EC7000832F821B8095182F111F1127111F5CCF26
:10EC8000288539854A855B856C857D858E850E94C2
:10EC90004F182F85388949895A896B897C898D89D4
:10ECA0000E946B171DCF82E01BCF0F931F93CF9352
:10ECB000DF938B0160912B0670912C060E94232418
:10ECC000EC0182E0CF3FDC07A9F060912B06709148
:10ECD0002C06C8010E9423248F3F980719F0C817FB
:10ECE000D90769F4E0912706F0912806B801CE0112
:10ECF000199580E0DF91CF911F910F91089583E0E6
:10ED0000F9CFEF92FF920F931F93CF93DF93CDB77D
:10ED1000DEB76E970FB6F894DEBF0FBECDBF7C0195
:10ED200000912B0610912C06B8010E942324019615
:10ED300089F5E0912506F0912606BE016F5F7F4FB1
:10ED4000C8011995CE0101960E948B23811115C02F
:10ED5000E0912706F0912806B701C801199580E0D7
:10ED60006E960FB6F894DEBF0FBECDBFDF91CF9188
:10ED70001F910F91FF90EF900895C8010E949A2370
:10ED80008C0180912B0690912C068017910789F6B3
:10ED900081E0E6CF83E0E4CFEFE3F7E085E393E0C3
:10EDA00091878087118210821092490710924A073A
:10EDB00010924B0710924C07E1E5F7E08AE9DF017A
:10EDC0001D928A95E9F7EBEEF7E08AE493E09187EC
:10EDD000808711821082E5EFF7E08FE593E091875D
:10EDE000808711821082EFEFF7E084E793E091874C
:10EDF000808711821082E9E0F8E01382128288EEA7
:10EE000093E0A0E0B0E084839583A683B7838DE888
:10EE100093E091838083E0ECF8E0138212828FE923
:10EE200093E09183808388E084838FEF858389E0FA
:10EE3000868384E0878385E0808786E0818787E01A
:10EE400082871386148615861686178681E00E94AF
:10EE5000CB3487E590E090931A08809319081092BC
:10EE6000150810921608109217081092180889E8D1
:10EE700098E00E94B23182E598E00E94B2318BE1C5
:10EE800098E00C94B231CF93DF93CDB7DEB7CA5A76
:10EE9000D1090FB6F894DEBF0FBECDBF789484B50C
:10EEA000826084BD84B5816084BD85B5826085BD86
:10EEB00085B5816085BD80916E00816080936E0014
:10EEC0001092810080918100826080938100809106
:10EED00081008160809381008091800081608093B7
:10EEE00080008091B10084608093B1008091B00077
:10EEF00081608093B0008091910082608093910046
:10EF00008091910081608093910080919000816058
:10EF1000809390008091A10082608093A1008091F5
:10EF2000A10081608093A1008091A0008160809306
:10EF3000A0008091210182608093210180912101B4
:10EF40008160809321018091200181608093200164
:10EF500080917A00846080937A0080917A00826048
:10EF600080937A0080917A00816080937A0080910A
:10EF70007A00806880937A001092C10083B7817F05
:10EF800083BF809164008F6E8093640080916500E0
:10EF90008F6380936500809164008F7D809364000F
:10EFA00080916400877F8093640080916500877FF3
:10EFB00080936500809165008F7E809365008091CD
:10EFC00065008F7D80936500809164008F778093CA
:10EFD000640061E08AE00E947A0F61E08DE00E94A7
:10EFE0007A0F61E08BE00E947A0F60E083E10E947B
:10EFF0007A0F62E080E40E947A0F62E081E40E946E
:10F000007A0F62E082E40E947A0F62E083E40E9459
:10F010007A0F60E08AE00E944C0F82E00E94CB34BD
:10F0200088E0EDE3F2E0DE01AC57BF4F01900D92B6
:10F030008A95E1F7BE016C577F4F80E00E947F35D3
:10F0400088E0E5E4F2E0DE01A458BF4F01900D92A4
:10F050008A95E1F7BE0164587F4F81E00E947F35B9
:10F0600088E0EDE4F2E0DE01AC58BF4F01900D9274
:10F070008A95E1F7BE016C587F4F82E00E947F3590
:10F0800088E0E5E5F2E0DE01A459BF4F01900D9262
:10F090008A95E1F7BE0164597F4F83E00E947F3576
:10F0A00088E0EDE5F2E0DE01AC59BF4F01900D9232
:10F0B0008A95E1F7BE016C597F4F84E00E947F354D
:10F0C00088E0E5E6F2E0DE01A45ABF4F01900D9220
:10F0D0008A95E1F7BE01645A7F4F85E00E947F3533
:10F0E00088E0EDE6F2E0DE01AC5ABF4F01900D92F0
:10F0F0008A95E1F7BE016C5A7F4F86E00E947F350A
:10F1000088E0E5E7F2E0DE01A45BBF4F01900D92DD
:10F110008A95E1F7BE01645B7F4F87E00E947F35EF
:10F12000EEE7F4E010823F9645E0EE36F407D1F7C3
:10F1300087E190E037E02EEF389FF001399FF00D26
:10F140001124E159FA4F20830197B0F78FEF809394
:10F150006E0501E010E02AE040E057EF6FE370E059
:10F160008FE397E00E94BB0E81E99DE190934007F9
:10F1700080933F07E0914707F09148070684F785A1
:10F18000E02D81E080837894E0914707F091480773
:10F190000280F381E02D808190914307892B808349
:10F1A0001092CE061092CD0610921C0710923E07C8
:10F1B0000E94CF2081E490E190931A068093190673
:10F1C00082E490E190931806809317068DEF9AE2FF
:10F1D000909324068093230680911F069091200629
:10F1E000A0912106B091220680931B0690931C06E5
:10F1F000A0931D06B0931E060E942E208EE00E9452
:10F200003B2B682F64608EE00E94722381E00E9495
:10F210005F2B82E00E945F2B8EE00E943B2B682FC9
:10F2200061608EE00E947223F8948091680084608F
:10F230008093680010926D0080916D008C638093C4
:10F240006D00789489E390E1909316028093150203
:10F25000809169008F7C806280936900EA9A0E94A5
:10F260002E206093B8067093B9068093BA069093E7
:10F27000BB0610922C0610922B0680EE91E0909324
:10F280002A068093290684EE9BE4909328068093B7
:10F2900027068EEB96E3909326068093250680E062
:10F2A00092E090932F0680932E0686E080932D06A1
:10F2B00086E48093300686E1E7E2F2E0DE01119613
:10F2C00001900D928A95E1F7CE0101967C016E01C5
:10F2D00097E1C90ED11CF70111917F018091300691
:10F2E000181708F458C0EEEFE10FE23408F059C0E7
:10F2F000F0E08827E158F6488F4F0C9496838D7A7A
:10F30000C179517A547A577A5A7A5D7A607A637AF7
:10F31000667A697A6C7AD179D179D179D179D179D2
:10F320006F7A727A757AD179D179D179D179D179A7
:10F33000D179D179D179D179D179D179D179D1797D
:10F34000D179D179D179D179D179D179D179D1796D
:10F35000D179787A7B7A7E7AD179D179D179D1795C
:10F36000D179D179D179D179D179D179D179D1794D
:10F37000D179D179D179D179D179817A847A877A21
:10F380008A7A62E076E180913006181750F4812F76
:10F390000E94F43706C0812F0E94C536882309F4E5
:10F3A000A2CFCE14DF0409F096CF4EE050E060E02B
:10F3B00078E08AEA96E00E94DF821091B306812FFE
:10F3C0008F770E94BB26882319F01F671093B3061E
:10F3D0000091B306902F991F9927991F1091B40699
:10F3E000812F8F73880F892B0E94BB26882331F0D1
:10F3F00000680093B3061F631093B4060091B4062F
:10F40000902F92959695969593701091B506812FB1
:10F410008F71880F880F892B0E94BB26882331F0BB
:10F42000006C0093B4061F611093B5060091B506F9
:10F43000902F9295969597701091B606812F8F70A8
:10F44000880F880F880F892B0E94BB26882331F0F4
:10F45000006E0093B5061F601093B6068091B70644
:10F46000982F987709F4D3C4F82EF694F694F6946E
:10F47000FF2DFF70FF2E1091B606912F92959F7071
:10F48000182F17701295107F192B00E0F01609F451
:10F49000BEC4802F810F0E94BB268111B3C40F5FB1
:10F4A000F5CF6BEF75E16FCF64EF75E16CCF6DEE6B
:10F4B00075E169CF66EE75E166CF6FED75E163CFFB
:10F4C00068ED75E160CF61ED75E15DCF6BEC75E1E5
:10F4D0005ACF65EC75E157CF6EEB75E154CF66EB13
:10F4E00075E151CF6EEA75E14ECF66EA75E14BCF1B
:10F4F00060EA75E148CF6AE975E145CF64E975E1F5
:10F5000042CF6DE875E13FCF64E875E13CCF6BE732
:10F5100075E139CF6EE076E136CF68E076E133CF42
:10F52000EAE5F6E08AEA96E02FEF20831182128264
:10F530001382148235968E179F07B9F747E050E083
:10F5400060EE71E083E596E00E94DF822091AA06DA
:10F55000122F1695169517704EE2E42E43E0F42E06
:10F5600055E3C52E53E0D52E61E0F70181917F016F
:10F570000E947A0FCE14DF04B9F78DE390E19093E7
:10F58000C8068093C70681E08093CC0610924E0790
:10F5900010924D071092500710924F0784E694E4A2
:10F5A0009093CA068093C90684EA9FE19093C606A9
:10F5B0008093C506212F30E02F5F3F4F032E000CB4
:10F5C000440B550B60E47FE180E090E00E9477837C
:10F5D00069017A0110E000E02DE0BA01A6018FEF89
:10F5E00097E00E94BB0E2DE0B701A6018BEE97E0DD
:10F5F0000E94BB0E2DE0B701A60185EF97E00E94A7
:10F60000BB0E36E1D32EC8018D5A994F7C01FC0107
:10F61000808186958695BE01615E7F4F8F710E94C5
:10F62000D223811114C0D09ED001D19EB00D1124DF
:10F63000FE01B796AF5AB84F8D2D01900D928A9565
:10F64000E1F7F70160816170802F0E94B7240F5F9E
:10F650001F4F07301105B9F680E00E94BF338FE0DD
:10F66000EDE7F2E0DE01DD9601900D928A95E1F77B
:10F6700085E08093330665E070E083E090E00E94CF
:10F680000C878093310690933206DE01DD96FC01F3
:10F690000F962D913D914D91219331934193E81710
:10F6A000F907B9F7109242061092410680EF9FE0E9
:10F6B0009093400680933F0684EE97E290933E0637
:10F6C00080933D0680EC99E290933C0680933B0644
:10F6D0008BE995E390933A06809339068EE99BE295
:10F6E00090933806809337060E94E427609334068F
:10F6F000709335068093360686E398E5909344062A
:10F700008093430685E49DE49093460680934506E6
:10F710008AE196E390934C0680934B0681E795E34C
:10F7200090934A068093490689EC94E390934806A7
:10F730008093470684E09BE490934E0680934D06A9
:10F7400084EC97E89093500680934F068EE1ECE8A6
:10F75000F2E0DE01119601900D928A95E1F762E0E8
:10F7600070E08FE090E00E940C87809351069093A8
:10F770005206DE011196FC014E962D913D9121938A
:10F7800031938E179F07C9F70AB402FE32C08BE28D
:10F7900096E19F938F938091BB068F938091BA06D9
:10F7A0008F938091B9068F938091B8068F9383E0F1
:10F7B0008F930E94D443CF55DF4F2883C15AD04046
:10F7C000CE55DF4F3883C25AD040CD55DF4F4883E6
:10F7D000C35AD040CC55DF4F5883C45AD040CB5584
:10F7E000DF4F6883C55AD0400FB6F894DEBF0FBE16
:10F7F000CDBF0AB403FE32C081E296E19F938F939E
:10F800008091BB068F938091BA068F938091B90641
:10F810008F938091B8068F9383E08F930E94D44397
:10F82000CA55DF4F2883C65AD040C955DF4F3883A9
:10F83000C75AD040C855DF4F4883C85AD040C75533
:10F84000DF4F5883C95AD040C655DF4F6883CA5A24
:10F85000D0400FB6F894DEBF0FBECDBF1EBA1ABCA3
:10F860001EBA8091AC0685FF3AC08091060186954C
:10F87000869580958F7009F44CC088E196E19F933E
:10F880008F938091BB068F938091BA068F9380915E
:10F89000B9068F938091B8068F9381E08F930E9471
:10F8A000D443C457DF4F2883CC58D040C357DF4FD1
:10F8B0003883CD58D040C257DF4F4883CE58D04010
:10F8C000C157DF4F5883CF58D040C057DF4F6883B0
:10F8D000C059D0400FB6F894DEBF0FBECDBF88E14F
:10F8E00099E20FB6F894A895809360000FBE9093AC
:10F8F0006000809160008F7B80936000F79A00E049
:10F9000010E00E94504701151105D9F30E94000034
:10F91000F8CF0E94E427D62E072F182F962F9F701E
:10F92000F92EE1E027E0A22E9E1741F08EEF890F1D
:10F93000AA24AA94A90E863008F0A92E0E941513B5
:10F94000C656DF4F2883CA59D040C556DF4F38838B
:10F95000CB59D040C456DF4F4883CC59D040C35612
:10F96000DF4F5883CD59D040C256DF4F6883CE5900
:10F97000D040C156DF4F7883CF59D040C056DF4FBB
:10F980008883C05AD040922F92959F70832F8170A8
:10F990008295807F892B36953F732F702A3008F02F
:10F9A0009ECF883108F09BCF3C3308F098CF87E09A
:10F9B000FE01E656FF4FDE01A457BF4F01900D92A6
:10F9C0008A95E1F7E12CF12FFF71CF2ECC0C802F1F
:10F9D000881F8827881FC82A402F4170B42EB294F0
:10F9E00090EFB9228D2D82958F70B82AC157DF4FC5
:10F9F0008881CF58D04087FD69C0C357DF4F9881B9
:10FA0000CD58D040492F46954F73892F881F88279E
:10FA1000881FC257DF4F2881CE58D0402F71220F48
:10FA2000282B302F36953F73C457DF4F8881CC5831
:10FA3000D040582F52955F70892F81708295807FBA
:10FA4000852B8B1929F4842F831B11F4822F8C1999
:10FA50001816E4F5C457DF4F8881CC58D0406A2D82
:10FA60008F700E94A011882389F1C157DF4F9881C0
:10FA7000CF58D0409F7729F02DEF290F223008F082
:10FA8000A1C1C457DF4F2881CC58D040C357DF4FA6
:10FA90003881CD58D040C257DF4F4881CE58D04032
:10FAA000C157DF4F5881CF58D040C057DF4F6881D2
:10FAB000C059D040CF56DF4F7881C159D040CE5683
:10FAC000DF4F8881C259D0400E94E011C457DF4FF8
:10FAD0002881CC58D040C357DF4F3881CD58D04013
:10FAE000C257DF4F4881CE58D040C157DF4F5881B1
:10FAF000CF58D040C057DF4F6881C059D040CF5653
:10FB0000DF4F7881C159D040CE56DF4F8881C2592E
:10FB1000D0400E946F16C457DF4F2883CC58D04086
:10FB2000C357DF4F3883CD58D040C257DF4F48838B
:10FB3000CE58D040C157DF4F5883CF58D040C05720
:10FB4000DF4F6883C059D040CF56DF4F7883C1590B
:10FB5000D040CE56DF4F8883C259D040922F929525
:10FB60009F70832F81708295807F892B36953F739C
:10FB70002F702A3078F4883168F43C3358F4BE0191
:10FB800066567F4FCE0184579F4F0E94C511882330
:10FB900009F42CCF87E0FE01E656FF4FDE01A457A3
:10FBA000BF4F01900D928A95E1F71F71110F802FC1
:10FBB000881F8827881F182BD2948FE0D822802F87
:10FBC00081708295807FD82AC157DF4F8881CF58B6
:10FBD000D04087FD69C0C357DF4F2881CD58D04042
:10FBE000422F46954F73922F991F9927991FC257FD
:10FBF000DF4F8881CE58D0408F71880F892B302FEE
:10FC000036953F73C457DF4F9881CC58D040592F59
:10FC100052955F70922F91709295907F952B9D19C0
:10FC200029F4942F931B11F4982F911B1916E4F1CA
:10FC3000C457DF4F8881CC58D0406F2D8F700E9401
:10FC4000A011882389F1C157DF4F9881CF58D04048
:10FC50009F7729F02DEF290F223008F0C3C0C45739
:10FC6000DF4F2881CC58D040C357DF4F3881CD5863
:10FC7000D040C257DF4F4881CE58D040C157DF4FE8
:10FC80005881CF58D040C057DF4F6881C059D0400D
:10FC9000CF56DF4F7881C159D040CE56DF4F888193
:10FCA000C259D0400E94E011C457DF4F2881CC5880
:10FCB000D040C357DF4F3881CD58D040C257DF4FB7
:10FCC0004881CE58D040C157DF4F5881CF58D040DF
:10FCD000C057DF4F6881C059D040CF56DF4F788181
:10FCE000C159D040CE56DF4F8881C259D0400E94C2
:10FCF0006F16C457DF4F2883CC58D040C357DF4F0F
:10FD00003883CD58D040C257DF4F4883CE58D040BB
:10FD1000C157DF4F5883CF58D040C057DF4F68835B
:10FD2000C059D040CF56DF4F7883C159D040CE560E
:10FD3000DF4F8883C259D040922F92959F70832FB6
:10FD400081708295807F892B36953F732F702A3082
:10FD500078F4883168F43C3358F4BE0166567F4F1E
:10FD6000CE0184579F4F0E94C511882309F42CCFE0
:10FD7000EE2009F4B4CD81E0C756DF4F8883C9591E
:10FD8000D040CD56DF4F2881C359D040CC56DF4FED
:10FD90003881C459D040CB56DF4F4881C559D04037
:10FDA000CA56DF4F5881C659D040C956DF4F6881C7
:10FDB000C759D040C856DF4F7881C859D0400E94FB
:10FDC000E0118DCD913009F081CE97E0FE01E4572E
:10FDD000FF4FDE01AD56BF4F01900D929A95E1F7AE
:10FDE000E82E74CE913009F05FCF97E0FE01E45722
:10FDF000FF4FDE01AD56BF4F01900D929A95E1F78E
:10FE0000E82E52CF8091B70687788093B70680910D
:10FE1000AC0682FF12C08091AE06863420F4809139
:10FE2000AF06863450F08091AC068B7F8093AC0691
:10FE300088E28093AE068093AF068091AC0683FF84
:10FE400012C08091B106863420F48091B2068634C7
:10FE500050F08091AC06877F8093AC0688E2809357
:10FE6000B1068093B2068091B3068F778F3779F011
:10FE70006091AC0666FB662760F991E069270E94F5
:10FE80004C0F8091B30661E08F770E947A0F6091EA
:10FE9000B306862F881F8827881F6091B4066F736A
:10FEA000660F682B89E898E00E94F5306091B406EF
:10FEB000862F82958695869583706091B5066F71C1
:10FEC000660F660F682B82E598E00E94F53060911E
:10FED000B506862F8295869587706091B6066F70FD
:10FEE000660F660F660F682B8BE198E00E94F53075
:10FEF00000E08091B706982F9695969596959F70FD
:10FF0000091708F00DCB1091B606912F92959F70AE
:10FF1000182F17701295107F192B100F61E0812F89
:10FF20000E947A0F6091B7066095661F6627661F6C
:10FF3000812F0E944C0F0F5FDCCFFC01882799278F
:10FF4000E89421912032E9F3293010F02E30C8F3E3
:10FF50002B3241F02D3239F4689404C00E94BB7FEB
:10FF6000820F911D219120532A30C0F31EF49095E9
:10FF700081959F4F08957AE0979F902D879F802DC0
:10FF8000910D112408950F931F93CF93DF93CDB755
:10FF9000DEB72E970FB6F894DEBF0FBECDBF0E8929
:10FFA0001F89888D998D2EE02C831A83098397FFF2
:10FFB00002C080E090E801979E838D83AE01445E8D
:10FFC0005F4F6A8D7B8DCE0101960E9439804D81F5
:10FFD0005E8157FD0AC02F813885421753070CF404
:10FFE0009A01020F131FF80110822E960FB6F89493
:10FFF000DEBF0FBECDBFDF91CF911F910F9108954E
:020000021000EC
:100000000F931F93CF93DF93CDB7DEB72E970FB625
:10001000F894DEBF0FBECDBF8C01FA018EE08C8359
:100020001A83098377FF02C060E070E861507109AC
:100030007E836D83A901BF01CE0101960E943980A4
:100040004D815E8157FD0AC02F81388542175307C5
:100050000CF49A01020F131FF80110822E960FB6AE
:10006000F894DEBF0FBECDBFDF91CF911F910F91EE
:1000700008952F923F924F925F926F927F928F924C
:100080009F92AF92BF92CF92DF92EF92FF920F9327
:100090001F93CF93DF9300D000D000D01F921F9208
:1000A000CDB7DEB77C013B018A01FC0117821682C5
:1000B000838181FFDDC1CE0101965C01F70193814F
:1000C000F30193FD859193FF81913F01882309F40A
:1000D00053C1853239F493FD859193FF81913F019E
:1000E000853229F4B70190E00E945182E7CF912C2C
:1000F000212C312CFFE1F31538F08B3211F190F403
:10010000803209F1833229F137FC3CC020ED280F01
:100110002A3050F536FE20C08AE0989E200D11242A
:10012000922E06C08D3291F0803371F7689430F8CA
:10013000F30193FD859193FF81913F018111DACF06
:1001400021C0689431F8689432F8F2CF689433F89B
:10015000EFCF689434F8ECCFEAE02E9E200D112406
:10016000222E689435F8E4CF8E3229F436FC04C18F
:10017000689436F8DDCF8C3619F4689437F8D8CF08
:100180008836B1F2982F9F7D95549330E0F08336F6
:10019000A1F18337C1F1833509F063C02801F2E092
:1001A0004F0E511CF801C080D180692D70E036FCE3
:1001B00002C06FEF7FEFC6010E943B824C01689442
:1001C00037F882010AC00C5F1F4FFFE3F9838824D0
:1001D0008394912C6501E89437F833FE2DC0522C9E
:1001E0008114910471F5552009F468CFB70180E2BC
:1001F00090E00E9451825A94F6CFF8018081898361
:100200000E5F1F4FE4CF2801F2E04F0E511CF801A2
:10021000C080D180692D70E036FC02C06FEF7FEFA7
:10022000C6010E9446824C018201D5CFB70180E20F
:1002300090E00E9451822A942814190409F0B0F722
:10024000CECFF60137FC859137FE81916F01B70162
:1002500090E00E94518251105A94F1E08F1A910857
:10026000BFCF843619F0893609F077C0F80137FE20
:100270006BC060817181828193810C5F1F4FF32D70
:10028000FF763F2E97FF09C09095809570956195F8
:100290007F4F8F4F9F4F689437F82AE030E0A501D9
:1002A0000E948182C82ECA188C2C432C36FE0CC0AA
:1002B000E89440F8C91440F434FE05C032FC03C091
:1002C000F32DFE7E4F2E892C44FEAAC0FE01EC0DBC
:1002D000F11D8081803309F09CC0242D297E422E9F
:1002E000842D8870582E43FCAAC040FEA4C09C2CCC
:1002F000821418F42C0C922C981844FEA6C0B70156
:1003000080E390E00E94518242FE09C088E790E0BD
:1003100041FE02C088E590E0B7010E945182C914F5
:1003200008F49FC0CA94D12C9FEFC91AD90ACA0CED
:10033000DB1CF60182916F01B70190E00E945182AF
:10034000AC14BD04B1F74FCF60817181072E000C52
:10035000880B990B0E5F1F4F92CFD32CE894D4F8E3
:100360002AE030E08537E1F1232D297FD22E8F3628
:10037000A9F1F0F4883551F1F701868197812B9628
:100380000FB6F894DEBF0FBECDBFDF91CF911F91A6
:100390000F91FF90EF90DF90CF90BF90AF909F9024
:1003A0008F907F906F905F904F903F902F90089527
:1003B000803749F0883701F7D4FE02C06894D2F83C
:1003C00020E130E00DC06894D4F8F6CF34FE03C0CD
:1003D000822F8660D82E20E132E002C028E030E093
:1003E000F801D7FE0FC060817181828193810C5F1B
:1003F0001F4FA5010E948182C82ECA183D2CE89487
:1004000037F852CF6081718190E080E00E5F1F4F1E
:10041000F0CF42FC02C0839463CF8394839460CF77
:10042000842D867809F45CCFF6CFB70180E290E0A6
:100430000E94518283948214C0F3512C5ECF522CBF
:100440005818821408F459CFF8CF842D867809F40F
:1004500066CF8BE241FE80E247FC8DE2B70190E07F
:100460005CCFB70180E390E00E9451829A9457CF0D
:100470008FEF9FEF84CFFC01059061507040011019
:10048000D8F7809590958E0F9F1F0895FC016150BD
:10049000704001900110D8F7809590958E0F9F1FA6
:1004A00008950F931F93CF93DF93182F092FEB011C
:1004B0008B8181FD09C01FEF0FEF812F902FDF91FE
:1004C000CF911F910F91089582FF14C02E813F811B
:1004D0008C819D81281739073CF4E881F981CF018F
:1004E00001969983888310838E819F8101969F83D3
:1004F0008E83E3CFE885F985812F1995892BA1F3A8
:10050000DACFFA01AA27283051F1203181F1E8949D
:100510006F936E7F6E5F7F4F8F4F9F4FAF4FB1E0F6
:100520003ED0B4E03CD0670F781F891F9A1FA11DF1
:10053000680F791F8A1F911DA11D6A0F711D811DF2
:10054000911DA11D20D009F468943F912AE0269FB7
:1005500011243019305D3193DEF6CF010895462F16
:100560004770405D4193B3E00FD0C9F7F6CF462FF7
:100570004F70405D4A3318F0495D31FD4052419360
:1005800002D0A9F7EACFB4E0A6959795879577951D
:100590006795BA95C9F700976105710508959B01A4
:1005A000AC010A2E06945795479537952795BA952D
:1005B000C9F7620F731F841F951FA01D0895DC01EA
:1005C000CB01FC01F999FECF06C0F2BDE1BDF89A5E
:1005D000319600B40D9241505040B8F70895DC01B7
:1005E000A40FB51F4150504048F0CB01840F951F18
:1005F0002E910E94008341505040D0F70895262F3D
:10060000F999FECF92BD81BDF89A019700B4021608
:1006100039F01FBA20BD0FB6F894FA9AF99A0FBEB6
:100620000895DB018F939F930E94B483BF91AF9194
:10063000A29F800D911DA39F900DB29F900D11243C
:100640000895991B79E004C0991F961708F0961B2E
:10065000881F7A95C9F780950895AA1BBB1B51E1A5
:1006600007C0AA1FBB1FA617B70710F0A61BB70B22
:10067000881F991F5A95A9F780959095BC01CD01C7
:10068000089597FB072E16F4009407D077FD09D044
:100690000E942D8307FC05D03EF4909581959F4FD5
:1006A0000895709561957F4F0895A1E21A2EAA1BB7
:1006B000BB1BFD010DC0AA1FBB1FEE1FFF1FA21712
:1006C000B307E407F50720F0A21BB30BE40BF50B0F
:1006D000661F771F881F991F1A9469F76095709598
:1006E000809590959B01AC01BD01CF010895052E29
:1006F00097FB1EF400940E948E8357FD07D00E9442
:10070000558307FC03D04EF40C948E83509540958E
:10071000309521953F4F4F4F5F4F089590958095AD
:10072000709561957F4F8F4F9F4F0895EE0FFF1F7C
:10073000881F8BBF0790F691E02D1994A29FB001FE
:10074000B39FC001A39F700D811D1124911DB29F05
:10075000700D811D1124911D08950E949E83B7FF85
:100760000895821B930B08950E949E83A59F900D70
:10077000B49F900DA49F800D911D11240895B7FF83
:100780000C94B4830E94B483821B930B0895505839
:10079000BB27AA270E94DF830C9491850E94838542
:1007A00038F00E948A8520F039F49F3F19F426F42E
:1007B0000C9459850EF4E095E7FB0C945385E92FD2
:1007C0000E94A28558F3BA1762077307840795073A
:1007D00020F079F4A6F50C94C4850EF4E0950B2E68
:1007E000BA2FA02D0B01B90190010C01CA01A00183
:1007F0001124FF27591B99F0593F50F4503E68F1DE
:100800001A16F040A22F232F342F4427585FF3CF1E
:10081000469537952795A795F0405395C9F77EF4EF
:100820001F16BA0B620B730B840BBAF09150A1F038
:10083000FF0FBB1F661F771F881FC2F70EC0BA0FBE
:10084000621F731F841F48F4879577956795B79546
:10085000F7959E3F08F0B0CF9395880F08F0992741
:10086000EE0F9795879508950E9448840C94918582
:100870000E948A8558F00E94838540F029F45F3FEA
:1008800029F00C94538551110C94C5850C9459850D
:100890000E94A28568F39923B1F3552391F3951B28
:1008A000550BBB27AA2762177307840738F09F5F91
:1008B0005F4F220F331F441FAA1FA9F335D00E2EFE
:1008C0003AF0E0E832D091505040E695001CCAF76B
:1008D0002BD0FE2F29D0660F771F881FBB1F26172E
:1008E00037074807AB07B0E809F0BB0B802DBF0105
:1008F000FF2793585F4F3AF09E3F510578F00C94D4
:1009000053850C94C5855F3FE4F3983ED4F38695F8
:1009100077956795B795F7959F5FC9F7880F911DF4
:100920009695879597F90895E1E0660F771F881FE0
:10093000BB1F621773078407BA0720F0621B730B93
:10094000840BBA0BEE1F88F7E095089529F416F092
:100950000C9453850C94C4850C9459850E94AA85E7
:10096000A8F39638A0F707F80F92E8942BE33AEA39
:1009700048EB5FE70E94A7860F920F920F924DB748
:100980005EB70F920E945D86E4EEF0E00E945C8507
:100990004F915F91EF91FF91E595EE1FFF1F49F099
:1009A000FE57E0684427EE0F441FFA95E1F74195A2
:1009B000550B0E94D7850F9007FE0C94CB850895A8
:1009C0000E94E7846894B1110C94C58508950E9433
:1009D000AA8588F09F5798F0B92F9927B751B0F0A2
:1009E000E1F0660F771F881F991F1AF0BA95C9F7B3
:1009F00014C0B13091F00E94C485B1E008950C9408
:100A0000C485672F782F8827B85F39F0B93FCCF3BA
:100A1000869577956795B395D9F73EF4909580952F
:100A2000709561957F4F8F4F9F4F0895E89409C04F
:100A300097FB3EF490958095709561957F4F8F4F11
:100A40009F4F9923A9F0F92F96E9BB279395F69527
:100A5000879577956795B795F111F8CFFAF4BB0FA5
:100A600011F460FF1BC06F5F7F4F8F4F9F4F16C009
:100A7000882311F096E911C0772321F09EE8872F93
:100A8000762F05C0662371F096E8862F70E060E04F
:100A90002AF09A95660F771F881FDAF7880F9695C8
:100AA000879597F9089597F99F6780E870E060E06F
:100AB00008959FEF80EC0895DF93CF931F930F93DA
:100AC000FF92EF92DF927B018C01689406C0DA2ED0
:100AD000EF010E94A486FE01E894A591259135912D
:100AE00045915591A6F3EF010E94DF83FE01970126
:100AF000A801DA9469F7DF90EF90FF900F911F91B2
:100B0000CF91DF91089500240A941616170618064F
:100B10000906089500240A94121613061406050601
:100B20000895092E0394000C11F4882352F0BB0F92
:100B300040F4BF2B11F460FF04C06F5F7F4F8F4FF5
:100B40009F4F089557FD9058440F551F59F05F3F30
:100B500071F04795880F97FB991F61F09F3F79F0DF
:100B600087950895121613061406551FF2CF469561
:100B7000F1DF08C0161617061806991FF1CF8695E3
:100B80007105610508940895E894BB2766277727C7
:100B9000CB0197F908959B01AC0160E070E080E81B
:100BA0009FE30C9434840C9453850C94FE860E942D
:100BB000AA85D8F39923C9F3940F511DA3F391503B
:100BC000504094F059F0882332F0660F771F881F49
:100BD00091505040C1F79E3F51052CF7880F911D51
:100BE0009695879597F908955F3FACF0983E9CF0F5
:100BF000BB27869577956795B79508F4B16093956F
:100C0000C1F7BB0F58F711F460FFE8CF6F5F7F4F5C
:100C10008F4F9F4FE3CF0C94C58516F00C94FE8642
:100C20000C94598568940C9453850E94AA85A8F366
:100C30009923C1F3AEF3DF93CF931F930F93FF92EA
:100C4000C92FDD2788232AF02197660F771F881F79
:100C5000DAF720E030E040E85FEB9FE3883920F0EE
:100C6000803E38F021968F770E94C883ECE0F1E057
:100C700004C00E94C883E9E3F1E00E945C858B0117
:100C8000BE01EC01FB2E6F5771097595771F880B1C
:100C9000990B0E94188528E132E741E35FE30E9447
:100CA000A486AF2D9801AE01FF900F911F91CF91B7
:100CB000DF910E94DF830C949185FA01DC01AA0F79
:100CC000BB1F9B01AC01BF5728F4222733274427C1
:100CD000507820C0B75190F4AB2F0024469537953B
:100CE0002795011CA395D2F3002071F0220F331F2A
:100CF000441FB395DAF30ED00C94C78361307105AD
:100D0000A0E88A07B94630F49B01AC016627772733
:100D100088279078309621F0208331834283538353
:100D200008950E94A4860C9491850E94838538F0D2
:100D30000E948A8520F0952311F00C9453850C9421
:100D4000598511240C94C5850E94A28570F3959F46
:100D5000C1F3950F50E0551F629FF001729FBB27B2
:100D6000F00DB11D639FAA27F00DB11DAA1F649F4E
:100D70006627B00DA11D661F829F2227B00DA11D01
:100D8000621F739FB00DA11D621F839FA00D611D87
:100D9000221F749F3327A00D611D231F849F600DA8
:100DA000211D822F762F6A2F11249F5750409AF0D1
:100DB000F1F088234AF0EE0FFF1FBB1F661F771F5D
:100DC000881F91505040A9F79E3F510580F00C9428
:100DD00053850C94C5855F3FE4F3983ED4F3869524
:100DE00077956795B795F795E7959F5FC1F7FE2BC8
:100DF000880F911D9695879597F908959F3F31F03B
:100E0000915020F4879577956795B795880F911D38
:100E10009695879597F908950F931F93CF93DF9336
:100E2000869F8001879F100D969F100D1124C80189
:100E30000E942887EC01009729F0A80170E060E08B
:100E40000E944D88CE01DF91CF911F910F9108959F
:100E50000F931F93CF93DF938230910510F482E0BC
:100E600090E0E091DA08F091DB0830E020E0B0E0BB
:100E7000A0E0309799F42115310509F44AC0281BE8
:100E8000390B24303105D8F58A819B8161157105B4
:100E900089F1FB0193838283FE0111C0408151815E
:100EA0000281138148175907E0F04817590799F450
:100EB000109761F012960C93129713961C9332962A
:100EC000CF01DF91CF911F910F9108950093DA0820
:100ED0001093DB08F4CF2115310551F04217530769
:100EE00038F0A901DB019A01BD01DF01F801C1CF92
:100EF000EF01F9CF9093DB088093DA08CDCFFE01A4
:100F0000E20FF31F81939193225031093983288393
:100F1000D7CF2091D8083091D908232B41F42091C4
:100F20002302309124023093D9082093D8082091CD
:100F30002102309122022115310541F42DB73EB72F
:100F40004091250250912602241B350BE091D808D0
:100F5000F091D908E217F307A0F42E1B3F0B2817D6
:100F6000390778F0AC014E5F5F4F2417350748F022
:100F70004E0F5F1F5093D9084093D80881939193E7
:100F80009FCFF0E0E0E09CCFCF93DF930097E9F0B4
:100F9000FC01329713821282A091DA08B091DB082B
:100FA000ED0130E020E01097A1F420813181820F23
:100FB000931F2091D8083091D9082817390709F0D4
:100FC00061C0F093D908E093D808DF91CF910895DC
:100FD000EA01CE17DF07E8F54A815B819E014115E2
:100FE0005105B1F7E901FB83EA8349915991C40F97
:100FF000D51FEC17FD0761F4808191810296840F63
:10100000951FE90199838883828193819B838A83D9
:10101000F0E0E0E012968D919C9113970097B9F55E
:101020002D913C911197CD010296820F931F209133
:10103000D8083091D9082817390739F6309751F573
:101040001092DB081092DA08B093D908A093D80860
:10105000BCCFD383C28340815181840F951FC817B1
:10106000D90761F44E5F5F4F88819981480F591FFE
:10107000518340838A819B8193838283211531052B
:1010800009F0B0CFF093DB08E093DA089ECFFD01C2
:10109000DC01C0CF13821282D7CFDC0101C06D9377
:1010A00041505040E0F70895FB01DC018D91019023
:1010B00080190110D9F3990B0895FB01DC0141500F
:1010C000504048F001900D920020C9F701C01D92D8
:0C10D00041505040E0F70895F894FFCF25
:1010DC00FF00000000FFFFFF1FFFFFFFFF43104357
:1010EC0010431043104310431043104310FFFF00F4
:1010FC00000000DC08800002030405060708090A4A
:10110C000B0C0D1314152C2D2E40414243081408C2
:10111C000304040403000E11150E0E0400000A1F34
:10112C00111F111F00000E1517110E0000040E0ADE
:10113C000E1F1F150401020407010A0C0E00000803
:10114C000C0E0C080000000A0A0A0A0A0001E83317
:10115C00002329022B4B03D72804692946577B3CD3
:10116C003E3F43262140A7395D3648561457F53982
:10117C008E3AB044BF55D138593B0103FF02FFFFF3
:10118C00FF0020291D291A291729142911290E2994
:10119C000B29082905290229FF28FC28F928F628FB
:1011AC00F3285A055705540551054E054B054805BE
:1011BC004505420507010203040506080A0B0D0349
:1011CC0004FFFFFFFFFFFFFF0506FFFFFFFFFFFF11
:1011DC00FFFFFFFFFFFFFFFFFFFFFFFFFFFFFFFF13
:1011EC00FFFFFFFFFFFFFFFFFF0001021F1C1F1E81
:1011FC001F1E1F1F1E1F1E1F5E00BC0077012C2D03
:10120C002E02030B0CA000A100A400A600A800AAAB
:10121C0000AC0072003900060708900091009400A1
:10122C00960098009A009C0071003800050203801B
:10123C000081008400860088008A008C006F0036D4
:10124C00000B0C0D200121012401260128012A018B
:10125C002C0173003A002E2D2C00000000432316A5
:10126C0023B424DF0B0F23FC22ED220000000079B5
:10127C00354410B424B3242020484947480020208A
:10128C00204C4F570053756D700054616E6B0054B9
:10129C00414E4B0053554D5000414D42490059456C
:1012AC0053004E4F0046414B4500525443004F6E85
:0612BC0020004F666600F1
:00000001FF
